:020000040800F2
:1000000000A00020A92F0108BD740008DD1F010811
:10001000BB740008B9740008B77400080000000041
:10002000000000000000000000000000B57400089F
:10003000B374000800000000B1740008837E00085B
:100040001130010811300108113001081130010888
:100050001130010811300108113001081130010878
:100060001130010811300108113001081130010868
:10007000113001082D4B000819D800081130010873
:100080001130010811300108113001081130010848
:10009000ED6C000811300108113001081130010821
:1000A000F97400081DD60008E774000841D600085E
:1000B00011D6000801D60008297500081130010882
:1000C0001130010811300108113001081130010808
:1000D0001130010811D8000809D8000811300108B2
:1000E000917E000811300108DD6C00081130010814
:1000F0000975000811300108197500081130010850
:1001000000000000000000000000000011300108A5
:1001100011300108113001081130010811300108B7
:1001200011300108113001081130010811300108A7
:10013000113001081130010800000000000000002B
:1001400011300108113001081130010800000000D1
:10015000000000000000000000000000000000009F
:1001600000000000000000001130010811300108FB
:100170001130010800000000000000000000000035
:0801800000000000113001082D
:100188002DE9F04F2DED028B754D764B2B60AFB0FE
:1001980000236B6010F06AF918B910F089F90BF0B8
:1001A800E3FF0CF09FF8704B704C1A7842F0010294
:1001B8001A706F4A4FF47001C2F888100022099231
:1001C8000A92226842F4803222600493236803F47E
:1001D80000330A93099B013309930A9B1BB9099BB6
:1001E800B3F5A04FF2D1236813F4003318BF0123ED
:1001F8000A930A9B012B00F089805D4F5D4BFB60E1
:10020800636AAB60636ADFF8A4B1DFF8A481DFF842
:10021800A49143F080736362636943F4FC032EAED8
:10022800636103238DF86A3041F6FF7326F8503D69
:100238004FF09040314604F06BFD4FF6FF734E4887
:10024800ADF86830314604F063FD4C48314604F09F
:100258005FFD4B48314604F05BFD5846314604F0DB
:1002680057FD3146474804F053FD304609F052FD2A
:100278001A9B454AB3FBF2F3444A1360444B454A80
:100288004FF0000AC3F800A0434B5A60F02287F8E9
:1002980023200722C3F808A0404F1A60D8F8083076
:1002A8003B6099E80F0086E80F0063691A9843F4E9
:1002B80000136361636943F4001363614FF4885367
:1002C800ABF828304FF48843ABF828301BA904F06A
:1002D8001FFD1DA91C9804F01BFD642007F0C3FD39
:1002E8004FF4A0722E48514615F085F8E3692D4A5F
:1002F80043F00703E361A36943F4E523A36163695A
:1003080043F4BC03636102F5907E55E0264B12224C
:100318001A606368636063686360636843F480635A
:100328006360636823F47C136360636843F4E813D1
:100338006360236843F08073236022680B4B92014B
:10034800FBD55A6822F003025A605A6842F002024A
:100358005A60636803F00C03082BFAD14DE700BF1D
:100368008801002017BA0008882D002000100240DC
:1003780000ED00E00005FA05000400480008004808
:10038800000C00480014004840420F00601C002088
:10039800641C00203F19010010E000E044290020FF
:1003A800A81C002094970108002002400010004873
:1003B8000413002088770108937B506892F80FC0D7
:1003C80003F00701DB0800EB83038900186A4FF08C
:1003D8000F0A0CFA01FC0AFA01F120EA010119627C
:1003E800196A10324CEA010172451962E4D10022FF
:1003F800B849002353540132122AF9D1DFF814A363
:100408000AF11E02FF2199540133082BF6D1B24A92
:10041800B24B1360DFF800B3B14A039303211170A4
:1004280058460021242214F0E6FF14228BF80020FD
:10043800AC49039B3F6801228BF8182098F805B057
:1004480081F800B0A3F5F071CAF82810A649A3F501
:1004580090730B60A54B03EBCB035B78CAF82C3089
:10046800BB0648BFCAF82C200023A14A40F2DC5141
:1004780022F813100133082BF7D113A800211C22EE
:1004880014F0B9FFBBF10E0F03D00BF0EF03082BEC
:1004980002D101238DF85C3002200AF075FB18B1F7
:1004A8004088003018BF0120C7F340038DF8523050
:1004B800C7F380138DF85430C7F340338DF84C30B0
:1004C800C7F3C03300F001008DF84F3017F4006314
:1004D8008DF8510007D098F8823103F1FF3EDEF124
:1004E800000343EB0E038DF85030C7F300438DF83B
:1004F8005530EB6AB8F84401ADF86000003318BF16
:1005080001238DF85630C7F300538DF85730B8F8EB
:100518004631ADF85A30B8F85231ADF8583007F0D6
:100528000101C7F38043C7F3C002FF0448BF714805
:100538008DF85330B8F8503144BFB0F84C01ADF8DD
:100548006000B3F5FA7FADF85E3084BF0023ADF8E4
:100558006030694898F8D23185F83030002385F842
:10056800313043709DF85C308DF84D10002B8DF8BC
:100578004E200CBF0023022301B902B1013309EB5D
:1005880083094FF0000AD9F810309A1E22330392DB
:100598000593039A32F8023F03924FF6FF72934293
:1005A80000F05E81DAB2190A9DF8553033B11301B3
:1005B8005248C058524B984200F04D819DF8523035
:1005C80053B14E4B4F4F03EB02135868B84203D157
:1005D8001B89012B00F03F819DF84F3053B1474BE9
:1005E800484F03EB02135868B84203D11B89042B08
:1005F80000F031819DF8503053B1404B414F03EB2F
:1006080002135868B84203D11B89022B00F02381DA
:10061800022902D19DF84C3003E0012904D19DF84C
:100628004D30002B00F01781344F9DF857304FEABA
:1006380002194F4433B19DF85C301BB9043A032AC0
:1006480040F2F2800129CBB268D1FF2385F87830D7
:1006580085F87930294BC5F8887003EB09024FF00B
:100668000008517B50688DF86A1002F1080B128956
:10067800ADF868201AA9022285F87C8006938DF8C7
:100688006B2085F83480C5F83880C5F83C80C5F8FB
:100698004080C5F8748085F87A8085F87B8004F0FE
:1006A80037FB069B9BF8021053F80900424604F0FA
:1006B80083F9384610F0CCFA134B1449C5F88C303E
:1006C800134BC5F89030C5F8948038460A1D0DF0D4
:1006D8003DF8C0E094010020C8200020F414002058
:1006E800D9120020500A0020641E0020609D0108D5
:1006F8004812002004130020B90100209497010833
:100708000044014000080048554700081402002032
:100718003548000888010020CC200020022B49D150
:100728005FFA8AF21C2101FB02FC9D4ACDF81CC02D
:1007380002EB0C089B4A88F87DA0012188F87C1000
:1007480002EB09014FF0000B91F80DE0486888F8BA
:100758007EB001F108020989ADF8681088F886B002
:100768001AA9C8F888708DF86AE006928DF86B307F
:1007780004F0CEFA8B4B069A53F8090091785A4642
:1007880004F01AF9384610F063FA854BDDF81CC0FE
:10079800854AC8F88C2003EB0C01844AC8F89020DD
:1007A8008C31C8F894B038460A1D0CF0CFFF0AF116
:1007B800010A50E0032B35D19DF85330DFF8E08172
:1007C800DFF820923BB198F832B0384608214FF64E
:1007D800FF7200231AE0BDF85E2098F832B0BDF829
:1007E8006030B2F5FA7F0BD97149B1FBF2F23846A5
:1007F800082192B204F0B5FA6E4B49F82B000AE0D2
:100808006D49B1FBF2F23846012192B204F0A9FA1F
:100818006A4B49F82B00C36098F83230013388F8E6
:10082800323018E0042B16D195F83180BDF85820E5
:10083800614B93FBF2F23846BDF85A30012192B26F
:1008480004F08FFA95F8313005EB88080133C8F8C1
:100858005C0185F83130039B059A93427FF499AE89
:1008680095F8312085F87C21554A564B92F800E0DE
:10087800AEF117020027022A1F709C461AD8AB6AED
:100888003B44D3ED007AF5EE407AF1EE10FA02D14E
:10089800EB6A63BB26E04C4A07EB02080FCB88E8FB
:1008A8000F009CF8003010370133C02F8CF800304F
:1008B800E5D1EDE7454B13F83E908CF8009003EB3B
:1008C800CE03D3F804A0BAF1000FE1D04F45DFDA28
:1008D8003D4A3B0103EB020853440FCB013788E83C
:1008E8000F00F3E73A4D2B68D80424D41DE0394BA8
:1008F800394A13F83E00107003EBCE035D68002DF3
:10090800F0D000238342EDDAC3EBC3016A18DFF8A5
:10091800D880D2F8009041F8089001EB0807918838
:10092800B9809279BA710133ECE70EF0EF03082B26
:100938002A4B20D122E09CF80020012AF5D9284B27
:1009480003EB0212103210339342EED053ED047AC7
:10095800B6EE007A67EE877A43ED047A53ED057AAE
:1009680067EE877A43ED057A53ED037A67EE877A67
:1009780043ED037AE7E7BEF10E0F09D11A7842F08A
:1009880010021A70BEF1180F30D107F0DFFC2DE00D
:100998001A7822F010021A70BEF1190FF4E700BF9E
:1009A8008801002094970108BD4A00082D470008D7
:1009B80000127A005548000840420F0045480008D8
:1009C800500A00204F1C00208C090020609D01085F
:1009D8004429002054850108F01D0020EC1A00204D
:1009E80094090020781C0020F11D002007F092FCDB
:1009F8002B68A848DFF8C8A2DFF8C8B259035EBF61
:100A0800A54B01221A70049B049A1B7843F0040337
:100A180013704FF40853ADF8683002238DF86B302B
:100A28006369012543F4001331468DF86A50636108
:100A380004F06EF9994B9A4A1A60002007F02CFAD4
:100A4800A36943F48053A361E36843F48053E360EC
:100A580063694FF0904943F400336361D9F820305B
:100A680023F47003C9F82030D9F8203043F4A003E8
:100A7800C9F82030D9F8203023F07063C9F8203045
:100A8800D9F8203043F0A063C9F82030D9F82030D5
:100A980023F07043C9F82030D9F8203043F0A04340
:100AA800C9F82030D9F8203023F47023C9F8203051
:100AB800D9F8203043F4A023C9F82030E0234FF0C0
:100AC80000080327484631461A9302238DF86C30F4
:100AD8008DF86D708DF86E808DF86F8009F090FA42
:100AE8001022484631461A9204928DF86D708DF89E
:100AF8006C508DF86E808DF86F8009F081FAE1688E
:100B080041F48051E160E16821F48051E160654978
:100B1800888820F480500004000C8880888880B27F
:100B280040F480508880088800F4415040F44570B3
:100B380038430880888820F470600004000C40F472
:100B4800E0608880888B20F400600004000C4FF07F
:100B580007098883A1F81090088880B240F0400007
:100B680008805149C1F800A0616941F480216161A0
:100B7800E16941F40011E161216B21F01001216369
:100B8800216B41F010012163DBF8201021F0706126
:100B9800CBF82010DBF8201041F08061CBF8201052
:100BA800DBF8201021F07041CBF82010DBF8201082
:100BB80041F08041CBF820104021022358461A9179
:100BC80031468DF86C308DF86D708DF86E808DF82B
:100BD8006F8009F015FA802158461A91314609F0BC
:100BE8000FFADAF80010314B049A21F00101CAF823
:100BF8000010DAF800002E490140CAF800102D490B
:100C0800CAF81010DAF800102943CAF80010CAF818
:100C18000880CAF80C80CAF80880DAF8081041F48D
:100C28000041CAF80810DAF80010CAF80010DAF81B
:100C3800041021F0784121F40041CAF80410DAF8D0
:100C480000102943CAF800101B4903930E68184680
:100C5800414614F0D0FB022306F4004B06F4006A68
:100C68008DF83D301E40039B8DF83C708DF83E801A
:100C78008DF83F801F4627D010480E950EA909F021
:100C8800BFF906223A7087F8018087F80390BD7093
:100C98001BE000BF00100048B80E0020902D002077
:100CA800397500080030014014120020202100206E
:100CB800FFE0CF007A25E000442900200008004822
:100CC80000540040000400483546BBF1000F0ED028
:100CD8000423BE480E930EA909F092F908233B712C
:100CE8000723FB7101237D711D44BB71EDB2BAF17D
:100CF800000F0DD00223B5480E930EA909F080F914
:100D080007233B73FB7301237D731D44BB73EDB253
:100D18000EA90823AD480E9309F072F909233B7216
:100D280007237D72FB720123BB721D44E36AA84846
:100D380023F4F873E362E36A43F4D873E362636904
:100D480043F0805343F00103636108F02CFF1AA8B5
:100D580008F0FEFE9F4B1A93EDB29F4B1B93012D9B
:100D68004FF000030CBF1A4680221F924FF4807286
:100D7800974C20924FF480622192202220462292A2
:100D88001AA94FF400521C931E9323922493ADF892
:100D9800745008F0EAFE236843F0010323604FF023
:100DA800A0440A20A36823F04053A360A36843F03B
:100DB8008053A36007F057F8A36823F08043A3602B
:100DC800A368A360A36843F00043A3604FF0A04268
:100DD8009368002BFADB9368804923F040539360B3
:100DE800936843F00053936088687D4B034043F455
:100DF80068338B60D1687B4B0B4043F40053D3605E
:100E0800136B013D23F00F031D43156300240123D9
:100E18003A19917800296CD05D1C042B3E5DD0787E
:100E2800EDB24FF0A04E0ED803EB4302DEF83010BF
:100E380052001F23934021EA030106FA02F30B43F1
:100E4800CEF8303031E0092B0ED8053B06225A4344
:100E5800DEF834101F23934021EA030106FA02F357
:100E68000B43CEF8343020E00E2B4FF006010ED89D
:100E7800A3F10A024A43DEF838C01F2393402CEA44
:100E8800030106FA02F30B43CEF838300DE00F3BAE
:100E980001FB03F2DEF83CC01F2393402CEA030158
:100EA80006FA02F30B43CEF83C30092E4FF0A0426D
:100EB8000FD99369A6F10A0303EB43039669072147
:100EC800994026EA0101916191699840084390612F
:100ED8000EE05369731E03EB4303566938219940AA
:100EE80026EA010151615169033398400843506172
:100EF8002B460434102C8BD14FF0A042936843F05A
:100F0800010393604FF0A0431A68D207FAD5DA6854
:100F1800354C22F00202DA60DA6842F00202DA6046
:100F2800DA6842F00102DA609A6842F004029A60D4
:100F3800B4F85831002B40F07087B4F95A21002AD0
:100F480040F06B87B4F95C21002A40F06687274B94
:100F5800274D1B682748B3F85630039300210C220D
:100F6800DFF8AC90B4F8608194F85FB194F86771D9
:100F780094F868A1204E14F03EFA14220021284665
:100F880014F039FA002389F80030C6F8803108F0E7
:100F9800A1FA4A46002800F01787184B2B60184B17
:100FA8006B60184BEB60B8F5807F174B2B61174BC4
:100FB80001D1002141E0B8F1BB0F01D901213CE08A
:100FC800B8F1610F26D9022137E000BF00080048B8
:100FD800080002404000005030210020000300506B
:100FE800E010FCFF07C0FFFD04130020581200208A
:100FF800B02700201029002088010020318B00082C
:101008003D8A00089588000890C1793D00000020BD
:1010180008080020B8F1290F01D903210DE0B8F123
:10102800130F01D9042108E0B8F1090F01D90521EE
:1010380003E0B8F1000FBCD006211970012313702A
:101048000223A84AA84913700B6843F001030B60F8
:101058009146A64A0023BBF1090F137001D99B469C
:10106800F7E7012202FA0BF340F2B23119400029E6
:1010780060D113F0450F09D11B075BD50023C6F8D3
:10108800803108F027FA002854D00DE019202721D4
:101098001AAB03F053FF0028F0D0954B954A1A601D
:1010A800954A5A6006234BE0062168200A460DEB54
:1010B800000303F043FF9DF86D1001F001029DF855
:1010C8006B1001F001014B0043EA82019DF8692091
:1010D80002F001030B430AD05BB2012B01D10023BC
:1010E80002E0022B0ED1012386F8843111E00EAB09
:1010F80068200C21012203F021FF9DF8383013F0FD
:101108000F0303D1032006F023FF02E0042BEAD1EA
:10111800E5E7774B794A1A60794A5A6096F884214C
:10112800002A0CBF6F226E221A72704B01221A70AD
:10113800032305E0BBF1010F09D94FF0000B88E745
:10114800694A89F80130136843F002031360BAF161
:10115800040F00F2A580DFE80AF003AD6C036C0011
:101168000A2006F080FE7720A02101220EAB03F0B2
:10117800E5FE00285DD01E210122772003F05AFFEA
:101188004FF42F6006F064FE4FF0000BABF16001E6
:101198004FF0000AC9B202221AAB77208DF868A076
:1011A8008DF869A003F0CAFE9DF869309DF86820A3
:1011B80043EA0222534B03F5C3712BF801200BF1CC
:1011C800020BBBF1100FE1D1B3F8942102F47F4E6A
:1011D800A3F894E102F00F0101205346D4462CF005
:1011E80001023244B2F88621002A18BF00201CF000
:1011F800010F03D0D2B25340082202E083EA12233F
:10120800FAE713F4004F18BF83F4C053013A4FEACA
:101218004303F6D10CF1010CBCF1100FDFD14EEAFB
:101228000102A6F8942120B9C3F30333994200F0D0
:10123800D78596F896B1DFF8CCA0BBF1000F40F047
:10124800E285142006F00FFE0AF297137620D021CB
:10125800012203F073FE9AF89731582B2AD10AF528
:10126800CC7388211822762003F068FE312276207C
:10127800F42103F0DFFE01238AF89631224B234A3A
:101288009A60234A5A6045F6D8125A80214ADA6091
:10129800214A1A61214AA3F800B05A6100F0B3BD8F
:1012A800BAF1010F06D0104A89F802A0136843F07A
:1012B800040313600C4B1A6812F0020F9A4602D00E
:1012C8000B4B1B68984718F0FF0F29D1DAF800304C
:1012D80013F0020F4FF07D0240F2712308BF4FF464
:1012E800FA7320E010010020E81A0020B42D002035
:1012F80010290020936B00083D6B0008998B0008AB
:101308007F8A000888010020E8060020D1860008AE
:10131800D3860008F9880008AB890008D58400083E
:101328004FF47A731A461344013B93FBF2F3013BE3
:10133800DBB203FB022286F8B431314B1A602B680A
:101348009847304A0023137090461FB1BA1E012AED
:1013580000F25D8500260C20314601221AAB8DF87B
:10136800686003F0EBFD002800F07F859DF8683089
:10137800482B11D1244B254A1A60254A5A60062366
:1013880088F80030032389F80330DAF8003043F096
:101398000803CAF8003002E0304600F066BD94F851
:1013A80054310BB11B4A137094F855310BB11A4ADA
:1013B800137094F856310BB188F80030DAF8003021
:1013C800164913F0080F2DD0BDF90C00DFED146A93
:1013D800642290FBF2F302FB130212B207EE902A8A
:1013E800B8EEE77A07EE903AF8EEE77AE7EE267A73
:1013F800B2EE047A67EE877AC1ED007A14E000BF96
:1014080088290020B52D0020C4060020C18A0008C4
:101418001789000808080020B42D0020701E00203D
:101428008988883C00230B60B84F3B7843F002035F
:101438003B70B74B4FF488429A614FF488521A8533
:101448004FF00A08B24EB28A92B282F48842B2824F
:10145800B28A92B282F48852B282192006F003FD51
:10146800012006F019FD192006F0FDFC002006F009
:1014780013FD08F1FF3313F0FF08E3D14FF488534D
:101488003385DAF800304FF488481B07A6F828801F
:1014980009D5A04BC6F818801B6898479E4BA6F83C
:1014A800288001221A709D4B9FED9D8A1B689D4ED6
:1014B8001B7B00EE103AB8EEC00A20EE080A0AF0CC
:1014C8005DFD338807EE903AF8EEE77A27EE800A5A
:1014D80014F0A0F9944B9FED957A1880338807EEA5
:1014E800903AF8EEE77A924BC7EE277AFF211B2253
:1014F8009FED907AC7EE877A9FED8F7AC3ED007AD9
:10150800D5ED047A8D4D8E4B67EE887A284667EEC6
:10151800877AC3ED007A13F06EFF00232B70DAF898
:101528000030884A012113F0020F18BF697011704A
:101538001FBF032111700221A9705E0748BF1178EF
:10154800284641BF4D1C15700325455413F00A0F5A
:101558000CD013780421C154591CC9B2052545542F
:10156800D91C0233DBB211700621C154764E3168A2
:101578008D0641BF13785D1C1570072548BFC554FB
:101588000B0608D513780925C5549D1C0133DBB219
:1015980015700A25C5546579082D01D00E2D08D17E
:1015A800137803F1010E82F800E04FF00B0E00F8FB
:1015B80003E0137811F4803F4FF00C0C00F803C0DF
:1015C80003F1010E1CBFDFF87CC102335FFA8EFE07
:1015D80082F800E01FBF8CF80030584B4FF00E0C1B
:1015E80003F80EC04B0741BF137803F1010E82F8D0
:1015F80000E04FF0100E48BF00F803E0137803F145
:10160800010E5FFA8EFE4FF0120C11F4806F82F813
:1016180000E000F803C00ED094F80CC2BCF1000F33
:1016280009D0DFF820C102338CF80030434B4FF06B
:10163800130C03F80EC0137811F4007F4FF0140C4C
:1016480000F803C003F1010E1CBFDFF8F8C0023335
:101658005FFA8EFE82F800E01FBF8CF80030374B2F
:101668004FF0150C03F80EC0182D13D113784FF056
:10167800160E00F803E003F1010E5FFA8EFE4FF03C
:10168800170C00F80EC003F1030E0233DBB282F828
:1016980000E0C5540B0341BF13785D1C1570192574
:1016A80048BFC554CD0541BF1378591C11701A2283
:1016B80048BFC25400219822244813F09CFE07F02A
:1016C800B4FF234B234A1A60234BB4F84E111980F8
:1016D800224900230B808B7021490A60B4F89421B9
:1016E80090B2204921F813000133122BF9D1336845
:1016F800D8045EBF1C48B0F89A0108801B0740F167
:10170800FB80194B93F88E3130E000BF882D002004
:1017180000100048C4060020DC06002094080020C1
:1017280035FA8E3C16000020B00800200AE81C415B
:10173800682D002000401C46BD3786352112002048
:101748009008002020120020442900202420002096
:10175800EC0F00208A140020F00F00200C2D002030
:10176800002D00202C2C002004130020062B00F252
:10177800BD80DFE803F004070E3D5878780045F295
:10178800F05201E042F6F822844B1A8008F003F880
:10179800ABE007EE902ADFED826A804BB8EEE77A7D
:1017A800DFED807AE7EE267A42F6F82119800023E9
:1017B800FCEEE77A7C4A17EE901A42F823100133C0
:1017C800122BF7D1794A7A4911607A4A402013706E
:1017D80009F0C2FA002800F0898001234FF00708B9
:1017E80090F90000744A8DE808014021734B77E0B6
:1017F8006A4B42F6F8221A806C4B714A1A606D4B9C
:10180800102240201A7009F0A7FA00286ED0012390
:101818004FF0000C90F900006A4A8DE8081040214A
:101828004FF4E1335CE05D4B42F6F8221A805F4BDF
:10183800654A1A605F4B082240201A7009F08CFA3A
:10184800002853D001234FF0000E90F900005F4AA2
:101858008DE8084040214FF4E13309F059F85C4B1A
:10186800C3F8B8013EE04D4ADFF89881DFF898C127
:10187800DFF898E1574D584C584842F6F821118046
:101888004C490C22062B0A700ED0002388F8003031
:101898008CF800308EF800301B232B700523227043
:1018A80003704FF4E1340BE0002188F800108CF845
:1018B80000108EF8001022702121494C2970037005
:1018C8003A4B484A1A60402009F046FA70B10123A1
:1018D8000025454A90F9000040218DE8280023465C
:1018E80009F016F8003018BF012028B908200AF0BE
:1018F80009FC2E4B3D4A1A6033682E4A13F4804F78
:101908001FBF082111702949394818BF086042F2E1
:101918000101194003F0010003F4005479B11F4993
:1019280044F620650D8024B1082111701F49314CFF
:101938000C6020B10C2111701C492F4808601178E7
:1019480004395170190640F19C802148DFF8C09095
:10195800DFF8C080C0F8BC8100242146152200F5BC
:10196800E070264D89F80140C9F80440C9F80840DC
:1019780013F041FDA8F1050320462B6007F01CFC7D
:101988001F4B02201B68C9F80C3009F0E5F9002844
:1019980042D180200AF0B6FB6BE000BFFE080020B1
:1019A800CDCCCC3F0000B0C4E42B00201C000020AC
:1019B80099150108C020002019180108A086010007
:1019C800851501086D1701086D1501082117010813
:1019D80088010020722C0020712B0020732C00201D
:1019E80090D003009514010801160108FD1501089F
:1019F800CD150108ED150108DD15010800080020C6
:101A080068290020722B0020712C0020702C0020E7
:101A1800E0070020F4140020447999F80130C54902
:101A28000C2202FB03125278A24204D00133DBB22B
:101A3800042BF4D9002389F801302B6899F8012088
:101A48001B7890F90000002B4FF00C0303FB0213E6
:101A580014BF0324012400225B7800940192022120
:101A680008F056FFB44B1860002892D0012007F008
:101A7800A3FBB24B1868B24B00F5C5721A6007F0A9
:101A880049FCB04AB04B1360B04AB14D8033136083
:101A980033680024DA032C7040F1AD800DF064FA4D
:101AA800DFF818C3DFF81893CDF810C040F22A3BCE
:101AB8004FF00108604621465A4685F8008013F029
:101AC8009AFCD9F81430A348A34D43F48023C9F8ED
:101AD8001430436A23F00F034362436A43EA08035E
:101AE8004362022203234FF4807A0CA98DF8342034
:101AF80003928DF835308DF83640CDF830A08DF84A
:101B0800378008F07DFAD9F81830039A43F4003387
:101B1800C9F818302B8823F440731B041B0C2B8046
:101B28001D23EB620EA92A8560232C862846C5F85A
:101B380014800E93ADF83E401094ADF84440ADF8D3
:101B48004640ADF84840ADF84A40ADF83C8008F052
:101B5800A3F8AB6943F00803AB616B6C43F4004333
:101B68006B64D9F8143043EA0803C9F81430A9F5AE
:101B78007D69484608F017F81AA807F0E9FF774B7F
:101B88001A9310231C938023DDF810C01F931AA901
:101B98004FF400534846CDF86CC02393ADF874B0A9
:101BA8001E94CDF880A021942294249407F0DDFFA0
:101BB800EB6843F40073EB60D9F8003043F002039C
:101BC800C9F800300BA80D238DF82C308DF82D8026
:101BD8008DF82E408DF82F800FF01CF82146604BB1
:101BE8001A68604B43F8212001312029F7D102F00F
:101BF800B1FF02F0AFFF33685B0556D55A4D5B4B1A
:101C0800D5F80085C3F80080042009F0A5F8042160
:101C1800C5F8040509F07AF8554B85F80805082039
:101C2800C3F8008009F098F8524B534C186008210B
:101C380009F06CF8002185F809052C22204613F0DC
:101C4800DAFB8E2363704FF07C0AE0234FF07D09A6
:101C5800E37084F800A084F82B90484C2C220021D3
:101C6800204613F0C8FB8A2363701020A023E3707A
:101C780084F800A084F82B90C5F80C8509F06CF85E
:101C88001021C5F8100509F041F885F81405202041
:101C9800C5F8188509F060F82021C5F81C0509F079
:101CA80035F885F820050FF0F9FE3368344A13F447
:101CB800002318BF0123137006F0AEF8314B1860EB
:101CC800314B5A79052A194602BF304B4FF4C87276
:101CD8001A802F4B4FF47A721A802E4BC8221A8022
:101CE8002D4A137843F0080313702C4A137823F015
:101CF80002031370326840F6020313406BB1284B9D
:101D0800284A1A60284B03221A70284B01221A709D
:101D1800274A00231380274A13808B683360264B99
:101D280001221A703B7863F07F033B702FB0BDEC43
:101D3800028B47E0187801085C2200205812002026
:101D4800481000209822002020150020942200200E
:101D5800B90E00200004004800440140344401400A
:101D6800A8770108BA0E002088010020DC1A00209C
:101D7800341B0020801B0020041B0020391B00207E
:101D880084290020D008002004130020FE0F002022
:101D9800AC2D0020B22D0020EC1A0020B72D002019
:101DA800D41A00207C140020381B002008010020D1
:101DB800E8100020EA100020B80E00205D03002083
:101DC80000100240BDE8F08F2C4B2B602C4B6B6051
:101DD8002C4B2B61042389F800300523FFF731B918
:101DE800294B42F210721A805A80284A5A60284AAF
:101DF8009A60284ADA60284A1A61284A5A614FF0DC
:101E0800030AFFF750BA4FF0040AFFF74CBA012F44
:101E18007FF6C5AA1F46FFF794BA1BB207EE903AA1
:101E2800DFED1F6AB4F95A311E4AF8EEE77A07EE79
:101E3800103A67EEA67AB4F95C31CDED1A7A07EE5E
:101E4800903AB8EEC77AF8EEE77A002127EE267ABC
:101E580067EEA67A11701AA813498DED1B7ACDED9D
:101E68001C7A0AF093F8FFF772B8012F7FF697AA49
:101E7800002788F80000FFF76DBA00BF316C000832
:101E8800D56B0008295C8F3DE80600200D89000805
:101E98002D8A0008038900081D8A0008D5860008D5
:101EA80035FA8E3C80000020FC200020954A2DE960
:101EB800F04F1568944C05F59C4320332DED028BAB
:101EC8002360924B196889B011F4804F05929846A7
:101ED80005D10FF031FD10B92379013323718C4BF3
:101EE8001F78C7B18B4A1268954240F2DF80013FE4
:101EF8001F70DBE0D9F800308748072D98BF595D7F
:101F0800864B88BF29461B689847032D0BD904EBDD
:101F180045050137E880804BDFF81C921E78FDB23A
:101F2800AE42E7D820E0D9F8002005F10E0302EB15
:101F380083039988DA880028E9D04FF47A73401A25
:101F48005843531A90FBF3F040F6C90300F57A7032
:101F5800984205DC40F2EE239842B8BF184601E0EB
:101F680040F6CA0080B2D2E70F23277984F82A30D6
:101F780094F82B300193032594F82C30B7FBF5F532
:101F880005EB45057D1B0393D9F800300293DFF874
:101F9800B0A1EBB204930025B54254DA6049019B25
:101FA80031F815B04FEA450953B90FF0C5FC28B10F
:101FB800039B002B08BF4FF0000B01E0DDF804B0D5
:101FC800029B988A584502D8D88A58450ED2E8B25A
:101FD8000FF05CFC032D8346DFBF94F82AE0012054
:101FE800A8402EEA0000D8BF84F82A000FF0A4FC0D
:101FF80018B14C4829F800B021E0049B94F8760009
:102008002AF813B028B9022F15D93F49012081F8C1
:102018007600BAF80210BAF800000844BAF80410BA
:102028000844414980B229F8010000B2032190FB1D
:10203800F1F080B200E058463A4929F8010001352C
:102048000AF1060AA8E794F82A203848384BA2F182
:102058000F014A424A4184F890206AB1354A126811
:10206800520109D40268D9689A60521AC82A1DD93F
:10207800012283F8212019E002689868DA605B6819
:10208800121A9A4288BF2A4B4FF0000184F82B108D
:1020980088BF83F821100025B54207DAE8B20FF0AF
:1020A800F5FB204B23F815000135F5E7D8F800308B
:1020B800DF0405D51F4B1B68DE0701D40FF0B2F90A
:1020C800059B19681C4B1868837A002B3AD0013B92
:1020D800144D027B35F813301AB1C3F53B6308334E
:1020E8009BB21BB2A3F57A73B3F57A7FA8BF4FF4FE
:1020F8007A7323EAE37307EE903A9FED107AF8EECD
:10210800E77A58E08C2D0020400F00204429002059
:10211800082D0020042D0020C02000201C000020D5
:10212800460F00202C2C0020B80F00206829002022
:102138000C2D00201C120020002D002000007A44E5
:102148006E0F0020D8F80020150440D5D4F894204C
:10215800934E8A1A002A3ADB01F59C422032C6F8CF
:102168009420904AC07A55798F4A32F8152096F80B
:102178009850013592B292FBF0F205F00F0086F804
:102188009800304480F899201A468848185C013332
:102198000244102B92B2F8D112B292FBF3F31BB2A5
:1021A800642BA8BF642323EAE37307EE903A9FEDFC
:1021B800807AF8EEE77AC7EE877A7E4A9FED7E7AD4
:1021C80067EE877AFCEEE77A17EE903A1380D8F834
:1021D80000307A4F13F4807F00F00981784BDFF8E4
:1021E800E491994205D999F8022012B9012289F897
:1021F800022099F80220002A00F0F980714A3E78FE
:1022080092F821506A1E554255416F4A1168002DB7
:10221800C1F38063C6F380060193924614BF4FF062
:10222800000B4FF0030B99F82020052A00F2D98003
:10223800DFE802F0034D527584A1002E3AD0D4F89D
:10224800AC00B4F8B01005F0A2FD012809D15F492F
:102258005F4A09681268C988642000FB0122C9F82E
:102268001020019B6BB1594A126812794AB10CF0DF
:10227800EDFD032289F820204FF47A72C9F81C205A
:10228800D1E7002D40F0AD80514AD9F81010106800
:102298004C4A88420AD902920CF0D8FD029A0321CE
:1022A80082F8201040F6B831D161BCE7012182F8EC
:1022B8002010B8E7019B4FF4806013B109F012FFBA
:1022C80001E009F0FEFE0022C9F8102089E0002D87
:1022D80046D10CF0BBFDA6E725B1052289F82020E0
:1022E800012000E0284666B1D4F8AC20D189394AEB
:1022F800118051809180354909684988D1804FF013
:10230800020B334A1168D9F81420914201D8002EE3
:1023180064D147F23052C9F81C20032221E03A78F0
:1023280042F002023A700FF07DF8294AD9F81C10E1
:1023380012680A44C9F81820042212E0244A9DB100
:102348001168D9F8182091424BD9234A12781AB942
:10235800DAF80020D30744D43A7822F002023A701F
:10236800052289F820205EE71268D9F81C100A4473
:10237800C9F8182035E01549154A09681268C9884E
:10238800642000FB0122C9F810204FF4806000226D
:1023980089F8202089F8032009F093FE43E700BF5D
:1023A800400F00202021002030210020D90F0020DC
:1023B8000000C8427812002000C07F44B72D0020DA
:1023C800404B4C000C2D00201C120020D027002070
:1023D800682900202C2C00201400002000287FF4FD
:1023E80022AFBBF1000F02D0584605F073FD934DA4
:1023F80005F5C370B5F84E1105F0C9FC834668B9F8
:102408000CF016FD8E4BC3F800B0C3F804B0C3F847
:1024180008B08C4B00221A605A609A603B785E07BD
:1024280036D5D8F80030D80632D5874B1B78D90670
:102438002ED4864B1B7893B195F8DE31BBF1000F93
:1024480015D17BB1824B1A68D4F8B4309B1A002B93
:1024580008DA0EF0E7FF7F4B83F8B8B018E0BBF15D
:10246800000F0DD1102005F035FD01230EE03BB122
:10247800774A12684FF47A7101FB0323C4F8B43029
:1024880094F8B83023B105F00DFD002384F8B83076
:10249800002295F8DCA195F8DD11B5F896E1B5F8BC
:1024A80098C113466C4E019636F912009B08704588
:1024B800C4BF63F07F03DBB201326045B8BF43F0AD
:1024C8004003042AEED194F8B92062489A4205D113
:1024D80090F8BA20F92A04D8013200E0002280F8E6
:1024E800BA2084F8B930594B5C4E1A789946E2B94B
:1024F8003368DA0708D5BBF1000F16D13B78DB0744
:1025080013D50EF0FBFD10E03B7858070DD5514B65
:1025180093F82B304BB1524BDB7833B911B10EF035
:1025280081FF02E0BBF1000FF9D094F8BA30494AB4
:10253800DFF840B1142B40F0AF8099F800301AF161
:10254800000A18BF4FF0010A6BB392F8B9305F2B3D
:1025580011D13B7803F0040303F0FF0113B10EF02F
:1025680061FF08E00B200391029205F0B3FC029A88
:10257800039982F8BA10BAF1000F14D094F8B93060
:102588007D2B10D13B7803F0040303F0FF0213B155
:102598000EF048FF07E00B20029205F09BFC2D4B44
:1025A800029A83F8BA203B7803F0040303F0FF0192
:1025B800002B71D194F8B930264A572B16D1294BE4
:1025C8004FF47A721A80D8F80030190601D506F04F
:1025D80003FF254B1B685A0742BF244A0A21118072
:1025E80013F0080358D1224A138055E0D8F80000A8
:1025F800400717D55A2B15D192F8BB302BB10123C0
:1026080082F8BB1082F8BC3046E092F8BD3083F007
:10261800010382F8BD300BB10C2000E00D2005F05D
:1026280059FC39E05D2B00F022855B2B00F02185F9
:102638005E2B21D1032000F01DBD00BF0413002034
:10264800C41B0020241C0020EC1A002014000020C9
:1026580068290020400F00202C2C00201C1200208C
:102668000C2D0020AC2D0020E81A0020B22D0020EF
:10267800F412002058120020562B01D109F0E8FF6F
:1026880099F80030002B00F00A8594F8B9306F2BC8
:1026980040F0FF840EF032FDD8F80030580736D5E8
:1026A80094F8BD30B84A93B13B7859070FD5019BD0
:1026B800B3F90610B5F89631994208DD336813F07E
:1026C800010302BF3221A2F8C01082F8BD3033687E
:1026D800DA030DD594F8C220AB4B2AB993F8BB2086
:1026E80012B93222A3F8C020012384F8C2300EE0C8
:1026F80094F8BB30A44A53B13B7803F0040303F0C9
:10270800FF0123B9012382F8BB1082F8BC30DBF843
:1027180000A0002333600AF17B090AF1CB0B99F87A
:10272800002099F8013019F8010C9A420BD2494659
:1027380005F0F6FA38B119F8022C012303FA02F26F
:1027480033681343336009F10409D945E7D18F4B46
:102758001B7853B18E4B8F4E1A68DFF850A212F0D7
:10276800020F994640F03A8331E30AF1CA060AF5A6
:1027780089793278737816F8010C9A4225D2314655
:1027880005F0CEFA08B3B37896F804E0824A96F8D2
:1027980003A07D480C21013B01FB0E4103EB4303E1
:1027A8001344D1F8C8209A420FD0C1F8C83000238A
:1027B80090F8F420C1F8CC30012303FA0EF322EA92
:1027C800030381F8C4A080F8F43006364E45D0D112
:1027D800724B1E68724B1B68039394F82B3004935A
:1027E800704B029300230193029B1B68002B00F09F
:1027F800E38293F800A0BAF1000F00F0DD82029A9C
:10280800039952688A1A002A0CDB01F5FA720299B8
:102818004A60019901228A4094F8F41021EA0202E0
:1028280084F8F420049A002A00F0C682029A5978A3
:1028380012F8042C0432D2B2002940F07C825A49A2
:1028480031F91210B5F8942102F1C800814202DD75
:1028580093F802B015E0C83A914203DA9978C1F1C9
:10286800000B0EE0019A0123934094F8F42022EA29
:10287800030384F8F430039B029A03F5FA73536058
:102888009AE294F8F430019A1341DB0700F194823C
:10289800BBF1000FCCBF0220012005F041FB0AF17B
:1028A800FF33DFF8E490132B00F27E82DFE813F0A9
:1028B8001400250037004B0064008600E9004C0135
:1028C800B301E10111027C024B005A008600E900C5
:1028D8004C01BB001E01830196F80090D944B9F160
:1028E800FA0FA8BF4FF0FA0929EAE979304686F8C5
:1028F800009005F0FBF901200FE096F80190D9440B
:10290800B9F1640FA8BF4FF0640929EAE9793046A4
:1029180086F8019005F0EAF902204946D6E196F8D2
:1029280003A0DA44BAF1640FA8BF4FF0640A2AEA98
:10293800EA7A86F803A03046D9F8F81008F014FAB5
:1029480003205146C2E1717959446429A8BF642122
:1029580021EAE17171710D2005F04AFABAF10D0F03
:1029680000F02282317959446429A8BF642121EA00
:10297800E17131710E20A9E1B179594481F308015F
:10298800B1710520A2E100BF400F0020BA2D002040
:102998001C120020E81A0020147C01087C12002078
:1029A80068290020081000202C2C0020B01B0020D3
:1029B80000007A440000C84200000000D9F8FC304A
:1029C8001A78022A20D107EE90BAB8EEE70A5FED2E
:1029D800077A93ED097A80EE270A30EE070AB5EEFA
:1029E800C00AF1EE10FA07D4B4EE670AF1EE10FA55
:1029F800C8BFB0EE670A01E01FED110A83ED090AAE
:102A08000F2005F0DFF90AE099785944C829A8BFD2
:102A1800C82121EAE17199700F2005F0E9F9BAF1AE
:102A28000F0F00F0C181D9F8FC301A78022A1ED1A4
:102A380007EE90BAB8EEE78A5FED227A93ED080ABE
:102A480088EE278A38EE000AB5EEC00AF1EE10FAD1
:102A580007D4B4EE670AF1EE10FAC8BFB0EE670A01
:102A680001E01FED2B0A83ED080A122056E1597880
:102A78005944C829A8BFC82121EAE1715970122018
:102A880024E1D9F8FC301A78022A20D107EE90BA4E
:102A9800B8EEE70A5FED397A93ED0C7A80EE270AF3
:102AA80030EE070AB5EEC00AF1EE10FA07D4B4EE1C
:102AB800670AF1EE10FAC8BFB0EE670A01E01FED31
:102AC800420A83ED0C0A102005F07CF90AE0197B14
:102AD8005944C829A8BFC82121EAE17119731020F7
:102AE80005F086F9BAF1100F00F05E81D9F8FC30D4
:102AF8001A78022A1ED107EE90BAB8EEE78A5FED7F
:102B0800537A93ED0B0A88EE278A38EE000AB5EE61
:102B1800C00AF1EE10FA07D4B4EE670AF1EE10FA23
:102B2800C8BFB0EE670A01E01FED5D0A83ED0B0A2E
:102B38001320F3E0D97A5944C829A8BFC82121EA4B
:102B4800E171D9721320C1E0D9F8FC301A78022A51
:102B580022D107EE90BA1FED6A0AF8EEE77A87EEFF
:102B6800800AD3ED0F7A30EE270AB5EEC00AF1EEEF
:102B780010FA09D45FED717AB4EE670AF1EE10FA33
:102B8800C8BFB0EE670A01E01FED750A83ED0F0AB2
:102B9800112005F017F90AE0997D5944C829A8BF02
:102BA800C82121EAE1719975112005F021F9BAF1DE
:102BB800110F00F0F980D9F8FC301A78022A20D1D8
:102BC80007EE90BA1FED860AB8EEE78A88EE008A0B
:102BD80093ED0E0A38EE000AB5EEC00AF1EE10FACF
:102BE80009D45FED8C7AB4EE670AF1EE10FAC8BF2B
:102BF800B0EE670A01E01FED900A83ED0E0A14207B
:102C08008CE0597D5944C829A8BFC82121EAE1713F
:102C1800597514205AE0D9F8FC301A78022A1ED1C6
:102C280007EE90BAB8EEE78A5FED9E7A93ED0A0A4E
:102C380088EE278A38EE000AB5EEC00AF1EE10FADF
:102C480007D4B4EE670AF1EE10FAC8BFB0EE670A0F
:102C580001E01FEDA70A83ED0A0A09205EE0D97892
:102C68005944C829A8BFC82121EAE171D9700920AF
:102C78002CE0D9F8FC301A78022A1ED107EE90BA57
:102C8800B8EEE78A5FEDB57A93ED0D0A88EE278AEC
:102C980038EE000AB5EEC00AF1EE10FA07D4B4EE29
:102CA800670AF1EE10FAC8BFB0EE670A01E01FED3F
:102CB800BE0A83ED0D0A0A2030E0597B5944C82921
:102CC800A8BFC82121EAE17159730A2005F090F8DC
:102CD8006AE0D9F8FC301A78022A22D107EE90BAB5
:102CE8001FEDCD0AB8EEE78A88EE008A93ED100A48
:102CF80038EE000AB5EEC00AF1EE10FA09D45FED1D
:102D0800D37AB4EE670AF1EE10FAC8BFB0EE670ADC
:102D180001E01FEDD70A83ED100A0B2005F052F8E9
:102D280042E0D97D5944C829A8BFC82121EAE171E8
:102D3800D9750B20CAE7012936D19878B84B33F9F1
:102D48001230B3F5617F05DB40F633029342A8BF2A
:102D5800134601E04FF46173BAF10C0F24D14FF41C
:102D6800966292FBF0F0AF4AA3F5617393FBF0F320
:102D78005FFA83F913784B4516D0B9F1040F34BFC5
:102D88004B4602231370A84A0AFB035303F2A673A7
:102D9800136009F083FA5046494605F029F809F10D
:102DA8000100C0B205F0BCF8019A0123934094F8E1
:102DB800F420134384F8F430019B01330193029B00
:102DC8000C330293019B042B7FF40EADC2E4D8F8B8
:102DD8000030D80510D5954BDB786BB1336899076F
:102DE8000AD5BAF8003013F0010B0AD10CF020F81C
:102DF800012009F077F904E0012009F062F90123C4
:102E080000E00023D9F8002052070DD563B1012056
:102E180009F057F9BAF800309B0708D40CF008F805
:102E2800022009F05FF902E0022009F04AF9BAF835
:102E380000307F4A13F0030F4FF4884114BF9161AB
:102E48001185326812F00A0F27D0D9F80020D00671
:102E580009D559070AD4042009F044F9754B1B8891
:102E6800A4F8003102E0042009F02BF9D9F8003069
:102E78009A0607D5BAF800305B0606D4402009F058
:102E880031F902E0402009F01CF9D9F80030580661
:102E980042BF684B1B88A4F802313368990609D4ED
:102EA800D9F800301A0540F191804FF4807009F08C
:102EB80019F98FE0604B1B789B0753D55F4B1B7844
:102EC800042B4FD9D9F8003013F4007B0FD0BAF88F
:102ED8000030DE063AD4102009F004F9202009F069
:102EE800F0F85748011D06F0CBF902232AE0BAF89A
:102EF800006006F01006B6B22EB1102009F0E1F815
:102F0800012684F804B1D9F80030580512D5D4F850
:102F180008314C495A89B1F90030002BB8BF5B42DF
:102F2800934207DAB1F90230002BB8BF5B429342F3
:102F3800C0F2F880BAF80030990608D5202009F0C8
:102F4800C0F8002384F80431012600E0002694F834
:102F58000C31BBB90E2004F0BDFF3B4B012283F8B6
:102F68000C210FE0BAF8003003F03003002B97D0A3
:102F7800102009F0A6F8202009F0A3F8002384F80F
:102F8800043101E0002E8BD0304B002003F12806DD
:102F980003F150042E4A002122F810102D4A5960DE
:102FA80022F810100432716022F8101000221A6002
:102FB8009A603260B26022606160A2601433143695
:102FC800143400287FF46CAF0120E3E74FF48070DD
:102FD80009F077F86B79082B01D00E2B02D140202D
:102FE80009F06FF8D8F800305A0540F1B18095F82B
:102FF8000C321BB93B7813F0040F03E0D9F800300A
:1030080013F4002F2AD0144B00221A703C2006F02B
:103018000BFC002800F09C800CF01EFFF6E700BFB8
:103028002C2C0020F02800207C1200200C2D0020E1
:1030380000100048F4120020EC1A0020F21A0020B8
:1030480084120020FC120020400F002050100020A5
:10305800AE2D0020C8100020C52000200EF01EFD57
:1030680009B0BDEC028BBDE8F04F06F0DEBA0120D6
:1030780000E002205FFA80F909F1FF3385F8A437F0
:1030880009F072F809F02EF9484604F049FFFFF7F5
:1030980003BBBAF1000F02D07E2B3FF4FBAA94F8D1
:1030A800B930972B06D12D4B4FF4C872A3F8BE2028
:1030B800FFF7F2BAA72B06D1294A137843F0040385
:1030C8001370FFF7E9BA0022BB2B079201D1022344
:1030D80003E0B72B04D14FF6FE73ADF81E300AE0BB
:1030E800BE2B01D1022304E0BD2B7FF4D5AA4FF6F5
:1030F800FE73ADF81C30DBF80030BDF81C10B3F8D7
:1031080058200A44A3F85820BDF81E10B3F85A20D6
:103118000A44A3F85A2009F09BFA002384F8BA302D
:10312800FFF7BABABAF800309B063FF510AF202077
:1031380008F0D8FF0B480C4B011D1A685B68436008
:10314800026006F09DF8054B012683F80461FEE64F
:1031580009B0BDEC028BBDE8F08F00BF400F002026
:10316800EC1A00208C120020F41A00202DE9F04FF0
:10317800C14BB3F90610C14B2DED028B1F687A893C
:1031880085B0914201930EDBB1F5FA6FFC79BDBFB2
:103198008B1A6343A2F5FA64C4F16404BCBF93FBC1
:1031A800F4F4643400E06424B54BB64AB3F894B13F
:1031B80093F95E31126802929BB21546039300227E
:1031C800AD4B33F912E0CBEB0E0303F2F31640F2EA
:1031D800E63086424FEA420C03D8002BB8BF5B4268
:1031E80001E04FF4FA73022A2ED0029E96F811617C
:1031F8001EB1B342CCBF9B1B0023A34E6FF0630AE2
:10320800642093FBF0F836F818900AFB083A08F1A6
:10321800010836F918600FFA89F8C8EB060606FBAC
:103228000AF696FBF0F699484E4420F80C60BE1852
:10323800642036797343964E93FBF6F364339BB25E
:10324800634393FBF0F02DE0029890F812611EB1F1
:10325800B342CCBF9B1B0023DFF860926FF063087A
:10326800642093FBF0F008FB003A39F91060013054
:10327800002B39F91000A0EB060000FB0AFABDF894
:103288000C009AFBF8FAC6EB0A0A1AFB00FA7F4808
:10329800A0F804A0B879B8BF5B4243437C4893FBCD
:1032A800F0F064306B787B4E4FF06408434393FB37
:1032B800F8F3B354784EEB7A434393FBF8F3B354E3
:1032C8006B7D724E5843754B90FBF8F0022A985468
:1032D800734B0ED1DE4583F802800DDB684CB4F8E1
:1032E8009621914214DBB1F5FA6FA8BF4FF4FA6149
:1032F8000FE0DE459C5404DA36F80C305B4226F8C1
:103308000C300132032A05F101057FF459AFE5E7D6
:103318001146DFF8BCE15D4D891A4FF47A736FF0FE
:1033280063075943C2F5FA626423B1FBF2F191FBDA
:10333800F3F23EF8120007FB0211013207B23EF920
:103348001220D21B514391FBF3F30344F380554BF6
:103358001B885F0635D5544B544A1B881288DFED0D
:10336800547A9B1A1BB208EE103AB8EEC88A28EEB7
:10337800278AB0EE480A08F001FEF0EE408AB0EE67
:10338800480A08F098FDB5F9023006EE903AB5F90A
:103398000030F8EEE66A07EE903A20EE667AF8EE2C
:1033A800E77AA7EEA87A67EE807ABDEEC77AE6EEEE
:1033B800A87A17EE103AFDEEE77A2B8017EE903ACE
:1033C8006B803C4D2B68980740F1A1803A4B3B4FEE
:1033D8001A687B6945F20721D31A8B4240F397801C
:1033E8007A6106F0E5FE364BDFF8E8901A78032A92
:1033F8009846B9F8003022D10A2B2AD90023282070
:1034080088F8003004F02FFD06F0D2FE2D4B188806
:103418000EF026FA2C4B1A68D37890FBF3F00130A3
:1034280008282A4BA8BF08201870537980B213FBCC
:1034380000F33B83137913FB00F0788309E00A2B30
:1034480007D80323214A88F80030002313703B83F0
:103458007B8398F800301A4A012B3DD002D3022B07
:103468004CD054E03A8BB9F800309A424FDD012332
:1034780088F8003040E000BF2C2C00207C1200208F
:103488000413002058120020501C0020FC120020B9
:103498000CFEFFFF381C0020DE1000204C1C002012
:1034A800C01B0020B01B0020F41200204210002096
:1034B80035FA8E3C442900208C2D0020D0100020A5
:1034C800381B002038210020D41A002008010020D1
:1034D80022220020D81A0020B9F800107B8B8B42DA
:1034E80002DD022313700FE0A34B1B8B01339942BB
:1034F80002DD002313700AE0082006E07B8BB9F890
:10350800002001339A42B2DC072004F0E3FC2D6866
:10351800290577D5994B984F1A68FB69C3EB0208C0
:1035280045F2072398456DDD954BB6F906B0D3F8FB
:103538000090FA6199F80A30B4F84E11914E012BB7
:103548004FF47A70ABF57A7B98FBF0F803D042D34E
:10355800022B20D041E08C4B396A5A7B8B4B33F8D5
:1035680012204FF0080E92B291FBFEF3C91A8B1885
:10357800BA843B6240F6E44293FBFEF39BB25343AA
:10358800B9F80820C2EB13335843B9F9063090FB59
:10359800F3F0306021E07E4BB9F808A01B78C6F83C
:1035A80000A05A0719D57B4804F0F1FB20B915F0A3
:1035B800100F18BF4FF0000B32220BFB0BF393FBDD
:1035C800F2F3B9F906205B445A434FF47A7392FB3D
:1035D800F3F3534400E000233360D7E90A0133686A
:1035E8006D4A03FB08F84FF47A7398FBF3F810EB75
:1035F800080041EBE8710023C7E90A010EF004FD59
:10360800664B1860664E3368DB0427D52F0622D533
:10361800644B1B789D071ED5634B187804281AD96C
:103628000022624BD7180521951C4FF00A0E122A6A
:10363800D154E9B287F801E004D0B0EB510F2A4623
:10364800EFD800E014215A18322002F8010CFF22AA
:103658005A540F2000E00A2004F03CFC544D2A681C
:10366800002A50D0534B544F186839688142984605
:1036780049D8524BDFF8509119785268E1B94FF0A8
:10368800010A83F800A0B9F80030D35C23B3504690
:1036980004F002FC4A4B83F800A00EF059F9B9F87F
:1036A8000030CBB92B681B78053B534514D804F080
:1036B800B3FB444B18600FE04FF0000A83F800A0FA
:1036C800B9F80030D35C3BB1504604F0E5FB3C4B05
:1036D80083F800A00EF03CF92A68B9F80030526867
:1036E8003948D25CFE2A01D100230BE0FF2A02D11F
:1036F80004F0D8FB07E0D8F800500A2111FB025269
:103708003A6001330380224D2B78580704D52F4B9C
:103718004FF488529A6171E03268D1075CBF43F078
:1037280001032B701F4B1B781F075EBF2B7823F0FC
:1037380001032B70D60248BF2B78214A44BF23F0DF
:1037480001032B70224B1B6813F0040F02D0214990
:10375800098851B92049098809B1980705D41F4B30
:103768001B88003318BF0123D3B3022313702B78AF
:1037780023F001032B7038E0D01000208C2D00209E
:10378800D41A0020E01A0020202100203021002037
:10379800B72D00208A140020407E0500E41A00207E
:1037A8001C120020EC1A0020F21A00201C2900200C
:1037B800741C0020682900206C1C0020681C002054
:1037C800302D0020282B0020701C002000100048FD
:1037D800E81A0020B22D0020FE0F0020AC2D00209A
:1037E8002978C90758BF0223137004F015FBB24BA0
:1037F8001B68C01A002801DB0EF0AAF80EF04EF97B
:10380800AE4B1E789846002E00F0A980AC4E336867
:10381800002B00F0D786306804F0F5FB002800F094
:10382800D186A74BA74C186804F0EAFB092801D0F9
:103838003F2850D14FF0000AD4F80090A24D5746C7
:10384800B9F1000F05D0A14829684A4611F020FEB9
:1038580010B9AA4607B92F469D4B10359D42EFD3A4
:10386800C7B1D7F800E0DAF800C023681EF80350A3
:103878001CF80300A8420DD15A1C944938B92D2BC5
:1038880005D8904D2A602025CD54885402E0CD54A7
:103898002260EAE723680BB1574511D08D480CF038
:1038A800CFFB574507D857F8100B0CF0C9FB092078
:1038B8000CF0BEFBF5E788480CF0C2FB4FF000099E
:1038C80023689945A7D2814B13F809000CF0B0FB87
:1038D80009F10109F4E72368002B40F05786042812
:1038E80040F09986794809F001F800F06BBED9F8E4
:1038F8000000DFF8F4A104F086FB30B3DAF800002A
:1039080004F07EFBDBF8003093F8481002460029EB
:1039180033D124286AD1012283F84820DBF800300B
:10392800DFF8C0A193F84820062AE0D193F84900AF
:1039380001F0EEFB002800F083803B6898790CF0DA
:10394800C8FA3B68002283F84820644B93F8353066
:10395800002B40F0FB854C36982E00F03386604BE8
:10396800F21892F84A100129F5D15E4FF3583A60DF
:103978005D4ABB4613609146B9E7012904D14D2839
:1039880014BF00220222C7E7022904D13C2814BF31
:1039980000220322C0E703290CD140284FF0000180
:1039A80002D983F84810B9E758711971D97198711B
:1039B8000422B1E7042906D1997983F849004A40DD
:1039C8009A710522A8E70529A8D15879197988425A
:1039D800987906D950409871481C18710B441A728E
:1039E8009CE790420CBF0622002295E72B783F49BE
:1039F800580793D4232ADAF8003014D1012088F824
:103A080000002F480391036034480292036338484A
:103A18000CF016FB30480CF013FB0399029A0B7854
:103A280043F002030B70334B1B681B78934201BFB2
:103A3800314B324A1A60324B04BF324ADA606DE7C2
:103A4800DAF8002092F849304C2B00F08A8478D8B4
:103A5800332B00F0C18421D8292B00F04E8409D8DB
:103A6800252B00F02584272B00F02984232B40F0F8
:103A7800CE8541E22D2B00F0518407D82B2B40F046
:103A8800C6850CF009FA607100F05BBD2F2B00F0C1
:103A98001085312B00F0228500F0B9BD3C2B00F0D9
:103AA8000D8131D8372B00F0CC84392B00F01484E9
:103AB800352B40F0AC855AE2342D0020BA2D002079
:103AC8000C290020902200204C830108602200204D
:103AD800FC840108D79B0108DC9B0108D01000205A
:103AE80024200020901B0020941B0020B72D0020CC
:103AF8000C9C0108C8200020FC9F0020EFBEADDE12
:103B080000ED00E00400FA05412B00F06A840CD8AF
:103B18003E2B40F07C850CF0BFF984F8DE010CF0F8
:103B2800BBF984F8DD0100F00CBD432B00F066847E
:103B3800442B40F06C85E94B012283F8352000F0D6
:103B480000BDD02B00F00A8355D8CA2B00F0C580E1
:103B580009D8C82B00F0858000F221834E2B00F095
:103B68000D8400F054BDCD2B00F0038304D8CC2B7A
:103B780000F0258200F04BBDCE2B00F00383CF2B45
:103B880040F045850CF092F96FF4AF6283189BB250
:103B9800C62B98BFA4F894010CF088F9A4F840014A
:103BA8000CF084F9A4F842010CF080F9A4F844015F
:103BB8000CF07CF9A4F8D6010CF06EF984F8EB014E
:103BC8000CF06AF90CF068F984F8EC010CF064F96F
:103BD80084F883010CF060F984F890010CF05CF92A
:103BE800BF4BD3F800900CF061F900EB8000400067
:103BF800A9F8560070E3D62B00F034820AD8D22BED
:103C080019D0C0F0F382D32B25D0D42B00F0368204
:103C180000F0FDBCEF2B41D005D8D82B40F0F7843D
:103C28004FF0000AEBE0F22B00F07082FA2B00F064
:103C3800B28200F0ECBC2B78590700F182840CF0BA
:103C48002BF9022884F8A40740F28E82A54B0022A3
:103C580083F8A42788E20CF029F9A34B188000F018
:103C680070BC92F805904FEA5909B9F1120F03D9BF
:103C780005F0D6FD00F065BC4FF0000ACA4507D232
:103C88000CF014F9994B23F81A000AF1010AF5E728
:103C9800924B012283F8342000F053BCDFF84092A5
:103CA800D9F800A00CF002F9AAF85A00D9F8009047
:103CB8000CF0FCF8A9F8580000F043BCDFF820929B
:103CC800D9F800A00CF0E8F88AF80000D9F800301C
:103CD800187804F0D7FB00F034BC814B1A681278CE
:103CE800022A824699466FD1D9F800B00CF0D4F870
:103CF80007EE900AF8EE677AB2EE048AC7EE887A81
:103D08000BEB8A0BCBED087AD9F800B00CF0C4F8AD
:103D180007EE900A9FED767AF8EE677A0BEB8A0B3E
:103D2800C7EE877ACBED0B7AD9F800B00CF0B4F86F
:103D380007EE900A9FED6F7AF8EE677A0BEB8A0B25
:103D4800C7EE877A0AF1010ABAF1030FCBED0E7AB2
:103D5800CAD1BAF1070FD9F800B01CD10CF09CF801
:103D680007EE900AF8EE677AC7EE887ACBED117AFB
:103D7800D9F800B00CF090F807EE900AF8EE677AE0
:103D8800C7EE887ACBED127AD9F800B00CF084F837
:103D98008BF84C0012E00CF07FF8D3448BF801004C
:103DA800D9F800B00CF078F8D3448BF80B00D9F8A8
:103DB80000B00CF071F8D3448BF815000AF1010A31
:103DC800BAF10A0FC5D1BCE3D9F800B00CF064F819
:103DD800D3448BF80100D9F800B00CF05DF8D34457
:103DE8008BF80B00D9F800B00CF056F8D3440AF160
:103DF800010ABAF10A0F8BF81500E5D1A1E3DFF843
:103E0800E0909FED3C8AD9F800B00CF04FF807EE2F
:103E1800900AF8EE677A0BEB8A0BC7EE887ACBED3F
:103E2800087AD9F800B00CF041F807EE900AF8EEDD
:103E3800677A0BEB8A0BC7EE887ACBED0B7AD9F849
:103E480000B00CF033F807EE900AF8EE677A0BEB47
:103E58008A0BC7EE887A0AF1010ABAF1030FCBED93
:103E68000E7ACCD1BAF1070FD9F800B01CD10CF0FA
:103E78001DF807EE900AF8EE677AC7EE887ACBED60
:103E8800117AD9F800B00CF011F807EE900AF8EEA4
:103E9800677AC7EE887ACBED127AD9F800B00CF0C1
:103EA80005F88BF84C0012E00CF000F8D3448BF8BE
:103EB8000100D9F800B00BF0F9FFD3448BF80B00E0
:103EC800D9F800B00BF0F2FFD3448BF815000AF1D3
:103ED800010ABAF10A0FC5D133E300BFD0100020A0
:103EE8005812002004130020401000202C2C002021
:103EF8000000C84200007A440BF0CEFF1328834626
:103F08003FF6B6AEDFF84CA3DAF800900BF0C4FF2A
:103F18000023CB4A0C2101FB0322117A814222D1D2
:103F28000FFA8BFB09EB8B09137889F879300BF0C2
:103F3800B3FF89F87A000BF0AFFF89F87B000BF02C
:103F4800ABFFC04BC04A1A6089F87C00BF4BDAF857
:103F5800000018600021793003F008FFBC4B80F0A6
:103F680001001870EDE201331C2BD2D180E60BF072
:103F780093FF0B2882463FF67BAEB64BD3F80090F2
:103F88000BF08AFF03283FF673AE062303FB0A995A
:103F980089F8CE000BF080FF89F8C9000BF07CFF90
:103FA80089F8CA000BF078FF89F8CB000BF074FF92
:103FB80089F8CC000BF070FF89F8CD00C1E2537985
:103FC800092B7FF655AE019BD3F800900BF064FFE8
:103FD800019B89F80000D3F800900BF05DFF89F889
:103FE80001000BF059FF019B64281B68A8BF6420DF
:103FF80018710BF051FF019B64281B68A8BF64204F
:1040080058710BF049FF019BFF281B68A8BFFF20D0
:1040180098710BF041FF019B6428D3F8009028BFEA
:10402800642089F807000BF037FF019B89F802002C
:10403800D3F800900BF030FF019B89F80300D3F808
:1040480000900BF033FF3B68A9F80A005B790A2B54
:1040580040F27782804BD3F800900BF01DFF89F86F
:1040680008006EE282460BF021FF7C4B23F81A0011
:104078000AF1010ABAF1080FF5D162E253790F2B60
:104088007FF4F6AD0BF008FF072881463FF6F0AD48
:10409800DFF8C0A1DAF800B00BF008FF0E2303FB2D
:1040A80009F9CB44ABF81901DAF800B00BF0FEFEC1
:1040B800CB44ABF81B01DAF800B00BF0F7FECB44A9
:1040C800ABF81D01DAF800B00BF0E6FECB448BF834
:1040D8001F01DAF800B00BF0DFFECB448BF82001AB
:1040E800DAF800B00BF0D8FECB448BF82101DAF8EF
:1040F80000B00BF0D1FECB44DAF800A08BF8220117
:104108000BF0DEFED144C9F823011AE20BF0C4FE1D
:104118000F2881463FF6ACAD0BF0BEFEC9EBC909CE
:10412800A14489F8D0000BF0B7FE89F8D1000BF054
:10413800B3FE89F8D2000BF0AFFE89F8D3000BF07C
:10414800ABFE89F8D4000BF0A7FE89F8D5000BF078
:10415800A3FE89F8D60004F0F9F8F2E12B785B07A2
:1041680000F1EF810CF0A4F907F0FEFF08F0BAF8AF
:10417800E7E12B78580700F1E481394B4FF4C87216
:104188001A80DEE12B78590700F1DB81354A137874
:1041980043F0040328E02B785A07E5D537E20BF003
:1041A8007BFE304B1A7810B142F0020201E022F097
:1041B80002021A700BF070FE2B4BDFF8C4901870D7
:1041C8000BF07EFEC9F800000BF07AFEC9F8040077
:1041D8000BF06CFE254B18800BF068FE244B254A2B
:1041E8001880137843F002031370AAE10BF054FE11
:1041F80002900BF065FE83460BF062FE82460BF0E0
:104208005FFE81460BF052FE0BF050FE0BF044FEB1
:10421800029BBBBB184B1020C3F800B0C3F804A026
:1042280007F04FFF0F4A137843F001031370B9F1F9
:10423800000F00F08681114BC3F8009081E100BFA8
:10424800807C010838100020441400203C10002015
:1042580014000020581200207C120020F2280020B0
:10426800FE0F0020EC1A0020F21A0020F01A00209D
:10427800EE1A0020821200208412002094120020DE
:10428800F41A0020102B40F05C81B94BC3F800B041
:10429800C3F804A0B9F1000F02D0B64BC3F80090E0
:1042A800B348B54B0222011D1A7004F0E9FF48E13A
:1042B800A0600BF005FEA3681843A06041E10BF075
:1042C800F5FDA4F858010BF0F1FDA4F85A010BF024
:1042D800EDFDA4F85C0134E10BF0DEFD84F8780113
:1042E8000BF0DAFD84F87C010BF0D6FD84F87B0135
:1042F8000BF0D2FD84F87D0123E10BF0D7FDA4F883
:104308007E010BF0D3FDA4F880010BF0C5FD84F805
:1043180082010BF0CBFDA4F8840112E10BF0BCFD87
:1043280084F88E010BF0C2FDA4F898010BF0BEFDD5
:10433800A4F894010BF0BAFDA4F896010BF0ACFDBB
:10434800DAF8003084F88F015B79082B40F2F980A5
:104358000BF0ACFDA4F89A010BF0A8FDA4F89C01A1
:10436800EFE00BF099FD84F8D4010BF095FD84F88B
:10437800D5010BF09BFDA4F8D601E2E092F8059078
:104388000323B9FBF3F9B9F1120F3FF671ACDFF86B
:10439800F8A14FF0000BCB4580F0D3800BF07CFDEB
:1043A8008AF89E010BF082FD40F2ED23984205DD6C
:1043B80040F6CA039842A8BF184601E040F2EE2032
:1043C800A0F2EE2019230BF1010B90FBF3F00AF198
:1043D800020A8AF89D01DEE70BF05EFD84F8900181
:1043E800AFE082460BF058FD04EB0A030AF1010A1C
:1043F800BAF1080F83F88601F4D1A2E00BF04CFD66
:104408000023A36060710BF05BFDA3681843A060F4
:104418000BF042FD84F88E010BF048FDA4F858011A
:104428000BF044FDA4F85A010BF040FDA4F85C0120
:104438000BF03CFDA4F87E010BF038FDA4F88001D8
:104448007FE053794FF0070AB3FBFAF2C2EBC202DE
:104458009A1A12F0FF0F7FF40BACB3FBFAFA0AF1C9
:10446800FF3A5FFA8AFABAF1FF0F6AD00BF014FD2F
:104478005FFA80FB4FFA8BF006F086FB8146002836
:104488003FF4F6AB80F800B00BF010FDA9F802007D
:104498000BF002FD89F804000BF0FEFC89F805001A
:1044A8000BF0FAFC89F807000BF0F6FC89F8060017
:1044B800D5E7DFF8D49009F1400A0BF0F7FCA9F82A
:1044C8009C020BF0E9FC89F89E020BF0E5FC09F16F
:1044D800040989F89B02D145EFD132E00BF0DCFCEE
:1044E8001F2881463FF6C4AB3B685B79082B7FF4F5
:1044F800BFAB0BF0DBFC09F1860904EB890900F07E
:104508003F00A9F806000BF0D1FCB9F8063080018D
:1045180000F4FE501843A9F806000BF0BDFC00019A
:1045280089F804000BF0B8FC99F8043000F00F008B
:10453800184389F804000BF0AFFC89F805000AF06D
:1045480013FD00200BF0F4FCFFF7F7B90B4B98595B
:1045580003F050FD18B9322003F085FCF6E703F0AC
:10456800B5FE07F0D7FD064B064ADA60FFF7F3B948
:104578008C120020941200204410002024200020D7
:1045880000ED00E00400FA05041300200C2844D0D4
:104598000A284BD1534D54480BF052FD284623218D
:1045A80010F05FFF08B1401B20602368002B60D12A
:1045B8004C4823600021302210F01DFF98F800308D
:1045C800002B2DD1494B1B689B0615D5484B4949F3
:1045D8001B688A6B9A1A002A0EDB474A1278042A4B
:1045E8000AD9464A03F5123303F5F8738B63938AA5
:1045F8009BB283F488439382414B9B68002B6BD01A
:10460800404805B0BDEC028BBDE8F04F184705F0F7
:1046180007F9FFF792B90C2804D13B480BF010FDBD
:104628003A480DE07F2812D1FFF7F5B80D28B1D030
:104638007F2809D1013B2B4A354823600021D154FA
:104648000BF0FEFCFFF7E7B82F2B3FF6E4A8A0F12C
:104658002002D2B25E2A3FF6DEA813B920283FF422
:10466800DAA85A1C22601F4AD0540BF0E1FCFFF76D
:10467800D2B85A1EA95C202901D1134696E7194AD7
:1046880023600021D154234B234DD3F800A0D5F843
:1046980000B0DFF85090584610F0F1FE07463A4651
:1046A8004846594610F0F4FE1C4A28B919F8073054
:1046B80053445B785B0703D010359542E7D306E097
:1046C800954204D2781CEB684844984702E01448A5
:1046D8000BF0B6FC00236BE705B0BDEC028BBDE820
:1046E800F08F00BF602200209EA70108E81A002072
:1046F8008C2D0020D0100020F21A00200010004855
:10470800B02700200C110020E19B0108DC9B010868
:10471800089C0108180100204C830108FC8401084A
:10472800EC9B010810F80A3C0133DBB20A2B84BF6A
:1047380010F8131C044A00F80A3C82BF002322F830
:10474800113000F80A3C7047502C0020334A136C93
:1047580090681944081A40F68C23984270B513469D
:104768009160D06051603BD9127893F945108A4224
:1047780010460BD1111F082908D893F8461018299C
:1047880001D8013103E083F8442002E0002183F8D6
:10479800461093F944402149A24219D191F8474063
:1047A800B4B10C310024944206DA1D4D51F8046F5F
:1047B80025F814600134F6E70C2805D018490024C0
:1047C80021F810400130F7E71648017801310170EF
:1047D80083F84520002201211A7083F8471070BD24
:1047E80092F84710C9B1A0F2EF2440F2DA518C4296
:1047F80008D811780B2905D80B1D0131117042F822
:10480800230070BD002283F84720074B03F13002D4
:10481800002143F8041F9342FAD170BDBC01002067
:10482800502C0020B4060020C8010020024A136C56
:104838000133194411647047BC010020024B53F83E
:1048480020301B6819607047781C0020064B53F80D
:1048580020301A681B89A1F57A7159434FF47A738D
:1048680091FBF3F111607047781C0020054B9842CA
:104878000CBF054A054A138801339BB213800020F8
:10488800704700BF00540040181200201A12002080
:10489800F0B5046D8668236823F0010323608379EB
:1048A800054613F0020F40790CBF4FF0000E4FF48D
:1048B800005E13F0040F14BF4FF48067002710F058
:1048C800010F14BF042100218307206820F0010094
:1048D8002060626822F440524EEA02026260226856
:1048E80022F4B05323F00C0348BF41F008013B43C6
:1048F8000B432360A36895B023F44073A360684614
:1049080005F008FA284B9C4201D10C9B0EE0274B7E
:104918009C4201D10D9B09E0254B9C4201D10E9B85
:1049280004E0244B9C420CBF0F9B109B2268A87983
:10493800170448BF5B00B3FBF6F206FB1233B3EB78
:10494800560F236828BF01321E0441BF4FF6F0738B
:10495800C2F34201134041EA03026B7992B213F0A9
:10496800020FA28100F0010114BF4FF400320022AF
:10497800DC0748BF42F480322B6D11B159680A43F5
:1049880002E0596821EA02025A609A6801074CBF9E
:1049980042F0080222F008029A601A6842F0010206
:1049A8001A6015B0F0BD00BF003801400044004057
:1049B80000480040004C00403D4B1B78012B30B5AF
:1049C80014BF00240324B1B9036A23F0010303626E
:1049D8008169036A21F0F30123F00A0341F0010120
:1049E80042F001021A4341EA0411816102628369BB
:1049F80023F00C031BE004291DD1016A4FF6EF7365
:104A08000B4003628169056A120121F473414FF674
:104A18005F7342F0100241F480712B4092B213434D
:104A280041EA043181610362836923F4406383614D
:104A38008369836130BD0829016A1AD14FF6FF6383
:104A48000B400362C169036A9BB289B223F42063F5
:104A580043F4807321F0F30143EA022241F001019B
:104A680092B241EA0411C1610262C2694FF6F3735E
:104A780019E04EF6FF730B400362C369056A40F6FE
:104A8800FF41194045F6FF732B4043F4805343EA36
:104A9800023241F4807192B241EA0431C16102628A
:104AA800C2694FF2FF331340C361C369C36130BDAC
:104AB800B801002038B510F80E2C50F8043C044614
:104AC80052B9012200F80E2C20F80C1C997A1868AB
:104AD8000222BDE838406FE730F80C2C20F80A1C99
:104AE800891A89B220F8081C074A10F80F0C00250B
:104AF80022F8101004F80E5C1868997A2A46FFF715
:104B08005BFF04F8065C38BD502C0020044B53F8BA
:104B180020301BB107289CBF1B681960704700BF75
:104B2800E4020020084A13689B050BD5074B0021B7
:104B38001970074908684FF6FE7303400B604FF47D
:104B480000735360704700BF00000240B62D00207C
:104B5800300002402DE9F047664D2B6866490A7817
:104B6800581C02F0FF068E460AB10346F6E72B6092
:104B7800687BAB6895F80C80AA7B374639B2202948
:104B880000F09B80DFF880C10CEB81033CF821101A
:104B9800DC789B78C3F1FF039BB2002B65D0C3F18F
:104BA800FF0363434FF03C0C1B12B1FBFCF9B9F156
:104BB800050F5DD8DFE809F0030B1A293A4AE01A15
:104BC800DAB24143B1FBFCF01044C0B251E0B1FB92
:104BD800FCF00CFB101189B2DAB2C1F13C01E31A06
:104BE8004B432046B3FBFCFC94442CE0B1FBFCF0A7
:104BF8000CFB10115FFA83F8E21A89B24A43B2FB40
:104C0800FCF24244D2B2204632E0B1FBFCF90CFB84
:104C1800191189B25FFA83F8E01AC1F13C014843DF
:104C2800B0FBFCF04044C0B2224621E0B1FBFCF8E6
:104C38000CFB1811D8B289B2E31A01FB03F2B2FBDC
:104C4800FCFC224684445FFA8CF412E0B1FBFCF8C9
:104C58000CFB181189B2D8B2C1F13C01E31A4B43DD
:104C6800B3FBFCF20244D2B203E02246204600E045
:104C780044464FEA042C4CEA004C4CEA020C172339
:104C880006F117014FF0010808FA03F8C91A18EAE3
:104C98000C0F89B2DFF8748014BF4FF011094FF080
:104CA800090913F1FF3308F80190E9D218360137E2
:104CB800B6B2BFB2114BA04660E7AA73AB60104A08
:104CC800E98001238EF800300E4985F80C8040F207
:104CD8002A336873AE80536000234B620B889BB203
:104CE80043F001030B80136843F001031360BDE830
:104CF800F08700BF10110020B62D00201C110020E5
:104D08003000024000440140BA0E00205D0300203C
:104D180073B506460D46002401232A88A340134292
:104D28001AD0AA78009302F003038DF80430EB78C8
:104D3800022B03D0032B0CBF032301238DF805306E
:104D48003046C2F301136946C2F381028DF806307A
:104D58008DF8072005F054F90134102CDCD102B08D
:104D680070BD2DE9F04F734EF57B07460C4687B0B2
:104D780011469A4600686B1C914622464FF0020B7A
:104D8800F37308F061FC3B897868ADF8043001A939
:104D98008DF806B08DF807B0FFF7BAFF0023ADF81D
:104DA8000A30ADF81230ADF8163070230193BA7A94
:104DB8003C68CDF80CA0012306F110082D01ADF8D0
:104DC80008304FF48073A844ADF810B0ADF8143033
:104DD8000C2A7ED8DFE802F0077D7D7D0F7D7D7D82
:104DE800387D7D7D5E00204601A904F055FFA3694A
:104DF80043F0080326E0236A4F4823F01003236298
:104E0800236A6168A26922F0807222F4E642844231
:104E180042F4E04206D000F50060844202D043F03C
:104E2800300307E023F0E00321F4406143F030034E
:104E380041F480616160A261C4F838A02362A3696B
:104E480043F40063A36144E0236A3B4823F480737E
:104E58002362226A6168E369844223F0730343F0A2
:104E6800700306D000F50060844202D042F440721C
:104E780007E022F4606221F4405142F4407241F4A8
:104E880080516160E361C4F83CA02262E36943F0A9
:104E980008031DE0236A284823F480532362226A0A
:104EA8006168E369844223F4E64343F4E04342F44F
:104EB800405203D000F50060844201D141F48041A2
:104EC8006160E361C4F840A02262E36943F40063CF
:104ED800E3613A7B3B681AB15A6C42F400425A6467
:104EE8001A8892B242F001021A80BA7A0C2A18D8AB
:104EF800DFE802F0071717170B1717170F17171701
:104F08001300721903F134010AE0721903F1380130
:104F180006E0721903F13C0102E0721903F1400145
:104F2800116135444046A5F818906B6107B0BDE89B
:104F3800F08F00BF10110020002C0140F8B53A4E48
:104F48003A4C4000C7B24FF420453068C4F8D050FE
:104F5800D0F818E01EF4004F05D0AE46013DBEF172
:104F6800000FF5D116E0D0F804E0314D0EEA050542
:104F780045F490353D4345604FF42045C4F8D05082
:104F8800D0F818E01EF0020F2DD1AE46013DBEF15B
:104F9800000FF5D1C4F8D0501FE02946013D002983
:104FA800F8D081694906F8D5C4F8D0502049456839
:104FB800294041F0007141F4105141EA024139435E
:104FC80041604FF42041A2B1306885696D071ED455
:104FD80011F1FF31F9D2C4F8D010FFF747FC0030C7
:104FE80018BF0120F8BD4FF420458162C4F8D050A5
:104FF800D7E73068C4F8D0100B46826992060CD403
:105008001A46013B002AF8D1C4F8D030E5E7416AD6
:1050180003F8011B013AD2B2D3E7C4F8D0302023F9
:10502800C3610120F8BD00BF141200201011002038
:10503800009800FC400070B5C5B23248324B006899
:105048004FF42044C3F8D0408669360404D5264678
:10505800013C002EF8D113E046682C4C344044F053
:10506800807444F490342C4344604FF42044C3F8D3
:10507800D0408669B60729D42646013C002EF8D1CF
:10508800C3F8D0401CE02146013C0029F8D08169D2
:105098000E06F8D544681D49214041F0007141F4DD
:1050A8008031294341604FF42041C3F8D01084690E
:1050B800A40711D40C460139002CF8D1C3F8D0103C
:1050C800FFF7D4FB003018BF012070BD4FF4204417
:1050D8008162C3F8D040DAE782624FF42042C3F815
:1050E800D0208169890606D41146013A0029F8D1F1
:1050F800C3F8D020E4E7C3F8D0202023C3610120FF
:1051080070BD00BF1412002010110020009800FC90
:105118002DE9F0474D282DED028B044600F034862A
:1051280000F29480302800F0CF8651D8222800F071
:105138006D8423D8032800F0CC8114D8012800F00E
:10514800BC81022840F0FE8604200AF0F1FE4320CC
:105158000AF0BFFE4C200AF0BCFE46200AF0B9FE59
:105168004C2000F037BE042800F0BC81052840F030
:10517800E9861A200AF0DCFE0024DDE1282800F088
:10518800C28515D8242800F0A585262840F0DA869F
:10519800DC4C06200AF0CCFEB4F858010AF0CBFE2D
:1051A800B4F85A010AF0C7FEB4F85C0100F08FBDEC
:1051B8002C2800F0BB852E2800F059862A2840F0BC
:1051C800C18601200AF0B4FECE4B587900F002BE29
:1051D8003B2800F014841AD8362800F029860BD80A
:1051E800322800F0F185342840F0AC8648200AF0D7
:1051F8009FFE002500F02CBC382800F071853A2865
:1052080040F0A08604200AF093FE00F096BE4228E3
:1052180000F0ED850BD83D2800F0B182402840F021
:10522800918608200AF084FE002400F0D6BD4628A6
:1052380000F06F864B2800F09885452840F082865C
:1052480013200AF075FE002400F06DBE702800F0EF
:10525800EB8200F2E580692800F04C8200F2B6800B
:10526800662800F0A68100F2A680642800F07D81FF
:10527800652840F06786A44C0B200AF059FE208868
:105288000AF059FE6268A14B9A420CBF20896089D6
:1052980080B20AF050FE9E4B1B68C3F3C000C3F3F4
:1052A8008002800040EA4200C3F340021043C3F387
:1052B800401240EAC20003F0100318430AF03BFE14
:1052C800944B1A88E368247C02F0080103F44759D8
:1052D80049EA010903F4804149EA010903F400415C
:1052E80049EA010903F4803149EA010903F400316C
:1052F80049EA010903F4802149EA010903F400217C
:1053080049EA010903F4801149EA010903F000732D
:1053180049EA0303DFF81C9299F8009012F0010F94
:10532800C9F3800914BF4FF002084FF0000843EAA0
:10533800090312F0020F43EA080314BF4FF0040CEC
:105348004FF0000C12F0040F43EA0C0C14BF4FF09E
:10535800100E4FF0000E12F0400F14BF2027002748
:105368004CEA0E0E12F0100F14BF4FF40076002610
:105378004EEA070712F0200F14BF4FF4806500258E
:105388003E4312F4807F14BF4FF400600020354381
:1053980012F4007F14BF4FF400110021284312F4C7
:1053A800806F41EA000114BF4FF0806300230020A2
:1053B80019430346E9E0672800F02381682840F094
:1053C800C18510200AF0B4FD00248AE16C2800F0A1
:1053D800A48117D86A2800F0FF836B2840F0B285B3
:1053E80005200AF0A5FD4C4B18880AF0A4FD4B4B8C
:1053F80018880AF0A0FD444B93F8720000F00100F1
:1054080000F0E8BC6E28404D00F0948100F2C281A3
:1054180006200AF08DFD686E0AF096FD404B87E184
:10542800782800F0FB8018D8742800F032830AD856
:10543800722800F09183732840F0848508200AF0D0
:1054480077FD0124C1E3762800F0E68300F25A8351
:105458002F200AF06DFD334CC9E2A42800F0038424
:1054680014D87B2800F06982A02840F06B850C20B6
:105478000AF05EFD2C4B18680AF066FD2B4B186885
:105488000AF062FD2A4B186800F058BDF12800F0B8
:105498000181FE2800F00E84F02840F053851A4C54
:1054A80004200AF045FDA36CB3F85A000AF043FD46
:1054B800A36CB3F8580000F00ABC03200AF038FDCA
:1054C80000200AF006FD20460AF003FD0D2000F03A
:1054D80081BC0AF02DFD01200AF0FBFC0A200AF02D
:1054E800F8FCBEE306200AF023FD43200AF0F1FC95
:1054F80048200AF0EEFC46200AF0EBFC33200AF0C4
:10550800E8FCE3E3041300201012002000540040DC
:10551800E81A0020B01B0020661B0020681B002032
:10552800EC1200204F7C0108ACF7FF1FB0F7FF1FFB
:10553800B4F7FF1FB72D0020AA4B185D01340AF0FD
:10554800C8FC0B2CF8D10024A74B185D01340AF0D5
:10555800C0FC082CF8D10024A44B185D01340AF0D3
:10556800B8FC072CF8D100F0EBBC07200AF0E0FCEF
:10557800E7200AF0AEFC9E4B58790AF0AAFC0020FE
:105588000AF0A7FC042000F0D9BCA3420AD2994A29
:105598009D5C012202FA05F50D421CBF9A4010439A
:1055A8000133F2E70AF0D0FC914B93F8A40700F01E
:1055B80011BC12200AF0BCFC8F4B1B88B3F5806F1E
:1055C8008CBF0825012500248C4B33F9140090FB6F
:1055D800F5F0013480B20AF0AEFC032CF4D1884C0B
:1055E800A08D0AF0A8FCE08D0AF0A5FC208E0AF038
:1055F800A2FC608E0AF09FFCA08E0AF09CFCE08E54
:1056080065E310200AF094FC00247E4B185D0134F9
:105618000AF05FFC102CF8D100F092BC70200AF060
:1056280087FC0026764D0E24AB6C74432344013668
:10563800B3F819010AF07FFCAB6C2344B3F81B01E3
:105648000AF079FCAB6C2344B3F81D010AF073FC33
:10565800AB6C234493F81F010AF03BFCAB6C23446A
:1056680093F820010AF035FCAB6C234493F8210130
:105678000AF02FFCAB6C234493F822010AF029FCB2
:10568800AB6C1C44D4F823010AF05EFC082EC9D187
:1056980000F056BC7020564C0AF04AFC04F1700524
:1056A80094F8D0000AF015FC94F8D1000AF011FC27
:1056B80094F8D2000AF00DFC94F8D3000AF009FC23
:1056C80094F8D4000AF005FC94F8D5000AF001FC1F
:1056D800073494F8CF000AF0FCFBAC42E0D100F0AC
:1056E8002FBC494B185D01340AF0F3FB102CF8D19C
:1056F80000F026BC454D2878400000F0FE000AF076
:1057080017FC00242B789C4280F01A84404B33F815
:1057180014000AF010FC0134F4E73E4C06200AF0AD
:1057280007FC20880AF007FC60880AF004FC3A4B62
:105738001888CCE207200AF0FBFB384B1888FF28B2
:10574800A8BFFF20C0B20AF0C4FB354B186880F32D
:10575800100080B20AF0EFFBB5F868000AF0EBFB26
:10576800234B93F883212F4B186822B10A235843FF
:1057780080F3100001E000F30F0080B2A7E21C4C98
:1057880002200AF0D5FB94F8DE010AF0A2FB94F897
:10579800DD011FE30B200AF0CBFBEB6E18780AF053
:1057A80098FBEB6E58780AF094FB0026EB6E144CCD
:1057B8003344013618790AF08CFB032EF6D1E36ED8
:1057C800D8790AF086FBE36E98780AF082FBE36EDC
:1057D800D8780AF07EFBE36E58890AF0ACFBE36EDA
:1057E800187AF7E20C99010818990108ED98010850
:1057F800041300202112002016000020E6120020C9
:1058080010120020481200205C120020C020002046
:105818002C2C00203C290020F4120020D81A00204B
:10582800E41A0020E01A0020C64C1E200AF080FB73
:10583800A36C1B78022B4FF000056BD1A36C03EB14
:10584800850393ED080AB2EE048A20EE080A0FF0E9
:10585800E1FF80F30800C0B20AF03BFBA36CDFED68
:10586800BA7A03EB850393ED0B0A20EE270A0FF0B3
:10587800D1FF80F30800C0B20AF02BFBA36CDFED68
:10588800B37A03EB850393ED0E0A20EE270A0FF097
:10589800C1FF80F30800C0B201350AF01AFB032DDE
:1058A800CCD1072DA36C23D193ED110A20EE080A61
:1058B8000FF0B0FF80F30800C0B20AF00AFBA36C37
:1058C80093ED120A20EE080A0FF0A4FF80F30800F7
:1058D800C0B20AF0FEFAA36C93F84C3000EE103A0E
:1058E800B8EE400A0FF096FF80F30800C0B20BE054
:1058F8002B4458780AF0EDFAA36C2B44D87A0AF0B6
:10590800E8FAA36C2B44587D01350AF0E2FA0A2D17
:10591800C7D115E3A36C2B4458780AF0DAFAA36CC4
:105928002B44D87A0AF0D5FAA36C2B440135587D5C
:105938000AF0CFFA0A2DEDD102E33C200AF0F8FA7A
:105948000024804D9FED818AAB6C03EB840393EDBB
:10595800080A20EE080A0FF05DFF80B20AF0EBFAA1
:10596800AB6C03EB840393ED0B0A20EE080A0FF0EF
:1059780051FF80B20AF0DFFAAB6C03EB840393EDBE
:105988000E0A20EE080A0FF045FF013480B20AF033
:10599800D2FA032CD5D1072CAB6C16D193ED110A92
:1059A80020EE080A0FF036FF80B20AF0C4FAAB6C9A
:1059B80093ED120A20EE080A0FF02CFF80B20AF0CD
:1059C800BAFAAB6C93F84C000BE0234458780AF011
:1059D800B2FAAB6C2344D87A0AF0ADFAAB6C234424
:1059E800587D01340AF0A7FA0A2CD4D1A8E214F899
:1059F800010F002800F0A4820AF06BFAF7E70120F3
:105A08000AF096FA4F4B9B6C1878E3E150200AF0A5
:105A18008FFA00254B4B9C6C4D4B04EB85040C21F5
:105A280094F8792001FB0233013593F838000AF025
:105A380050FA94F87A000AF04CFA94F87B000AF0CD
:105A480048FA94F87C000AF044FA142DE2D177E27F
:105A58003C4B9C6C062303FB0544013594F8CE00AF
:105A68000AF037FA94F8C9000AF033FA94F8CA0031
:105A78000AF02FFA94F8CB000AF02BFA94F8CC002D
:105A88000AF027FA94F8CD000AF023FA0C2DDFD19A
:105A980056E24FF00008012600272A4B1A7C97424D
:105AA80027DA11330024FA5C294D0C2305F1300163
:105AB8006343595C914207D12B44586B0FF0DFFCCC
:105AC80082462EB9B14605E001341C2CECD10EE01B
:105AD80080440CE0D1450ADA0C2303FB04535B6BCA
:105AE80013F809000AF0F5F909F10109F2E701379D
:105AF800D3E7002E00F024825FFA88F00AF018FA43
:105B08000026C9E70F4D287C0AF012FA00242B7CE6
:105B18009C4280F015820F4BE65C00210C480C2259
:105B280000F1300702FB01F3DA5DB24205D103440C
:105B380093F838000AF0CDF902E001311C29EDD1C3
:105B48000134E4E7101200200000C84200007A4443
:105B5800507C010821120020D04C16200AF0E8F9E8
:105B6800B4F894010AF0E7F9B4F840010AF0E3F94F
:105B7800B4F842010AF0DFF9B4F844010AF0DBF99D
:105B8800B4F8D6010AF0D7F994F8EB010AF0A1F9B4
:105B980000200AF09EF994F8EC010AF09AF994F8BA
:105BA80083010AF096F994F890010AF092F900201E
:105BB8000AF08FF9BA4B9B6C0A20B3F9563093FB65
:105BC800F0F080B20AF0B7F98EE0E0B201340AF0E2
:105BD80080F9092CF9D1B3E110200AF0A9F9B14BE9
:105BE800B14C187800F002000AF073F9AF4B18783E
:105BF8000AF06FF920680AF0A7F960680AF0A4F9BA
:105C0800AB4B18880AF097F9AA4B18880AF093F951
:105C1800A34BB3F870005AE00AF03EF90746122089
:105C28000AF086F99E4C17B9666FA56F06E0102F2B
:105C380013BF0025E66FD4F880502E4638460AF088
:105C480048F930460AF080F928460AF07DF9D4F878
:105C580084000AF079F900200AF06DF900200AF0B2
:105C68006AF90020B6E08E4D95F888008000013072
:105C7800C0B20AF05DF995F888000AF02AF9002404
:105C88002E4696F888309C4280F05A818A4D285DCD
:105C98000AF01FF905F11003185D0AF01AF905F169
:105CA80020033035185D0AF014F9285D0AF011F95F
:105CB8000134E6E708200AF03BF900200AF03BF936
:105CC80000200AF038F900200AF035F900200AF01F
:105CD80032F935E104200AF02BF9704B98682DE170
:105CE80004200AF025F96D4C94F878010AF0F1F8CF
:105CF80094F87C010AF0EDF894F87B010AF0E9F8D1
:105D080094F87D0166E0654C07200AF011F9B4F8B3
:105D18007E010AF010F9B4F880010AF00CF994F841
:105D280082010AF0D6F8B4F88401D0E75B4C0C2065
:105D38000AF0FEF894F88E010AF0CBF8B4F898014E
:105D48000AF0F9F8B4F894010AF0F5F8B4F89601F5
:105D58000AF0F1F894F88F010AF0BBF8B4F89A0148
:105D68000AF0E9F8B4F89C01B1E74C4C04200AF0B9
:105D7800DFF894F8D4010AF0ACF894F8D5010AF0E9
:105D8800A8F8B4F8D601A2E74C4C4D4D207800EBAA
:105D98004000C0B20AF0CCF8002623789E4205F1F4
:105DA800020580F0CD8015F8020C0AF092F815F87B
:105DB800010C00EB800000EB800000F2EE2080B2C6
:105DC8000AF0B9F80136E8E701200AF0B1F8334BD8
:105DD80093F890010AF07DF8B2E0304B2344013487
:105DE80093F886010AF075F8082CF6D1A8E02B4C38
:105DF80010200AF09DF860790AF06BF8A0680AF0A4
:105E0800A3F894F88E010AF064F8B4F858010AF07F
:105E180092F8B4F85A010AF08EF8B4F85C010AF066
:105E28008AF8B4F87E010AF086F8B4F880014EE7E3
:105E38001B4B1A4C93F8C900C0EBC000C0B20AF063
:105E480077F804F118051F4A94F8F20192F9001046
:105E580043B2994278D092F90C10994274D092F9D1
:105E680018209A4270D00834AC42ECD168E0402047
:105E78000A4C0AF05DF804F14005B4F89C020AF0F7
:105E88005AF894F89E020AF024F8043494F89B0215
:105E98000AF01FF8AC42F0D152E000BF0413002012
:105EA80010120020EC1A0020F41A0020F21A002028
:105EB800F01A0020EE1A002099120020C0200020BD
:105EC800A2140020CC200020E0202D4C0AF030F84D
:105ED80004F18005B4F81E0200F03F000AF02BF828
:105EE800B4F81E02C0F386100AF025F894F81C02D4
:105EF800000909F0EEFF94F81C0200F00F0009F009
:105F0800E8FF043494F8190209F0E3FFAC42E1D148
:105F180016E00D200AF00CF8002009F0DAFF002046
:105F28000AF012F806E0174B185D013409F0D1FFAA
:105F38000B2CF8D100200AF007F800200AF004F82A
:105F4800012018E0002016E009F0C3FFB4F8F401BE
:105F580009F0F1FF94F8F60109F0BBFF94F8F70196
:105F680009F0B7FF94F8F90109F0B3FF94F8F801C4
:105F780009F0AFFF77E7BDEC028BBDE8F08700BF03
:105F8800041300200C9901082DE9F047C94CCA4EAA
:105F9800237886B00746002B00F0138232686368C6
:105FA800D31A7C2B40F20D82237A6260013323726C
:105FB8004FF0000808F12400BE4DC0B20BF05EFDA2
:105FC80005F10A0333F9183007EE903ABB4B1B88EA
:105FD800B8EEE77A07EE903AF8EEE77A08F10108AA
:105FE800C7EE277A9FEDB67A67EE877AFDEEE77AF5
:105FF800CDED037ABDF90C000BF02EFDB8F1030FBF
:10600800D8D130200BF03AFDB5F910000BF024FD83
:106018000BF02CFD2B7A9A072CD16A6841F2883351
:106028009A4218D910200BF029FD4FF064086869CE
:1060380090FBF8F000B20BF00FFD21200BF01EFDD5
:10604800686990FBF8F308FB13000028B8BF4042CA
:1060580000B20BF001FD14200BF010FDB4F918008C
:106068000BF0FAFC1C200BF009FD00200BF0F4FCEF
:106078000BF0FCFC237ADFF83C825B0740F07E8162
:1060880002200BF0FBFCD8F81C00DFF848926423D0
:10609800323090FBF3F000B20BF0DEFC0320B8F9CD
:1060A80026500BF0EBFC874B1B7813F0040F4FF0D6
:1060B800050A95FBFAF5ADB20DD008F5D77039464B
:1060C80001F065FE28B9D9F8003013F0100F18BF99
:1060D800002528B205E0D8F8F8379889B0FBFAF01F
:1060E80000B20BF0B9FCD9F800309F0740F18A8064
:1060F800DFF8E491B4F8FE7799F80030B4F8FC279B
:106108006C4D3F014FF06408BFB208FB02325B00E0
:10611800B2FBF3F347EA0327BFB2C3F303231F43DA
:1061280006200BF0ABFC38B20BF096FCB4F8FE3747
:1061380099F8001001339BB293FBF1F201FB123383
:10614800A4F8FE37D4F800389B7B012B05D1392001
:106158000BF094FCB5F9FC071AE0B5F8FC576E2370
:106168003A205D4315270BF089FC95FBF7F5AFB294
:10617800B7FBF8F528B20BF06FFC08FB15753B2050
:106188000BF07CFCA8B2451D0A2095FBF0F000B28C
:106198000BF062FC28200BF071FCD4F80438454D54
:1061A8000A2093FBF0F000B20BF056FC04200BF031
:1061B80065FCD4F8F837D5F808089A894FF6FF73C4
:1061C8009842A8BF1846C2B10028ACBF131A13469C
:1061D80007EE903A9FED3C7AF8EEE77A67EE877A19
:1061E80007EE102AB8EEC77AC7EE877AFDEEE77A8F
:1061F80017EE900A6428A8BF642020EAE07000B275
:106208000BF02AFCD4F80C382A4F9D0640F1AB80DD
:1062180097F8103898071DD511200BF02FFCB7F808
:1062280012082A4B4FF4F365684390FBF3F000B271
:106238000BF012FC19200BF021FCB7F812084543AB
:10624800642095FBF0F595FBF0F300FB135000B2CA
:106258000BF002FC94F81038B4F8145813F0020F3D
:1062680008BF002501200BF009FC28B20BF0F4FB55
:1062780009200BF003FC00200BF0EEFB144B94F804
:1062880016581A88B2F5967F0AD90A4B1B7A03F07A
:106298000F03072B04D842F20F75954228BF154605
:1062A80005200BF0EBFBD4F800385B7BC3B928B2B0
:1062B80033E000BFDC12002068290020160000200F
:1062C80000007A44B72D00200000C842A0860100D3
:1062D8000A01002044290020080100206666E63FE4
:1062E800A5F1200307EE903A1FED047AF8EEE77A5D
:1062F800F6EE006AC7EE877ABEEE007AF5EEC07A4F
:10630800F1EE10FA58BFB0EE667A77EE877AFDEEB6
:10631800E77ACDED037ABDF90C000BF09DFB94F8FC
:106328001028C94B910703D493F81728012A04D1E0
:10633800012384F81738C5481CE0D3F80038DFED8E
:10634800C46A93ED017AD3ED027A27EE267A67EED6
:10635800A67ABDEEC77AFDEEE77A8DED047ACDED2B
:10636800057A04A806E0BB4A92E8030004AB83E878
:106378000300184605F092FA0BF078FB237A282BD5
:106388001FD1B14B00221A723C2733684FF47A7040
:10639800B3FBF0F817200BF071FBB8FBF7F5B5FB72
:1063A800F7F007FB1050000200B20BF055FB182065
:1063B8000BF064FB07FB158000B20BF04DFB0BF0F4
:1063C80055FB94F82038A04D002B00F0628101F0B5
:1063D80023FDD5F82438A04AC31A9342074640F251
:1063E800C680002385F82A3885F82C38B5F8FC379C
:1063F800DAB21B0A85F8462885F8473885F83C281C
:1064080085F83D38D5F8542833689A1AD5F858389D
:10641800D97B4FF47A734B439A420ED38F4B1B6848
:10642800C5F8543895F85C38013B012B9FBF102301
:1064380085F82A38022385F82C380A20D4F804284D
:1064480092FBF0F284F84428121284F8452894F854
:106458001028D4F8083893FBF0F384F848381B1256
:1064680084F84938920794F81638774984F87738C9
:1064780003D42D2381F8783877E0042BD4F81898C2
:10648800D4F81C68DFF8E481754A8CBF33233223C3
:1064980081F878384FF0060C724B99FBF3F096FBB5
:1064A800F3F308FB009108FB036803EB83030CFB81
:1064B80001F103EB830391FBF2FE642502FB1E113D
:1064C8009B0091FBF5F184F8691809120CFB08FC94
:1064D80084F86A189CFBF2F143FA81F39BB202FB41
:1064E80011C292FBF5F284F86E28121284F86C3807
:1064F80084F86F281B0AB4F8122884F86D3824230E
:10650800534393FBF5F5B4F88A3884F8703800EBF8
:1065180080001B0A00EB8000800084F871380A2292
:10652800B4F81438B3FBF2F303F5FA739BB240FAEC
:106538008EF080B284F872381B0A4FEAD97984F851
:106548006708F60F000A84F8645884F87338C5F3AE
:106558000725B4F88C3884F8669884F8680884F8B5
:106568006B6884F8655884F87938C4F8247894F806
:106578008E88354DB8F1000F0DD1D5F8940801F08B
:1065880042FD012807D90228374E00F0628205F043
:1065980077F90123B370D4F898282B4D002A78D0C6
:1065A80095F88E683EB1D5F8A03840F6B731FB1A99
:1065B8008B4219D86DE00123D5F8940885F88E38F8
:1065C80004F08BF9D5F8A43893F9000002238DE87C
:1065D8004800082132464FF4964304F099F985F8AB
:1065E800A868C5F8940852E095F89C68CEB9D5F823
:1065F8009408C5F8986885F88E6804F06EF9D5F89F
:10660800A43893F9000001238DE848000821324698
:106618004FF4964304F07CF9C5F8940805F030F976
:1066280035E0013EF6B285F89C6895F8A81895F80B
:10663800A938EEB94A1C013385F8A82885F8A93885
:10664800D5F8940821E000BFDC120020F41A0020DD
:106658008096184BDC7D01083F0D03006829002057
:1066680040420F008096980016000020806967FF5E
:1066780012F8016BC5F89828701885F8A808013336
:10668800D5F8940885F8A938314601F0BFFCC4F85C
:10669800A07894F8AA38A24DF3B1D5F8AC38DBB19C
:1066A800D5F8B038C3B1C5F8B4381B689D4AC5F8E9
:1066B800B838D5F8BC381344187AFEF729FDD5F850
:1066C800B438987909F005FCD5F8BC380133092BA2
:1066D80088BF0023C5F8BC38934D94F8C0282E68AD
:1066E8008F4B002A00F0F081D3F8C428002A00F06C
:1066F800EB8193F8C838013B012B00F2E581D4F80F
:10670800C408874F01F07FFCE0B1D7F8C40801F056
:1067180077FC97F8C938D5F800907E2B80460ED1C3
:1067280002231B2887F8C83809D1D7F8C40801F014
:106738006AFC20B90123C7F8CC9887F8D03884F8C8
:10674800C988DCE7D7F8CC282B689B1A41F6583261
:1067580093421ED9032387F8C838B5E1734A32F843
:10676800130010B903464FF403600133B0F5C06F4E
:10677800DBB279D01ED9B0F5006F7FD032D9B0F531
:10678800036F3FD184F8D138D4F80C38644F990698
:106798003FD494F8D01894F8D138002900F05681E5
:1067A8002A68921B012AD9D984F8D138002384F8A1
:1067B800D03889E1B0F5007F43D007D8B0F5807FA5
:1067C80049D0B0F5887F00F08D80E6E7B0F5806F9E
:1067D80000F0B080B0F5826F00F0F580B0F5047F6E
:1067E800DBD123E0B0F5E26F00F08D80B0F5E46F07
:1067F80000F08E80B0F5E06FCFD184F8D138B4F9CD
:106808000A1089E0B0F5046F76D0B0F5026FC4D1F4
:1068180005E197F810389A07BBD5B7F81218242362
:106828004B431233642193FBF1F109E184F8D13829
:106838003F4B3B4F1B689B07ABD5B7F8FC370A218A
:10684800FDE084F8D1383A4B354F1B681905A0D5BF
:10685800D7F80418F4E084F8D138D4F80C38304F5D
:106868005A0796D57969EBE084F8D138304B2C4F2C
:106878001B681B058DD5D7F80818E1E0D4F80C186B
:10688800274A84F8D1388F0683D592F810188807DC
:106898007FF57FAFD90712D5D2F81C3883EAE371A8
:1068A800002BA1EBE37101EB51014FF01902B1FB91
:1068B800F2F1ACBF41F0004141F040410FE0D2F8A5
:1068C800183883EAE371A1EBE371002B01EB510166
:1068D8004FF01902B1FBF2F1B8BF41F080414FF41B
:1068E80000608BE084F8D138D4F80C380C4F5B0783
:1068F8007FF54FAF3969A3E0B4F9181084F8D1389F
:10690800642359437AE084F8D138B4F90C1003E0D1
:10691800B4F90E1084F8D1382C2391FBF3F16DE013
:10692800DC120020DC7D0108682900202A9D01086E
:106938004429002084F8D13894F8D238644A0133C5
:10694800DBB2032B88BF012382F8D23894F8D2181F
:1069580042F2107359435F4B1B78D80748BF013187
:106968009A0748BF02315F07B4F8D43848BF0431EA
:10697800D80748BF0A319A0748BF14311F0648BFD5
:106988002831D80548BF28315A0748BF64311F0746
:1069980048BFC831980548BF01F5C8719A0648BF75
:1069A80001F57A71DF0648BF01F5FA61580648BF5C
:1069B80001F57A614FF4806004F02EFF444B002209
:1069C80083F8D028E5E6D4F80C18DFF8048184F8B9
:1069D800D13811F0200717D098F8102812F0020FBC
:1069E80014BF4FF47A71002112F0010F14BF4FF455
:1069F800FA6300230B4494F81618194404F00CFFAA
:106A0800002384F8D038C4E6334B1B6819067FF599
:106A1800C0AE394604F000FF88F8D078B9E684F8AB
:106A2800D138D4F80C382A4F9A067FF5B2AE97F8C9
:106A380010389B077FF5ADAEB7F814386421594379
:106A480004F0EAFE002387F8D038A2E684F8D138AB
:106A58003AE0B37823B1C5F8907886F802809AE5D1
:106A6800D5F89038FB1AB3F57A6FFFF494AD01238B
:106A7800D5F89408B37001F0C3FA0646D5F894081F
:106A880001F0BEFA76067FF486AD8A2802D08E28F9
:106A98000DD080E5D5F80C3898067FF57CAD95F8D3
:106AA8008E38002B7FF477AD05F65D0306E095F888
:106AB8008E38002B7FF46FAD05F62803C5F898389B
:106AC8002D2385F89C3866E506B0BDE8F08700BF41
:106AD800DC120020B72D0020442900200D4B0E4960
:106AE8001A680E4B92B213445B000D4A1B68C3F33D
:106AF800090310B5136013689BB201335B100022C1
:106B08009A4206D0074851F8044B20F81240013247
:106B1800F6E710BD505C0040206200401E300020A7
:106B2800A4280020A9280020014B00221A607047E1
:106B3800A028002013B506220446A82119206B4678
:106B4800FEF7FCF9F8B19DF800309DF8012043EA02
:106B5800022202219DF8033012B292FBF1F2228048
:106B68009DF8022042EA032212B29DF8053092FBFA
:106B7800F1F262809DF8042042EA03231BB201204F
:106B880093FBF1F3A38002B010BD08B52421802245
:106B98001920FEF74FFA642001F065F920219722A9
:106BA8001920FEF747FA0A2001F05DF91022232187
:106BB8001920FEF73FFA642001F055F9024B4FF413
:106BC80080521A8008BD00BF16000020154B37B54B
:106BD800082205461A85E82009F0F4FF0024002061
:106BE80009F0F0FF0DF804000134062CF7D10D4B25
:106BF80008229A619DF800209DF8013043EA02239B
:106C08002B809DF802209DF8033043EA02236B8015
:106C18009DF804209DF80530012043EA0223AB804B
:106C280003B030BD00100048274A73B55369274C9C
:106C380043F40013536103236946082501268DF8A0
:106C48000530204600238DF806308DF80730009572
:106C58008DF8046003F0D4F91D4AA561138823F068
:106C680040031B041B0C1380138823F038031B04F8
:106C78001B0C2B43138013889BB243F040031380F3
:106C88002420258509F09EFF802009F09BFFA5613F
:106C9800642001F0DDF82585202009F093FFAF205E
:106CA80009F090FF3046A56101F0D2F82585232030
:106CB80009F088FF602009F085FFA561642001F0D4
:106CC800D2F802B070BD00BF0010024000100048AA
:106CD80000300140024B4FF480221A60704700BF19
:106CE800140401402DE9F04F944D954C2B68954EB6
:106CF8009BB22380228831880A40900585B007D549
:106D08004FF6FF53904A2B6013780133DBB21370B0
:106D180023880B40190440F143830023ADF80A305F
:106D28002B6887499AB21804228040F139830B886E
:106D380003F00F038B70002B40F00483834A844FC9
:106D4800136884489BB23B803B8803F03003038080
:106D58003B8803F440533B80D2F800E04BF6BF7306
:106D68000EEA030383F4005383F0200343F4004343
:106D780043F0800313600B8813F0100F804626D170
:106D8800116848F60F730B40734913600B681A7A41
:106D9800022A894601D0042A05D102F09DFDD9F8BE
:106DA80000301B7A3FE1062A6ED15A78052A09D1AC
:106DB8001A78520606D1D87802F072FD674B1B6824
:106DC8001B6A9847664B1B689B6898475CE013688A
:106DD8009BB2ADF80A30BDF80A301B0540F1F381CB
:106DE80011685D4840F68F730B405E4913600A686E
:106DF8005D4B92B213445B0081461A68036893F8AE
:106E080008E0BEF1090F8A4617D092B2520002F18B
:106E1800804202F5C04211781970517859709188F2
:106E2800C8B2090A41EA002159801189C8B2090A81
:106E380041EA002199809289DA8001221A72DA885F
:106E480093F801B0002A40F0F1801A7812F07F021E
:106E580050D1BBF1090F10D1DA78012A00F2CA80AB
:106E68009978002940F0C6809988002940F0C280AE
:106E78009A723A4B1B685B68BAE0BBF1050F10D1F8
:106E880093F90320002A01DA0823CCE09A78002A33
:106E9800FAD19A88002AF7D19B7A002B00F0B480A7
:106EA800F2E7BBF1030F0FD1DA78012A40F0A28094
:106EB8009A88002A40F09E805A7A42F020025A723C
:106EC800264B1B68DB6993E0BBF1010F40F0928011
:106ED800DA78012A40F08E809A88002A40F08A8069
:106EE8005B7A980640F1868002F0A4FD002800F045
:106EF8008B807FE0012A39D1BBF10B0F7AD1184A78
:106F080058791268D97892699047D9F800309A7AF6
:106F1800002A6FD000286DD11A79002A6AD19B788F
:106F2800002B67D10D4B1B68DB6898470A4B1B6821
:106F38005A79DA72DA781A7366E000BF445C004066
:106F4800B41B0020EA280020B82D0020005C004077
:106F5800F2200020F02000201C200020202000200B
:106F68001C220020505C004004300020022A41D13D
:106F7800BBF1010FB8D0BBF1030F3BD1587920F01A
:106F8800800E4FEA8E0202F1804101F5B84110F0FF
:106F9800800F096814BF01F0300101F44051BEF1BF
:106FA800030F27D8B3F802E0BEF1000F22D109B3CE
:106FB8009B7AFBB102F1804202F5B84201061368E0
:106FC8004BBF23F4E04323F4804323F0400323F032
:106FD80070034BBF9BB29BB283F0100383F48053C2
:106FE80043F4004343F080031360A94B1B689B697B
:106FF800984709E0A74B1B6858465B6998470328E0
:1070080010D000287FF440AFDAF80020A24B92B2EB
:1070180013445B001A6800221A603023A8F8003075
:10702800062300E00923D9F8002065E1BBF1060F2B
:1070380013D11A7850067DD19A78964B012A02D13D
:107048001B68DB696AE0022A02D11B681B6A65E0DB
:10705800032A6FD11B685B6A60E0BBF1000F3AD16D
:107068005988002966D15A6822F47F42B2F5003F58
:1070780060D11A7812F07F0204D19B88002B00F0AF
:10708800F48157E0012A0AD1824A58791268926934
:10709800904700284ED1D9F800309B7A17E0022A91
:1070A80048D15A7902F00F010BB29B0003F18043DB
:1070B80003F5B84312F0800F1B6814BF03F03003C8
:1070C80003F44053032935D812F0700F32D1002B46
:1070D80040F0CB812EE0BBF1080F04D11B78590694
:1070E80000F0C58126E0BBF10A0F23D11A7802F01F
:1070F8007F02012A1ED19A7AE2B15988D1B95A6819
:1071080022F47F42B2F5803F14D1624A587912685E
:1071180092699047002800F0AC810BE053B1D9F890
:1071280000204FF0000AA2F812A093615046984739
:1071380050460BE0574BD9F800201B6850781B6964
:107148009847032802D1554B1B6806E0D9F8003050
:107158001A8A4FF6FF718A4201D1092203E00228F8
:1071680000D012B908221A72C7E093F9001000295A
:1071780023DAD98803910398DFF818E1824202D90B
:10718800039A1A8211E08A420FD2DEF8001091F8B1
:107198002C00824201D2002105E092FBF0F100FBB5
:1071A800112212B901213E4A1170DEF8002092F82E
:1071B8002C209A8202F090FB9FE003221A724FF46F
:1071C80040533B8099E0BDF80A301BB2002BBFF654
:1071D800A7AD116840F68F730B4013602F4AD2F8A1
:1071E800009099F80830022B934600F08280042B17
:1071F8007FD0032B01D0052B75D1D9F81830B9F8F9
:1072080010209BB9B9F81020002A4FD04FF44053F2
:107218003B80244B1968204B89B20B445B001968EA
:10722800002119603023A8F800303FE0002AE9D097
:10723800B9F814A0924528BF92461FFA8AF2104660
:1072480001929847019AB9F810309B1AA9F81030A2
:10725800B9F812301344A9F81230124B1A68124BBD
:1072680092B213445B000AF1010A1B689BB203F156
:10727800005303F540534FEA6A0A5B000021514569
:10728800C0D053F8212020F811200131F7E700BFC2
:10729800202000201C220020023000201C2000207A
:1072A800B92D0020505C004004300020B9F814309B
:1072B8009342DBF8003001D8032201E012B1052225
:1072C8001A720CE0062119726C4B19686C4B89B262
:1072D8000B445B0019681A603023A8F80030DBF80B
:1072E80000301B7A06E0072B03D1664B1B68DB686E
:1072F80098470823DBF80020137202F07FFB624BEB
:107308001A684BF6BF7313403A88D2043A8848BFCC
:1073180083F480539004B8F8002048BF83F40053E6
:10732800D106B8F8002048BF83F01003920648BF82
:1073380083F0200343F4004343F08003524A9BB296
:1073480013602DE09A0002F1804202F5B8421168FC
:1073580089B2ADF80A10BDF80A1009B2002909DA95
:10736800106840F68F7101401160013B474A52F89E
:1073780023309847BDF80A301F067FF5D1ACA178B5
:107388008B0003F1804303F5B84348F60F72186881
:1073980002401A603D4B03EB81039B699847BFE4A9
:1073A800228833881340590505D54FF6FF332B60E3
:1073B800374B5B689847228831880A40920444BF5B
:1073C8004DF6FF732B602388324A0B40DB0452D5FD
:1073D8004EF6FF732B600023D370D378052B41D86A
:1073E800DFE803F0030D1418222DA368294D1BB9FB
:1073F80008F016FC062300E00523EB703BE008F0DC
:107408000FFC0423E3700123A36034E002232371FB
:10741800032328E02379013BDBB22371237953BB93
:107428001C4B0422DA7026E01B4A13689BB243F017
:10743800100313600523E3700A2323711BE02379EB
:10744800144A013BDBB22371237903F0FF0093B99F
:1074580011490C684FF6EF7323400B600623D37075
:10746800906008E00623E37005E00C4B57E60C4BF0
:1074780055E60C4B53E605B0BDE8F08F505C004074
:10748800023000201C220020005C0040F07D010832
:1074980020000020B41B0020405C00400B95000831
:1074A800B195000891950008704770477047FEE74E
:1074B800FEE7FEE7704730B50024E3B293420DD2F1
:1074C800030F092B94BF3033373301F8143001EB25
:1074D8004403002500015D700134EEE730BD024829
:1074E800024906F048B800BF00480140C01D00200E
:1074F8000148024906F03FB800400140701D0020D5
:107508000148024906F037B800340140481D002000
:107518000148024906F02FB800340140481D0020F8
:107528000148024906F027B800080040201D002045
:10753800034B4FF4085208B19A6170471A85704797
:1075480000100048034B4FF4085208B11A857047E1
:107558009A617047001000482DE9F04F2DED028B1D
:1075680085B006460393894B1B889807914636D504
:10757800109B8748DC89B0F900301B1B03F2F31518
:1075880040F2E632954203D8002BB8BF5B4201E0D7
:107598004FF4FA73B0F90220121B02F2F31440F20E
:1075A800E630844203D8002AB8BF524201E04FF4C3
:1075B800FA729342B8BF1346C3F5FA73052293FBD8
:1075C800F2F30A22643B5343327FD21053436422BE
:1075D80093FBF2F3134423EAE373DBB200E0642382
:1075E8000093CB1C0293B2460024029BDFF8C081B3
:1075F80013F8015F0293022C4FEA440705D1B8F94A
:1076080004201B3555436D114AE0624938F814309F
:1076180031F91410022013FB0011C9F1000399423B
:1076280003DB49450B46A8BF4B465B4931F907B018
:10763800CBEB030B039B33F914309B4406F062FD3C
:1076480088B107EE90BA554BB8EEE70AB2EE048A55
:10765800185D80EE080A09F027FB20EE080AFDEE07
:10766800C07A17EE90BA494B1988CA0714D438F96A
:1076780007301B355D438B074FEA251510D5B37CC2
:107688009DF9002003FB0BFB02FB0BFB64239BFB18
:10769800F3FB05EB2B1503E0357A05FB0BF52D11F4
:1076A800DFF810E13E4B0422DB5F93FBF2F314F8A2
:1076B8000E2090469AF80120EB1A5A4341464A4355
:1076C800642192FBF1F2D2110192364A9AF80B50DA
:1076D80010880EF1040C00FB03F25CF82410D2129F
:1076E80005FB0215B5F5001F2F4AA8BF4FF400157A
:1076F8000EF110019542B8BF154651F8242041F803
:1077080024309A1A00094FF6FF7396F85010B3FB0D
:10771800F0F0424393114CF824504FEA840B6D1358
:1077280000EE103A59B10EF11C00B8EEC00A00EB99
:10773800C400DEED0D0A04F071F9BDEEC00A9AF836
:1077480015300199019810EE102A534342465A43C6
:107758006918642392FBF3F3144A1B121944D1539A
:1077680002F1080101344BF8010002F11401203242
:10777800032C4BF801504BF802300AF1010A7FF450
:1077880034AF05B0BDEC028BBDE8F08FB01B002014
:107798002C2C0020AE2D00203C290020287E01083A
:1077A8003C120020101200200000E0FFF81B00200F
:1077B800FC120020C01B00202DE9F04F2DED0A8B94
:1077C80085B08246039390F85030029190461BB1E1
:1077D800322BA8BF322300E0012307EE903AB8EE1F
:1077E800E7BADFEDD97AD94BDFEDD9BA1B88D94C86
:1077F800019487EE8BBA002B08BF0123D64D07EE04
:10780800903AF8EEE79A238869EEABBA13F0020FC4
:107818003BEE2BBA8BEE8BBA26D0B5F90030B5F912
:10782800022083EAE37182EAE270A1EBE371A0EB44
:10783800E27088420646B8BF0E46B6F5E17F16DA12
:107848008842DFEDC6AA05DD002AD8BF524207EEFE
:10785800902A04E0002BD8BF5B4207EE903AF8EE7E
:10786800E77AC7EEAAAA04E0DFEDBDAA01E0F7EEC9
:1078780000AA9FEDBB9ABB4C56464FF0000BB0EEEA
:1078880049AADFF8189339F91B300CEE103AB8EE14
:10789800CCCAF5EE047A35F91B302CEE27CA08EE6F
:1078A800903A019BBDEECCCA1988F8EECC7A9FEDD0
:1078B800AECA89074FEA4B0727EE8CCAF8EEE88A6A
:1078C80000F08580A94931F91B3007EE903AF8EEAF
:1078D800E77AB0EE007AE8EE877AC8F10000FDEEAC
:1078E800E77A17EE901A814203DB4145A8BF41466B
:1078F80008469F49039B795E401A33F91B100844D8
:1079080007EE900AB8EEE78A06F0FCFB50B19949F9
:10791800B2EE049A88EE090A11F80B0009F0C4F9CE
:1079280020EE098A9AF81C30DFED936A0AEE103AC5
:107938009AF8083007EE903AF8EE677AB8EE4AAA55
:1079480068EE277AB1EE047A67EEA67A2AEE077A0D
:10795800FDEEE77A17EE901AF1EE477ABDEEE7AA48
:107968001AEE103A994208DBBDEEC7AA1AEE103A91
:107978008B42A8BF0B460AEE103A804901EB8B01F7
:10798800D1ED007AE8EE2B7ABBEE0E7AF4EEC77AE8
:10799800F1EE10FAB8EECAAA09D4B3EE0E7AF4EEF4
:1079A800477AF1EE10FAC8BFF0EE477A01E0F0EE40
:1079B800477AC1ED007A9AF8123009EE103AB8EE1B
:1079C800499A67EE897A9FED6E9A27EE899A019B0C
:1079D8001988CA0750D439F907000028B8BF4042AF
:1079E800B0F5206F02DD0020206025E09FED657A6C
:1079F800737868EE877A07EE103AB8EE477A87EE22
:107A0800877AD4ED007A37EE4C7AE7EE2B7A9FED41
:107A18005E7AF4EEC77AF1EE10FA09D49FED5B7A3C
:107A2800F4EE477AF1EE10FAC8BFF0EE477A01E0BB
:107A3800F0EE477AC4ED007AF37AD4ED007A08EED6
:107A4800103AB8EE488A8B0768EE277A9FED508A7D
:107A580027EE888A14D578EECA8AF0EE4A7AEAEEDA
:107A6800A87A38EE498AF0EE678AF0EE497AEAEEAB
:107A7800887AB0EE678A03E0B0EE498AF0EE4A8A67
:107A8800DFF81C919FED437A09F1780109F17C0038
:107A98001BF8013007EE903AF8EEE77A4FEA8B01CF
:107AA80067EECC7A0844E7EE878A0434013690ED15
:107AB800007A80ED00CA3CEE477A09F1840087EE2F
:107AC8002B7A0144D1ED007A37EE677AF0EE68CA76
:107AD800EBEE077A3CEE880AC1ED007A09F18C01D9
:107AE8001BF8013008EE903AF8EEE88A67EEA87ABB
:107AF800DFED298A67EEA88A30EE680A0DF08AFE63
:107B080009F13801FDEEECCAC8531CEE903A09F1B0
:107B18004001BDEEC88AF1EE688A41F82B30FDEECF
:107B2800E88A09F14C0118EE103A41F82B3009F1B6
:107B3800580118EE903A4F4641F82B30BBF1000F30
:107B480030D14FF0010B9CE683F9223E1012002041
:107B5800BD378635B01B0020FC1200200000E14331
:107B680000000000241C0020CDCC4C40AE2D00208D
:107B78003C290020287E01086F12033C301C00209D
:107B88000AD7A33D0000A043000040C300004043C3
:107B98000AD7233CA69B443BF7CC92383C120020E2
:107BA800C01B0020029AB5F9043094796400283487
:107BB8005C434A4BB3F9043000EE103ABAEECF0AF0
:107BC8000DF028FE6411201A002C07EE900AB8BFA9
:107BD8006442322CF8EEE76A03DD0023C9F80C3062
:107BE80029E0FDEEE99A19EE903A23F0030307EE37
:107BF800903AF8EEE79ADFED3A7A9AF80D30C9EE46
:107C0800A77A07EE103AB8EE477AD9F80C3026EE84
:107C1800877A67EE277AFDEEE77A17EE902A134403
:107C2800304A9342A8BF13462F4A9342ACBFC9F8C3
:107C38000C30C9F80C20FB685B13B3F5807FA8BF34
:107C48004FF480736FF0FF029342B8BF134607EEFC
:107C5800903AF8EEE78AFDEEE67A9AF8032017EEF6
:107C6800903A53439B1107EE903A97F88F30032BC5
:107C7800B8EEE78A14D9BAF84E20B2F5FA7F0FD2D7
:107C8800FDEEC87A534217EE901A994204DB9142EE
:107C980017EE903AA8BF134607EE903AB8EEE78A77
:107CA80038EE280ABDEEC00A8DED010ABDF9043090
:107CB80000EE103AB8EEC00A0DF0ACFDBDEEC88A71
:107CC800FDEEE88A0023B88787ED128AC7ED158A8A
:107CD8003B6605B0BDEC0A8BBDE8F08F3C12002076
:107CE80000803B45FEFFFF0F020000F010B544780E
:107CF8000078002202FB02F3193B634303F6C41326
:107D0800534340F6C411434393FBF1F3034921F86D
:107D180012300132072AEDD110BD00BF501C0020DF
:107D28000430114B33F91000B0F5617F10B506DB54
:107D380040F6330398420246A8BF1A4601E04FF4C2
:107D480061720C78192340F2833013FB04049442C7
:107D580007DA497813FB01039342B4BF00200120DE
:107D680010BD002010BD00BF2C2C002010B500F164
:107D7800500302788A4203D18478C278944204D3AB
:107D880004309842F5D1002010BD012010BD0B4BE6
:107D98001B6813F4805F0A4BB3F9063005D0C0891D
:107DA800421A934207DD084400E0008A8342B4BFC8
:107DB8000020012070470120704700BF442900209F
:107DC8002C2C00201FB5094B1B681B030AD58DF806
:107DD800040001230D2001A98DED030A8DF805305B
:107DE80003F08AF905B05DF804FB00BF44290020C0
:107DF8001FB5084B1B681B0309D58DF804000291B9
:107E080000230D2001A98DF8053003F075F905B0A0
:107E18005DF804FB4429002010B50A4A0A4B116892
:107E28009B6800BF12689142F7D1084AD2F8A04077
:107E38004FF47A7000FB04F2D31AB3FBF4F300FB9F
:107E4800013010BD6829002010E000E0C01B0020B0
:107E580038B50446FFF7E0FF0546FFF7DDFF401B96
:107E6800A042FAD338BD10B504462CB14FF47A704D
:107E7800FFF7EEFF013CF8E710BD024A1368013333
:107E88001360704768290020024BD3F8A43003B16F
:107E980018477047C01B0020014B1B68184700BFDC
:107EA800902D002010B50020FFF7F6FF074B0024A7
:107EB8001C7009F04DFD064B83F8A840C3F8AC4090
:107EC800A3F8B040C3F8B44010BD00BF302D002067
:107ED800C01B002010B510B9BDE81040E2E7002330
:107EE8000C225A430C4C1119125D824203D0013303
:107EF800102BF5D110BD094BD3F8B40018B14A784E
:107F08004078824206D20022C3F8B410A3F8B02009
:107F1800C3F8AC2010BD00BFE4870108C01B0020D7
:107F280010B540001428A8BF14200023074A0221D6
:107F380099540B4499181424834201F8014CF5DB39
:107F4800FF21D1540F20BDE81040C3E71C290020B1
:107F58002DE9F84380460B25013D3FD0224B4FF4D5
:107F680088429A614FF488521A8508F1010632272F
:107F78004FF005091C4CA38A9BB283F48843A38263
:107F8800A38A9BB283F48853A3820120FFF784FF5E
:107F98003846FFF768FFA38A9BB283F48843A3821D
:107FA800A38A9BB283F488530020A382FFF774FF4F
:107FB8003846FFF758FFB9F1000F08D0B9F10109A9
:107FC800D8D14FF4FA70FFF74EFFFA27D2E7013EF7
:107FD800D0D14FF47A70FFF746FFBDE7034B044A50
:107FE800DA60BDE8F88300BF0010004800ED00E04B
:107FF8000400FA0503681B6918470368DB6818471B
:1080080003689B68184703685B68184703681B6820
:1080180018472DE9F84FB0F90230934218BF0023F2
:108028002DED028B18BF0370057804460E46914665
:10803800002D40F08B8007EE902A9FED770AF8EE2E
:10804800E77AB6EE008A27EE800ADFED747A20EE32
:10805800270AA04620EE080A0DF052FCDFED706AF0
:1080680060EE266AB7EE006AB0EE667AA0EE007A95
:1080780040F2DC536365D0EE006A1023A4F8523056
:1080880037EE067A76EE866AC6EE077A1823A4F8E3
:108098005030274684ED046A27EE807A27EE007A6E
:1080A80077EE075A84ED017AC4ED025A70EE005A51
:1080B80084ED037AB8EE007AA5EE807A27EE877A07
:1080C80067EEA67A84ED057AC4ED067ADFED557A77
:1080D80098ED047A27EE277AF0EE678AB5EEC07A33
:1080E800F1EE10FA4CBF77EE487A77EE087A013550
:1080F80017EE900A09F0A4FFD8ED017A67EEA87A86
:10810800C7E90E01F5EEC07AF1EE10FA4CBF77EE32
:10811800C87A77EE887A08F1040817EE900A09F011
:108128008FFF032DC7E9080107F10807CED1A6F292
:10813800DC531B042367E3676367C4F88030A367D5
:10814800C4F884300123A4F802902370D4F8549022
:10815800B4F95280636A276A206FE26FD4F840C08E
:10816800D4F88010C4F88020C9EB060606FA08F691
:108178004FEAE67B734307FB0B332667A7FB0667CB
:108188001F44636C656F60674FEAE27B53430CFBE7
:108198000B3EACFB02237344B61A67EB0307E36A92
:1081A800A26AC4F884104FEAE07B434302FB0B3E0B
:1081B800A2FB00237344B6185F41E36CA06CB4F9CA
:1081C8005020A5674FEAE17B4B4300FB0B33A0FB34
:1081D80001011944636B361A206B4FEAE57B05FBF6
:1081E80003F300FB0B3367EB0107A0FB0501194400
:1081F8008019794109F0FAFE08F1FF320123934012
:10820800E067C01841EBE371424609F0EFFEBDECB0
:10821800028B4844BDE8F88F6F12833ADB0F494060
:10822800F404B53F0000804B2DE9F8430024244BAB
:1082380093F88F60E0B2B0420DD203EB8003214A7D
:10824800D3F8B83032F810101BB10B2801D8DB680E
:1082580098470134EBE71C4B1B685B032DD50024C2
:108268002346E2B2B24228D2DFF8549009F1B807A7
:108278004FEA840857F8242055689D4215D02846AF
:1082880005F030FAEFF31283502282F31288282186
:108298006A6A01FB00900132C0F80C216A6942F059
:1082A80001026A61DBB283F3118857F808301B6852
:1082B80000221A6001342B46D3E7BDE8F88300BFDB
:1082C800C01B00205C1200204429002008B50E4B7A
:1082D8001B6813F4805F0D4B14BFD3F82822D3F822
:1082E8002C2293F88F1092880023D8B2884204D2A7
:1082F800074820F813200133F7E7FFF795FF3220EE
:10830800BDE80840AFE500BF44290020C01B00209D
:108318005C1200200A4B1A680A4B30B502F48052EE
:10832800D3F82842D3F82C5200230AB1A18800E0E0
:10833800A988054820F8131001330C2BF5D130BD5E
:1083480044290020C01B0020F228002070B5124DDF
:108358000024214605F23120702285F830420DF0C4
:108368004AF82146D5F8A4320B4A0B4493F9020087
:1083780080B102F231241E680E5108199C8884804D
:108388009B79837192F8303207310133702982F872
:108398003032E7D170BD00BFC01B0020094B1A68FE
:1083A8000E2303FB0020437AFF2B07D0064A1278DE
:1083B8009A4203D9054A32F8130000E0808800B2D7
:1083C800704700BF9C220020C02000202C2C0020D9
:1083D80038B5294C2DED048B94EDAA8AB0EE480AE5
:1083E800054603F0CBFDF0EE408AB0EE480A03F0F4
:1083F80062FD94EDAB9AB0EE408AB0EE490A03F004
:10840800BDFDF0EE409AB0EE490A03F054FD95ED3B
:10841800017AD5ED027A95ED006A68EE676A27EE73
:10842800088AE7EE286A68EE000A67EE807AE6EEC8
:10843800290AB0EE660AE7EEA80A0DF0EDFADFEDBC
:108448000F7A20EE270ADFED0E7A80EE270AD4EDA8
:10845800AC7A30EE270AF2EE047A80EE270A0DF0A5
:10846800D9F9BDEC048B83B21A0444BF00F5B4708B
:1084780083B218B238BD00BFC01B00200000E14421
:10848800DB0F494001380A4B042804D8DFE800F024
:108498000507090B0D00074A08E0074A06E0074AE6
:1084A80004E0074A02E0074A00E0074A1A607047FA
:1084B8000C010020C1E7000861750008A1EA000866
:1084C800A5E4000831E10008C17700086D4B6E4A49
:1084D8009FED6E7AD2ED007ADFED6D4ADFED6D3AF1
:1084E80030B51C88B3F90AE01D8A06EE904AB8EE4A
:1084F800E76AF8EE666ADFED687AB3F9044067EE7A
:10850800E67AB7EE004AE6EE077A9FED647A67EE00
:10851800666A9FED637AE6EE076A27EEA77A07EEAA
:10852800904AB3F902409FED5F6AF8EEE77A67EE8A
:10853800277A07EE104AB8EEC77ADC89E6EE877A22
:10854800B6EE007AFDEEE76A87EE866AC3ED066A44
:10855800F8EEE66AD2ED017A9A89E6EE874A06EEE7
:1085680090EAB3F908E09FED507A05EE90EAF8EE4C
:10857800E66AF8EEE55A66EEA46A65EEA45A66EE77
:10858800A46AB3F806E0E6EE875A65EE875AA5EEC8
:10859800A34AF0EE445A04EE10EAB8EE444A25EE37
:1085A800844AB5EE404AF1EE10FA5BD02DB205EEE2
:1085B800905A24B224EEA45A07EE104AF8EEE55A6F
:1085C80012B265EE255AB8EEC75A65EEA35A64EEA4
:1085D800854AB0EE007AE4EE875AB5EE007A65EE89
:1085E800875A07EE102AB8EEC75A9FED307ADFEDAA
:1085F800306AB3F91620E5EE075AF8EEE77A9FEDF0
:108608002D7A76EEE77ADFED2C6AE5EEC77A05EE8D
:10861800902AB0EE677ADFED297AB3F91420B3F91E
:10862800123067EE277A07EE102AC7EE847AF8EE42
:10863800E55AB8EEC77A65EEA75A27EE877A65EE4F
:10864800A75A27EE237AA5EEA67AF0EE476A07EE38
:10865800103AB8EEC77A36EE877ADFED196AE7EE98
:10866800267A01E0DFED177A18B1FDEEE77AC0ED62
:10867800007A31B1FDEEC67A642217EE903A534380
:108688000B6030BD20030020741E0020000000375E
:1086980000007AC700000038000000390000803A66
:1086A800000080380000A045000000360000804728
:1086B8000000804900008039000000300050C345A8
:1086C8000000803D00000000704770476C4B6D4A09
:1086D8002DE9F04F5E8994684FEA062AB4EB0A0A3E
:1086E8009C884FEA04481C894FF000054FF0000BA6
:1086F80065EB0B0BA4FB0A6704FB0B77F40944EA50
:10870800476418EB04065C884FF000094FEAE71548
:108718004FEAC438DC8849EB050787B0CDE9046720
:10872800A4FB0A6704FB0B77340A44EA076418EBD6
:1087380004064FEA27259C894FF0000949EB0507F5
:10874800CDE90067AAFB046704FB0B77F40D44EA44
:10875800472414F5FA664FEAE75545F10007B6F5E0
:10876800FA6F77F10003CDE90267964667DAA4FB52
:10877800046704FB05F34FF0050C07EB4307DDE93D
:108788000489A6FB0C230CFB07335F104FEA320663
:10879800B8EB06084FEA920669EB070946EA8376C2
:1087A8009F10DDE90023921B63EB0703DDE90267F5
:1087B800CDE90023344A4FF0FF33964277EB0303A9
:1087C800CDE9048928DA40F6AC52A4184FF000032A
:1087D8005D4104FB05F3A4FB044505EB43056FF07D
:1087E8000602664202FB0566A4FB0223334418EB2B
:1087F800020649EB0307CDE904670B26A4FB062311
:1088080006FB0533DDE900455B104FEA3202A41A86
:1088180065EB0305CDE900450AFB0BF3DDE90245ED
:10882800AAFB0AAB0BEB430B4FEADA7242EA4B02A4
:10883800A41A4FEAEB7365EB0305CDE90245DEF8B0
:108848000C40009B019DA4FB032304FB05334FEA66
:1088580052584FEA635948EAC328DDE90423B8EBC4
:10886800020269EB03039946D30B43EA494300B17B
:10887800036009B1029B0B6007B0BDE8F08F00BF31
:108888000E030020741E002024FAFFFF054B1A7CFB
:1088980002F0FF0122B10122027000221A7470470F
:1088A80001707047741E002007EE900AF8EEE77A10
:1088B800DFED0C6A9FED0C0AF5EEC07AF1EE10FAC6
:1088C800D4BFB1EE677AC7EEA67A08B5D8BFC7EEAF
:1088D800267A27EE800A03F051FB044B83ED000A49
:1088E80008BD00BF8096184B35FA8E3CAC000020BE
:1088F8007620F4213122FCF79DBB77204821012204
:10890800FCF798BB772058210122FCF793BB1FB5D1
:10891800044602210C2001220DF10703FCF70EFB8F
:1089280008B900203BE09DF80730DB07F9D50321A3
:10893800062202AB0C20FCF701FB0C2009210122C6
:108948000DF10703FCF7FAFA0028EAD09DF8073082
:1089580013F00C0FE5D19DF809209DF8083043EA83
:108968000223C3EB83339B009DF80B2023809DF8E3
:108978000A3043EA0223C3EB83339B009DF80D20A2
:1089880063809DF80C3043EA0223C3EB83339B00DA
:10899800A3800C200A210122FCF74CFB012004B023
:1089A80010BD07B5F7216B4606227620FCF7C6FAFC
:1089B8009DF800309DF801100B4A1B0343EA011390
:1089C8009DF8021043EA111353609DF803309DF897
:1089D80004101B0343EA01139DF8051043EA111321
:1089E800136003B05DF804FB741E002007B5002176
:1089F80001AB03227720FCF7A1FA9DF805309DF81A
:108A080004001B0243EA00439DF80600184303B024
:108A18005DF804FB08B5FFF7E9FF014BD86008BD16
:108A2800741E002008B5FFF7E1FF014B986008BDF0
:108A3800741E002013B506220446432168206B46A5
:108A4800FCF77CFAA8B19DF800209DF8013043EAB4
:108A5800022323809DF802209DF8033043EA022375
:108A680063809DF804209DF8053043EA0223A38023
:108A7800012002B010BD13B5062204463B21682030
:108A88006B46FCF75BFAA8B19DF800209DF8013011
:108A980043EA022323809DF802209DF8033043EA2D
:108AA800022363809DF804209DF8053043EA0223E1
:108AB800A380012002B010BD07B50A2100220C20B6
:108AC800FCF7B8FA1420FFF7CEF90A210F220C2080
:108AD800FCF7B0FA0A20FFF7C6F901AB1021032210
:108AE8000C20FCF72BFA0A20FFF7BDF90A21002217
:108AF8000C20FCF79FFA0A20FFF7B5F90DF10303E4
:108B0800022101220C20FCF719FA0DF103030921B7
:108B180001220C20FCF712FA0A2101220C20FCF792
:108B280089FA03B05DF804FB08B507F051F86B212A
:108B380080226820FCF77EFA6420FFF794F96B2105
:108B480003226820FCF776FA0F4B19211A7868205F
:108B5800FCF770FA0F20FFF786F90C4B1A211A78E8
:108B68006820FCF767FA1B2118226820FCF762FAD4
:108B78001C2110226820FCF75DFA682037210022AA
:108B8800BDE80840FCF756BA3C030020000000206E
:108B980008B507F01DF8074B1B7813B1012B03D05C
:108BA80008BD4FF4006201E04FF48052024B1A8076
:108BB80008BD00BF0C03002016000020F8B59E4B2E
:108BC8001B680546187818B1012800F06B81E6E2A9
:108BD800242D9A4C0CD006D80A2D00F0DC800D2DDF
:108BE80000F0D98048E12A2D06D02C2D04D043E18D
:108BF8006074A074E07451E1914BA17C677C8F4A4A
:108C0800002058542FBB19781775472921D1597856
:108C180050291ED19978472907D1D978472904D1F5
:108C28001979412901D1012111759978844A52296C
:108C380003D1D1784D2900F0B4829978804A472928
:108C480007D1D178532904D11279562A04BF0322B7
:108C58002275227D794E022A3AD0032A4DD0012A64
:108C680040F08780BA1E072A00F28380DFE802F00E
:108C780004080F131A25812B08F0A4F9A06178E0E5
:108C88001B78532B75D1A3695B42A36171E008F08F
:108C980099F9E0616DE01B78572B6AD1E3695B4273
:108CA800E36166E01B78302B664B1A788CBF42F084
:108CB800020222F002021A705BE0002008F0E2F9DA
:108CC80084F8200055E0002008F0DCF9608450E0CA
:108CD800072F06D0082F4CD1012008F0D3F9F084D3
:108CE80047E0012008F0CEF941F2184358434FF409
:108CF8007A73B0FBF3F0B0843BE0022F07D0032F68
:108D08000BD1002008F0BEF94F4B187031E000205D
:108D180008F0B8F986F828002BE02AD93A1F9210F3
:108D280096F828300132D2B2013B02EB8303DBB262
:108D3800102B1ED8F91EC2F1010201EB8202D2B239
:108D4800012A0BD0042A11D100205E1E08F09AF9DE
:108D58003E4B98553E4B00229A5507E05E1E3D4A11
:108D68000020935508F08EF93B4B9855E36A013380
:108D7800E362324B2A2D18BFDA7C07F101074FF066
:108D880000000CBF012255406774A0740CBF83F823
:108D98003020DD7482E094F83000002847D02F4B53
:108DA80013F8012D2E495A708B42F9D1244A234DCC
:108DB80013785278402B85BF373B1B011B01DBB270
:108DC80098BF03F0F003402A8CBF373A303AD2B24A
:108DD8001344E27CDBB29A4226D121230B70287D12
:108DE8006B6B1F4A013301286B630AD002281DD11F
:108DF800722313701B4BAA8C1A801B4BEA8C1A80A7
:108E080014E0672313700F4B1B789F070FD5174B80
:108E1800AA691A60EA695A60154B95F820201A70F9
:108E2800144B6A8C1A8002E03F230B700020002349
:108E380084F8303032E000BF00080020741E0020A3
:108E480070290020EC1A002098120020C912002076
:108E5800B912002099120020A91200205C030020FA
:108E680048030020EE1A002080120020F41A002087
:108E7800F21A0020F01A0020A37C94F830000E2B80
:108E88009FBFAC4A591C9174AB4A98BFD554A94AA4
:108E980018B9D37C5D40D57400E00020003018BFBD
:108EA8000120F8BDA34B93F838100022082900F2DE
:108EB8007681DFE801F0050C101A2B3B607E8B00F1
:108EC800B52D40F06C8183F83920012250E0622DE5
:108ED80008BF02224CE0032283F8382083F83A5076
:108EE80083F83B5083F83C5059E1042283F838203A
:108EF80093F83B2093F83C1083F83D502A44D2B2B3
:108F080083F83B200A4483F83C2048E1052283F893
:108F1800382093F83B2093F83C10DD872A44D2B2DE
:108F280083F83B200A4483F83C2038E1062283F882
:108F3800382093F83B2093F83C102A44D2B283F8A7
:108F48003B200A4483F83C20DA8F02EB0525ADB2BA
:108F5800B5F5AC7F88BF774ADD8784BF012182F8E9
:108F680039100022A3F84020002D40F01881072274
:108F780083F8382013E193F83B2093F83C102A44F7
:108F8800D2B283F83B200A4483F83C20B3F840204F
:108F9800B2F5AC7F3CBF6749891802F1010238BFBE
:108FA80081F84450D98F92B29142A3F84020DED97B
:108FB800F5E0082283F8382093F83B30AB4200F004
:108FC800EE805C4B012283F839200FE05B4C83F87C
:108FD800382014F8012D6270594A9442F9D193F857
:108FE8003C10544AA94206D03F232370554A53687F
:108FF80001335360D3E0516B92F83900013151636A
:1090080010B13E232370CAE02121217092F83D104F
:10901800062941D004D8022907D0032923D0F8BD56
:10902800122959D0302967D0F8BD502121704649FE
:10903800946C4C60D46C0C60516D4FF47A7491FB55
:10904800F4F1424C218092F89C11414A19B11178EF
:1090580041F0020102E0117821F0020111700122B1
:1090680083F89D218DE05321217092F84910CE0795
:1090780005D592F84820D51E6A426A4100E00246AA
:1090880002F0010183F89C11002A7AD130490A784C
:1090980022F002020A7074E04F21217092F84F10FA
:1090A800CC0705D592F84E20D11E4A424A4100E02D
:1090B800024602F0010183F89C1122B924490A787A
:1090C80022F002020A70234A93F873101170224AA0
:1090D800B3F87010118054E0562121701F49946D27
:1090E8000C8042F21074D16D91FBF4F11C4C21807C
:1090F800012182F89E1144E04921217092F848101C
:10910800184A102988BF10211170174914780022B5
:10911800A24233D2154D0E7A5655154D4E7A5655F4
:10912800144DCE7A5655144D11F80C6F5655013220
:10913800EEE700BF741E0020702900205C030020A9
:1091480048030020E0070020F41A0020F01A00204D
:10915800EC1A0020F21A00200A010020EE1A002062
:109168008012002098120020B81E002099120020BA
:10917800A9120020B9120020C9120020DA6A0132AF
:10918800DA6293F89D310B4A93B192F89E317BB124
:10919800002182F89D1182F89E111846F8BD002022
:1091A800F8BD1279432A7FF448AD0222227544E5BE
:1091B800F8BD00BF741E00200449054B09681870EB
:1091C80000225A6199611A77704700BF6829002008
:1091D800E007002010B5121A07EE902A5B1A2DED51
:1091E800028BF8EEE78A07EE903A184B059CB8EE2A
:1091F800E78AD3ED007A28EE278A28EE080AA8EE37
:10920800A80A0CF0ADFDDFED127A049B20EE270AC8
:10921800F0EE480ABCEEC00A83ED000AB1EE680A17
:109228000CF0FAFBDFED0B7A9FED0B7AE0EE077A94
:10923800BDEC028BFDEEE77A17EE903A002BBCBF2F
:1092480003F50C43A033236010BD00BFAC00002021
:109258002C7D8E3F00A00C46A00CB34544F2506311
:10926800984203DDA0F50C40A0387047034B9842A4
:10927800BCBF00F50C40A030704700BFB0B9FFFF7D
:1092880073B51A4C036823600B686360184D006857
:10929800184EFFF709FB184B009395E8030094E874
:1092A8000C000196FFF796FF144B32681A60686845
:1092B800636813491B1A07EE903A124B286893ED1E
:1092C800007A23681B1A0B600F4BF8EEE77A1A60D6
:1092D8000E4B67EE877A1B68FDEEE77ADA880C4B4F
:1092E800C1ED017A1A8002B070BD00BF402800208D
:1092F800F41A00204C280020482800208828002044
:1093080050280020AC0000208028002048100020B1
:109318007C2800204279DFED2A5A2A4B9FED2A5AF1
:1093280007EE902AF8EE677AC27BC7EEA57AB2EE0E
:10933800047AC3ED007A07EE902AF8EE677A234A9A
:10934800DA60C7EEA57AC3ED017A8179204B07EE82
:10935800901AF8EE677A017CDA60C7EE877AC3ED77
:10936800007A07EE901A817E06EE101AF8EE677AF8
:10937800B8EE466AC7EEA57A86EE056AC3ED017AAD
:1093880083ED026AC179134B06EE901A417CDA60CC
:10939800F8EE666AC6EE876A07EE101AC17EC3ED5C
:1093A800006A07EE901AB8EE477AF8EE677A87EE09
:1093B800257AC7EE857A83ED017AC3ED027A704784
:1093C8000000C8425828002000007A440000FA44EF
:1093D800682800208C28002010B50C4C23789B07A7
:1093E80013D50B4B1B78042B0FD90A4A0A4B10686C
:1093F80052685A601860FFF757FA084B1A88084BEA
:109408001A80237843F00103237010BDEC1A002062
:10941800F21A0020F41A002084120020F41200200E
:109428009C2800201C4B1B681B0307B530D51B4A22
:109438001B4BD2ED007A1B788DF80030B2EE047A1F
:1094480067EE877A174B9FED187A1B788DF80130F5
:10945800FCEEE77A0A2017EE903AD2ED017A8DF801
:10946800023067EE877A6946FCEEE77A17EE903AA3
:10947800D2ED027A8DF80330FCEEE77A17EE903AD7
:109488008DF80430094B1B788DF8053001F034FE57
:1094980003B05DF804FB00BF4429002058290020D0
:1094A800362900205429002000007A443A29002057
:1094B800054A137883F001031370044A00231360EC
:1094C800034A1360AEE700BF3A2900205029002064
:1094D8004C29002007B52320FEF7C5FC682075211C
:1094E80001220DF10703FBF729FD28B19DF80700BC
:1094F800A0F168035842584103B05DF804FB00BF6F
:10950800704708B51F4A18B9536802221A8208BD65
:109518000020516810800B7813F07F030DD14B7A2F
:10952800990644BF0221117013F0400F137814BF3D
:1095380043F0010323F0010315E0012B1FD0022B98
:109548001ED14B7913F0800F03F00F034FEA83030A
:1095580003F1804303F5B8431B6806D003F03003DA
:10956800102B07D10123137004E003F44053B3F523
:10957800805FF6E793681B699847024808BD104664
:1095880008BD00BF1820002010B5064C18B9636844
:1095980001221A8210BDA3689B68984760680C3046
:1095A80010BD00BF1820002010B5064C18B963681C
:1095B80001221A8210BDA3681B68984760680A30A8
:1095C80010BD00BF18200020084BDA68D10709D465
:1095D800DA68D20608D4DB6813F0040F14BF03203E
:1095E8000420704701207047022070470020024085
:1095F80010B50446B0F9000007F0DDFAB4F902002E
:1096080007F0D9FAB4F90400BDE8104007F0D3BA5E
:1096180010B50446006807F0CEFA606807F0CBFA88
:10962800A068BDE8104007F0C6BA2DE9F74F012041
:1096380001F092FB002488B3012C2FD8194E4FF06B
:109648004C0909FB04FA06EB0A0808F15407BD782F
:1096580015B10134E4B2EEE790F9003090F804E077
:109668001846114B03228DE8240001212A4653F89D
:109678002E3001F04DF9834660B106F10C005044DC
:1096880029464A460BF0B7FE01231C44C8F80CB023
:10969800BB70E4B2012001F043FBCCE703B0BDE8A6
:1096A800F08F00BF182000202C7E010810B5184C40
:1096B800002120461A220BF09EFEA4F5F870142310
:1096C80080F8F23105230022042180F8F63180F871
:1096D800F83180F8FE3180F8003280F8063280F8E0
:1096E80008325223012480F8F71180F8F92180F814
:1096F800FF1180F8012280F8071280F8092280F80B
:10970800F03180F8FA2180F80242A0F8F44110BD47
:10971800F414002010B5FFF757FF4FF43024012848
:1097280006D11CB1FFF750FF013CF8E7052010BD3A
:10973800002C08BF052010BD70B50646441E14F85D
:10974800011F89B1094D28460BF08BFE0028F6D081
:1097580005F1080398423FBF054B401BC018A31BE7
:1097680038BF80F88631EAE770BD00BF4A9D01081E
:1097780004130020031EB8BF2D2210B5B8BF5842ED
:109788000C46B8BF01F8012B0A2202F065FA002343
:109798000370204610BD07B51C4B03F1A802C3F89F
:1097A800A4201B4A92F88E215AB1012A14D1032110
:1097B80083F8AA10072183F8AC2083F8AB100C2299
:1097C80008E0022183F8AA10032183F8AC2083F86B
:1097D800AB10072283F8A8200E4B0F4A1A604020CE
:1097E80001F0BAFA70B10122002390F9000040217B
:1097F8008DE80C00094A4FF4E13301F089F8003094
:1098080018BF012003B05DF804FB00BF182000203A
:10981800041300201C00002041150108D51601087A
:109828000120002106F066BBF0B51C4A92F8AD3065
:10983800D2F8B05092F8B47092F8C06092F8CCE0C8
:10984800022B0ED805EBC304591CA31CC9B206D0C1
:109858002346A48814F0010F01D0204205D10B46FD
:10986800EEE782F8AD300020F0BD93F902307CB20B
:109878009C4201D1002307E074B29C420CD04FFAFD
:109888008EF49C42EBD1022382F8AD100C2101FB2F
:109898000322D2F8B800F0BD0123F5E71820002014
:1098A80030B5002202F1805303F5B8539B0042F40F
:1098B80000441D6840F60F7144F0800429400132CD
:1098C8002143042A1960EDD1024B40F08000186052
:1098D80030BD00BF4C5C00402DE9F843324D6E6846
:1098E800328A377ABAB9042F15D130480378012B58
:1098F8000CD12F4B19682F4B89B20B445B001968A8
:109908001A603023A5F8D830027049E01023A5F872
:10991800D830072744E0B48AB369A24294BF042729
:109928000227944228BF14461FFA84F840469847F5
:109938001F4A13689BB203F1005303F540535B00C1
:1099480004F1010E1B689BB203F1005303F5405369
:109958004FEA6E0E5B000021714500F1020009D04C
:1099680010F8019C10F802CC4CEA092C23F821C00D
:109978000131F1E712680F4B92B213445B001A6889
:109988001C60338AC8EB03033382738A98443023FC
:10999800A5F8D8304FF44053A6F81280A5F8DA306D
:1099A8006B681F72BDE8F88318200020B92D0020CD
:1099B800505C0040023000200E4B0F4A1B689BB2DF
:1099C80003EBC00002443E294FEA420209D94B0981
:1099D800C80604BF03F1FF339BB29B0243F4004364
:1099E80004E04B08C90748BF01339B0211681360A4
:1099F800704700BF505C00400630002008B50B4B94
:109A0800002093F83010FFF7D7FF094B5A68107AF7
:109A1800082801BF4FF48052A3F8DA201022A3F8D7
:109A2800D820A0F109035842584108BD1C00002065
:109A38001820002038B5444D6A68107810F07F006F
:109A480004D1537A23F02003537238BD022879D108
:109A58005388002B77D11379002B74D1537923F0D5
:109A68008000840004F1804101F5B84113F0800FB3
:109A7800096814BF01F0300101F44051032861D88E
:109A880000295FD0927A002A5CD004F1804404F562
:109A9800B8441906226825D502F03002102A4CD1A4
:109AA80003F07F039B0003F1804303F5B8431A6872
:109AB800510641BF196840F60F720A4042F400424D
:109AC80044BF42F0C0021A601A6822F4E04222F051
:109AD800400292B282F0300242F4004242F0800228
:109AE8001A602AE002F44052B2F5805F25D128B905
:109AF800164B93F83010FFF75FFF11E09B0003F15E
:109B0800804303F5B8431A68520441BF196840F608
:109B18000F720A4042F4404244BF42F080021A6089
:109B2800236823F4804323F070039BB283F44053EB
:109B380043F4004343F080032360AB685B699847B4
:109B4800002038BD022038BD182000201C0000204D
:109B58000023036043608360838103614361836101
:109B6800C36103624362836270478A68036810B501
:109B78000C6A14430A6914434A6914438A691443F2
:109B8800CA6914434A6A14438A6A23F4FF4323F0D8
:109B980070032243134303608B8943600B6883601F
:109BA8004B68C36010BD02684FF6FE731340036034
:109BB8000023036043608360C360294B984201D14E
:109BC800284A27E0284B984201D1264A2AE0274B09
:109BD800984201D1234A2DE0254B984201D1214AD0
:109BE80030E0244B984201D11E4A33E0224B984280
:109BF80004D11C4A536843F470032EE01F4B98426B
:109C080004D1184A536843F0706326E01C4B98420D
:109C180004D11C4A536843F00F031EE01A4B9842C4
:109C280004D1184A536843F0F00316E0174B9842E2
:109C380004D1144A536843F470630EE0144B9842FD
:109C480004D1104A536843F4704306E0114B98421C
:109C580004D10C4A536843F470235360704700BF23
:109C680008000240000002401C0002403000024090
:109C780044000240580002406C000240800002404C
:109C880008040240000402401C0402403004024060
:109C98004404024058040240036A23F001030362AB
:109CA800036A70B5446882690D6822F4803222F034
:109CB800730215438A8923F0020313438A881343E6
:109CC800134A90420FD002F5006290420BD002F581
:109CD8004062904207D002F58062904203D002F5BC
:109CE800806290420DD1CA89CE8823F008031343BD
:109CF8000A8A24F4407414434A8A23F00403334341
:109D080014438A68446085614263036270BD00BF82
:109D1800002C01409D4A536803F00C03042B2DE9E5
:109D2800F04105D0082B06D099490160B3B916E077
:109D3800974B036012E053685468C3F38343991C3C
:109D4800E30349BFD36A934B914C03F00F0344BF1D
:109D58000133B4FBF3F34B43036000E00023516885
:109D68008D4FC1F30311394491F834500168EDB2B5
:109D780021FA05F444605668C6F302263E4496F874
:109D8800346024FA06FEC0F808E05668C6F3C22616
:109D98003E4496F83460F6B2F440C460D2F82C80A1
:109DA800C8F3041808F00F0C07EB4C0C18F0100F50
:109DB800BCF844C01FFA8CFC07D0BCF1000F04D0DB
:109DC800B3FBFCFCC0F810C000E00161D2F82CC065
:109DD800CCF3442C0CF00F0807EB48071CF0100FCD
:109DE800B7F84470BFB204D01FB1B3FBF7F74761AF
:109DF80000E04161176BFF065ABF654F87618161BB
:109E0800176BBF065ABF624FC761C161176B7F06E8
:109E18005ABF5F4F07620162176BFF0506D599426B
:109E280004D1AE4202D14F00476200E04462176B92
:109E3800FF0406D5994204D1AE4202D14F00876291
:109E480000E08462176BBF0506D5994204D1AE4283
:109E580002D14F00C76200E0C462176B7F0506D5C8
:109E6800994204D1AE4202D14F00476400E04464F5
:109E7800176B3F0506D5994204D1AE4202D14F0077
:109E8800876400E08464176BBF0406D5994204D147
:109E9800AE4202D14B00C36400E08464156B3B4BB7
:109EA800AD0701D1046315E01C6B04F00304012C19
:109EB80001D101630EE01C6B04F00304022C02D1F3
:109EC8004FF4004305E01B6B03F00303032B01D1A0
:109ED8002F4B0363146B2D4B14F4403F02D1C0F891
:109EE80034E018E01C6B04F44034B4F5803F01D131
:109EF800416310E01C6B04F44034B4F5003F02D118
:109F08004FF4004306E01B6B03F44033B3F5403FC6
:109F180001D11F4B4363146B1C4B14F4402F02D127
:109F2800C0F838E018E01C6B04F44024B4F5802F26
:109F380001D1816310E01C6B04F44024B4F5002FB8
:109F480002D14FF4004306E01B6B03F44023B3F542
:109F5800402F01D10E4B8363146B0C4B14F4401F3C
:109F680002D1C0F83CE021E01C6B04F44014B4F5C5
:109F7800801F01D1C16319E01C6B04F44014B4F5CF
:109F8800001F0BD14FF400430FE000BF0010024048
:109F980000127A0000093D001C0000201B6B03F42E
:109FA8004013B3F5401F01D1134BC363126B134B1E
:109FB80012F4400F03D1C0F840E0BDE8F0811A6BFD
:109FC80002F44002B2F5800F02D10164BDE8F081CD
:109FD8001A6B02F44002B2F5000F02D14FF40043AD
:109FE80006E01B6B03F44003B3F5400F01D1024BAD
:109FF8000364BDE8F08100BF00127A00001002403F
:10A00800F0B500230E681C460125A54005EA060E9A
:10A01800AE452BD10F797A1E012A15D885680322FF
:10A028009A4025EA020282604D7982689D40154374
:10A038008560828892B222EA0E0282808A798588B7
:10A04800A2402A4392B28280032205689A40D243F2
:10A058001540056005689F402F430760C768174093
:10A06800CA7902FA03F547EA0502C2600134102CE6
:10A0780003F10203C8D1F0BD38B52DED048B4A4C6D
:10A088000368C4F8DC308388A4F8E030013A0D4650
:10A09800072A42D8DFE802F0040A101822292F35CF
:10A0A800B4F8DC300B80B4F8DE3013E0B4F8DE30FE
:10A0B8000B80B4F8DC3005E0B4F8DC305B420B8090
:10A0C800B4F8DE305B4205E0B4F8DE305B420B806A
:10A0D800B4F8DC306B80B4F8E0301DE0B4F8DC3064
:10A0E8005B420B80B4F8DE3012E0B4F8DE300B804F
:10A0F800B4F8DC300CE0B4F8DC300B80B4F8DE30B7
:10A1080005E0B4F8DE305B420B80B4F8DC305B422B
:10A118006B80B4F8E0305B42AB80244B93F864303A
:10A12800002B3ED1B5F9003094ED3C0AD4ED397AD4
:10A1380009EE103AB5F9023008EE103AB8EEC88ABE
:10A14800B5F90430B8EEC99A28EE000A08EE903A3C
:10A15800A7EE890AF8EEE88AD4ED3F7AA7EEA80AB6
:10A168000BF058FB94ED3D0AD4ED3A7A288028EE9E
:10A17800000AA7EE890AD4ED407AA7EEA80A0BF0E8
:10A1880049FB94ED3E0AD4ED3B7A688028EE000A3C
:10A19800A7EE890AD4ED417AA7EEA80A0BF03AFB9C
:10A1A800A880BDEC048B38BD182000201C000020BE
:10A1B80008B50A4890F8093100EB43030A22B3F8BE
:10A1C800181189B2A0F8201100F59470FDF721FF4D
:10A1D80080B207F045FB024B188008BD182000200C
:10A1E800D81A0020F8B504460E4617460025204622
:10A1F80020210BF036F90446D0B1013420460BF08B
:10A2080095F9B0F5617F05DB40F634039842A8BFA5
:10A21800184601E04FF46170A0F56170192390FBB6
:10A22800F3F00DB9307000E070703B7801333B708B
:10A238000DB90125DBE72046F8BD30B505460C46CB
:10A248001346294622460248BDE8304001F005BEC3
:10A25800309E01087FB504780646E4B9354B1B6883
:10A2680003EB8403192193F87B0093F87C6093F83F
:10A27800792093F87A304FF4617511FB005011FB87
:10A288000651009001912C482146013401F0E5FD6A
:10A29800142CE3D14BE00BF049F91328054641DCB7
:10A2A800244B701C1C68202100238DF80F300BF004
:10A2B800D8F81E35064670B1013630460BF036F92F
:10A2C8001A289FBF04EB850358709DF80F3001339F
:10A2D80098BF8DF80F30304620210BF0C2F80646A3
:10A2E80070B1013630460BF021F90D289FBF04EB01
:10A2F800850398709DF80F30013398BF8DF80F30A3
:10A3080004EB85043046E11C0DF10F02FFF76AFFEC
:10A318009DF80F30042B0AD0601C002104220BF09A
:10A328006AF804E0054800211322FFF786FF04B00D
:10A3380070BD00BF581200204F9E0108649E01089E
:10A34800014805F07DBE00BF6A9E0108F8B5047893
:10A35800064674B9304DB5F8C221B5F8C4312F4856
:10A368002146013401F079FD042C05F10405F2D1F0
:10A37800F8BD2B490BF048F8A8B9274B4FF47A7170
:10A388004FF4FA62A3F8C211A3F8C421A3F8C611C6
:10A39800A3F8C821A3F8CA11A3F8CC21A3F8CE11B9
:10A3A800A3F8D021F8BD30460BF0C0F803280546C5
:10A3B8002BD8304620210BF054F8044630B1013434
:10A3C80020460BF0B3F80126074600E00646204673
:10A3D80020210BF046F810B9BDE8F840B0E701308D
:10A3E8000BF0A4F8012EF7D1A7F2EE2240F2DC53CD
:10A3F8009A42F1D8A0F2EE229A42EDD8064B6E3579
:10A4080003EB85035F819881F8BD0648002103228C
:10A41800BDE8F84011E700BF04130020789E01084A
:10A428008B9E0108B1A901082DE9FF410478054672
:10A43800002C39D17348744D05F002FED5ED047A2D
:10A44800F5EE407AF1EE10FA00F0D88021466F4818
:10A4580001F003FD95ED040A684601F093FB0146FF
:10A468006B4801F0FAFC95ED050A684601F08AFB95
:10A478000146674801F0F1FC95ED060A684601F0CF
:10A4880081FB0146624801F0E8FC95ED070A684641
:10A4980001F078FB013401465E4801F0DEFC0C2C2B
:10A4A80005F11005CAD1A9E05B4905220AF0F0FFC1
:10A4B80040B9554B03F1C002002143F8101F9342E5
:10A4C800FAD19BE02846554904220AF0E1FF0446E8
:10A4D8002846002C40D120210AF0C3FF002800F0B4
:10A4E8008D80451C28460AF0CAFF07464C4B53F896
:10A4F80024601EB94B4805F0A3FD7FE0284631468D
:10A50800FAB20AF0C5FF01340028EFD13E4B03F13F
:10A51800C0029E46002143F8101F9342FAD1424BD5
:10A5280003EBC4029846D2F804C0BCF1000F04D172
:10A5380031463E4801F091FC57E0002718F83430C6
:10A548009F42F5DA3B010EEB030563440FCB103550
:10A5580085E80F000137F1E70AF0E8FF0B28064607
:10A5680047DC284620210AF07CFF054650B101351A
:10A57800284601F07DFA244B03EB061383ED040A09
:10A58800012400E00446284620210AF06AFF054617
:10A5980048B10135284601F06BFA1B4B03EB061353
:10A5A80083ED050A0134284620210AF05AFF0546A2
:10A5B80048B10135284601F05BFA134B03EB06134B
:10A5C80083ED060A0134284620210AF04AFF10B913
:10A5D800FFF7B6FE12E0013001F04AFA0A4B032CED
:10A5E80003EB061686ED070AF2D11148FFF71CFFA8
:10A5F80004E0104801210C22FFF71FFE04B0BDE85B
:10A60800F08100BF919E010804130020AC9E010850
:10A61800B29E0108E0A601088B9E0108B69E0108BB
:10A62800F0950108BB9E0108609D0108CA9E0108BB
:10A638000B9C0108649E0108F0B5047887B00646B3
:10A648001CBB514B1968062303FB0411192091F810
:10A65800CA5091F8CB7091F8CE2091F8C9304FF4D8
:10A66800617610FB056510FB07600095019091F875
:10A67800CC000290C83145484979039121460134FC
:10A6880001F0EBFB0C2CDCD17CE00AF04FFF0B282F
:10A69800044672DC3C4B701C1D68202100238DF899
:10A6A80017300AF0DEFE064680B1013630460AF061
:10A6B8003DFF03289FBF062303FB045383F8CE0006
:10A6C8009DF817309CBF01338DF817303046202194
:10A6D8000AF0C7FE074680B1013738460AF026FF60
:10A6E8000D289FBF062303FB045383F8C9009DF878
:10A6F80017309CBF01338DF8173006266643A91919
:10A708003846CA310DF11702FFF76CFD20210AF017
:10A71800A8FE074670B1013738460AF007FF14282B
:10A728009FBF9DF817307619013386F8CC0098BF83
:10A738008DF81730384620210AF093FE78B10130A1
:10A748000AF0F4FE0D289FBF062303FB045383F889
:10A75800CD009DF817309CBF01338DF817309DF858
:10A768001730062B0ED0062202FB04500021C930F8
:10A778000AF041FEFFF7E4FD04E0054800210B2242
:10A78800FFF75BFD07B0F0BD58120020D69E010808
:10A79800649E01082DE9F347047806464CB9204623
:10A7A80001A9FEF7E7FF0134FFF7F4FF122CF6D1F9
:10A7B8007BE00AF0BBFEC5B2112D71D83C4C05F107
:10A7C800CC0704EB4703701C202193F80680394E10
:10A7D8000AF047FE034630B9A8F10202D2F1000898
:10A7E80048EB020845E000F1010A597830460AF0C2
:10A7F80038FE60B1032D8CBF03230023801B334434
:10A8080053FA80F090F80490B9F1030F02D1FFF7E2
:10A8180097FD4AE0A9F10203D3F1000850464FF032
:10A82800200148EB03080AF01CFED8B1B8F1000F6C
:10A83800EDD001300AF07AFE40F2ED2380B2984262
:10A8480005DD40F6CA039842A8BF184601E040F269
:10A85800EE2004EB4703A0F2EE20192290FBF2F061
:10A86800D87102E0B8F1000FD1D104EB470383F8A7
:10A87800069004EB4704A379F25CB8F1000F0AD004
:10A88800E3790D48294640F2EE24192505FB0343D8
:10A8980001F0E3FA09E02946084801F0DEFA04E08D
:10A8A800074800211122FFF7C8FC02B0BDE8F08775
:10A8B80004130020507E0108F69E0108089F010835
:10A8C800B1A9010810B504462046FDF793FB18B955
:10A8D8000A20FDF7C8FAF7E710BD0C4B5A68824208
:10A8E8001A4607D01B69834206D0D36983420BD12D
:10A8F800022302E0002300E001230021C1620C20B2
:10A9080000FB032319725960704700BFCC20002058
:10A918002DE9F04F06468A4890F9004087B0B442C6
:10A9280088469DF8445011461A469DF8403009D093
:10A9380090F90C40B44207D090F91840B44209D1BC
:10A94800022702E0002700E001270C2404FB07008F
:10A95800047A0CB10020EFE0012E00F0DC80142E08
:10A9680005D0002E40F0E78000957648D5E0DFF866
:10A9780014A2DAF8183043F00103CAF81830DAF8EC
:10A9880014304FF0904543F40033CAF814304FF0B8
:10A99800010903224FF4805B04A94FF090408DF821
:10A9A80015200392CDF810B08DF814908DF81690FC
:10A9B8008DF81740FFF724FBA5F828B0C820FDF74D
:10A9C80052FAC5F818B0DAF81430039A43F4003391
:10A9D800CAF8143028464FF4C0534FF0020B04A9AC
:10A9E80004938DF815208DF814B08DF816408DF865
:10A9F8001740FFF705FB6B6A23F470436B626B6AC1
:10AA080043F460436B626B6A23F470236B626B6A76
:10AA180043F460236B624C4B4C4D4FF480221A6018
:10AA280002F18042A2F53F3212232B63082385F8F6
:10AA38003530136885F8369023F480231360536803
:10AA480023F48023536095F8343003F1804303F5F1
:10AA580082331A6842F480221A602A6B3C4B22F037
:10AA68001F0002F01F02C15809FA02F221EA02028D
:10AA7800C2502A6B374922F01F0002F01F0250F81B
:10AA880001E009FA02F22EEA020242502A6B22F091
:10AA98001F0102F01F02C85809FA02F20243CA5005
:10AAA8002D4B2E4A1C60DAF81C3043F40003CAF818
:10AAB8001C302B4B04A8DA608DF810608DF811B0AB
:10AAC8008DF812408DF8139006F0A4F82A238DF81B
:10AAD80010309DF813308DF811908DF812401BB18D
:10AAE80004A806F097F804E01E4B4FF48062C3F800
:10AAF80084201D4B1D4C1C60022385F840301C4AE5
:10AB08001C4B1D496B6511601B6898471B4B2B60DC
:10AB1800A4F1380006E01A48009502F09BFE0028D0
:10AB28003FF418AF064B06710C2202FB073787F873
:10AB38000880786000E0204607B0BDE8F08F00BFCD
:10AB4800CC2000200038014014040140C821002016
:10AB5800080401400C040140D80042420005FA05EF
:10AB680000ED00E000E100E01C20002000220020B1
:10AB78002020002020000020840000205C7E0108A6
:10AB880000440040001002400C4B1B6893F902205F
:10AB9800824209D093F90A20824207D093F9122001
:10ABA800824208D1022002E0002000E0012003EBED
:10ABB800C000023070470020704700BFC820002046
:10ABC800F0B5027887B0AAB94C4C04F118064C4B82
:10ABD80094F9F21193F900208A4273D093F90C206A
:10ABE8008A426FD093F918308B426BD00834B44244
:10ABF800EDD181E0002204920592451C0AF096FCF2
:10AC0800C4B260B2FFF7C0FF074618B18DF8104014
:10AC1800012400E00446284620210AF022FC0546CB
:10AC280038B1013528460AF081FC0134ADF812002C
:10AC3800E4B20026284620210AF013FCB0B3451CD4
:10AC480028460AF073FC00222E4951F8223083422C
:10AC58005FFA82FE04D00132082AF5D1002300E011
:10AC6800734651F82320824220D1022E0FD0032EA2
:10AC780012D05A1E012ED2B204D0042A13D88DF84D
:10AC880014300EE0042A0ED88DF8153009E0052B93
:10AC980009D88DF8173004E09A1E052A03D88DF8D4
:10ACA80016300134E4B20136042EC3D1052C04D881
:10ACB80007B0BDE8F040FFF743BB04AB03CB3860F7
:10ACC800796019E094F8F7010E4B94F8F65153F8AF
:10ACD8002000B4F8F421009094F8F90153F820000A
:10ACE800019094F8F80153F82000029053F82530A9
:10ACF800054801F0B2F879E707B0F0BD0413002069
:10AD0800CC2000202C7E0108179F010838B1438809
:10AD180011EA030003D08B420CBF012002207047C8
:10AD280030B50B4B0B491C6891F85820022A0BD8F8
:10AD3800134604EBC303551CEAB29D882842F5D09C
:10AD480081F85820981C30BD81F85820002030BD6B
:10AD5800C8200020C8210020024B002283F8582078
:10AD6800DEE700BFC82100202DE9F047877890F87A
:10AD780003C0214DBBB2C7F1640E03EB83065C42EE
:10AD8800C3F178005FFA8EFE7600CCF16408A4B2B5
:10AD980080B2A3B20FFA83F9B9F1000F05DC002BDA
:10ADA80014BFBA464FF0010A00E0F24613FB03F362
:10ADB80003FB0CF21AFB0AF392FBF3F3434403FB85
:10ADC80009F30A2293FBF2F333449BB225F8023FBE
:10ADD800B1F800904A880A34C9EB020AA4B21AB240
:10ADE80002FB0AF24FF47A73844292FBF3F34B446A
:10ADF8002B80CED1BDE8F087202200202E4B2F4A91
:10AE08001B68126810B51A602D4A1168596051689C
:10AE18009268DA602B4A99601168196151689268E2
:10AE28009A61294A59611168D961516892685A62D0
:10AE3800264A196211881985518859859188D288BE
:10AE4800DA85234A99851188198651885986928806
:10AE58009A86204A1188D986518819871946928876
:10AE680021F83A2F1C4A10780022824206DA1B4C3D
:10AE780034F8124021F8024F0132F6E7184A1288D6
:10AE8800A3F86420174A1288A3F86620164A118886
:10AE9800A3F86C1051889288A3F87020134AA3F87D
:10AEA8006E1012689A66124A1288A3F87220114A24
:10AEB8005289A3F85E2010BDA82900208C2D0020FF
:10AEC800001C00200C1C0020181C0020FC12002074
:10AED8003C120020E61200204F1C00205C120020CB
:10AEE80038210020F410002042120020F012002027
:10AEF80078120020481200202DE9F8430E4B93E801
:10AF0800800305460E460024B44213DA7B1933F950
:10AF1800140008EB050333F9142009EB050333F992
:10AF280014301344022293FBF2F3C01A05F043FED7
:10AF38000134E9E7BDE8F883A829002070B5472067
:10AF480005F088FD174B1B681B0307D5164B174ADE
:10AF58005B6810681B68C01A05F01EFE144E154C7D
:10AF6800154D307805F018FE23682868C01A05F0DA
:10AF780022FE63686868C01A05F01DFE0F4B18882A
:10AF880005F00AFE0E4B188805F006FE0D4B1888D2
:10AF980005F002FE337823742B68A3606B68E360C6
:10AFA80070BD00BF142B0020A82900208C2D002084
:10AFB800F21A002094290020F41A0020F01A002028
:10AFC800EE1A0020801200207FB5264C264E274D11
:10AFD8002749284A284B20B128480088B0F5805FC7
:10AFE80031D23088ADF8040028781E4D91F8201031
:10AFF80012788DF806008DF807108DF808201B7858
:10B008008DF8093001A8294606220AF0D9F930B38B
:10B018000198BDF808302860AB80532005F01AFD70
:10B02800208805F0B9FDA07805F0B6FDE378019316
:10B038002379029301A86379039305F013FD0F4B5D
:10B0480000221A800BE03088208091F820102878A0
:10B0580012781B78A070E17022716371DDE704B08B
:10B0680070BD00BF3C220020B01B0020EC1A00205D
:10B078000C2D00206B0F0020D00F0020342B002057
:10B08800A0F17D03012B70B504460D460A4E05D884
:10B0980030687D21FCF7BAFF84F02004306821462F
:10B0A800FCF7B4FF35B12B881C4404EB142404F0DE
:10B0B800FF042C8070BD00BFA01B00200A4A138823
:10B0C80001331380094A136801331360084A13884F
:10B0D80001339BB2202B01BF00231380054A13883C
:10B0E80008BF013313807047342B00201C2B00202D
:10B0F800202B0020222B002038B53A4B1B78083B28
:10B10800012B05460C466BD8452005F0A3FC2846C4
:10B1180005F0A0FC0C2D23D004D80A2D0AD014D891
:10B1280035B138BD0E2D4BD02ED3FF2D50D038BDA4
:10B13800206849E0207805F08DFC62796378002A60
:10B1480014BF80200020184300E0207805F082FC1E
:10B15800A07805F07FFCE07805F07CFC20793BE0E6
:10B16800B4F9000005F00EFDA07805F073FCE07856
:10B1780005F070FCB4F9040005F004FDB4F906000C
:10B18800BDE8384005F0FEBC637820788BB180F0CC
:10B19800800005F05FFCA468E0B205F05BFCC4F336
:10B1A800072005F057FCC4F3074005F053FC200EB8
:10B1B80012E005F04FFC6068BDE8384005F0FBBCC4
:10B1C800206805F0E9FC6068BDE8384005F0E4BC9B
:10B1D800054805F01DFC0020BDE8384005F03ABCE4
:10B1E80038BD00BF84290020369F01082DE9F04FA3
:10B1F800B74BB84F1A888BB00193002A40F0A38050
:10B20800B7F8CA07B44E42F20103C21A504250417D
:10B21800FFF7DAFEFFF7F2FD3468492005F01AFC63
:10B22800AE4B2546186805F0B7FC55F8040B05F039
:10B23800B3FC2846FEF7ECF904F11000FEF7E8F934
:10B2480004F11C094FF01008A54D01232A6803FAE0
:10B2580008F3134203D0D9F8000005F0ACFC08F15C
:10B268000108B8F1130F09F10409EDD104F1280020
:10B27800FEF7BEF9B7F84031B4F92E00C01A05F050
:10B288008BFC2B68DB0408D5964BB4F864001B884C
:10B29800181AC0F30D0005F07FFC2B68980403D53D
:10B2A800B4F8660005F078FC2B68590503D504F15D
:10B2B8006C00FEF79DF92B681A0502D5A06E05F003
:10B2C8007AFC2B681B0403D5B4F8720005F064FC03
:10B2D80004F13000A046FEF78BF904F13600FEF7C2
:10B2E80087F9B7F8403138F93C0FC01A05F054FC1B
:10B2F80001277D4B1B789F4208DA38F9020FB4F911
:10B308003C30C01A05F057FC0137F2E72B68980566
:10B3180005D5B4F95E00A0F2DC5005F04CFC3268AB
:10B3280072487260B260121A9110714A4A43531CF3
:10B33800032293FBF2F202EB42029A1A742303FBF4
:10B3480002033360C9E16B4B6B4A1B6811688B427F
:10B3580006D00AA9002041F8203D1360FFF7CCFE73
:10B36800019B97F8CA171B8897F8CB070B44013B3A
:10B37800B3FBF0F200FB12338B4280F07981564C1C
:10B388000120FFF721FEFFF739FD50202668656888
:10B3980005F060FBA268236810681B6862680344B4
:10B3A8001068A3EB400005F006FC6A6873689B1AF6
:10B3B8000293AA68B3689B1A0393EA68F36802A821
:10B3C8009B1A0493FEF724F92A6933699B1A02939E
:10B3D8006A6973699B1A0393B369AA6902A89B1ADD
:10B3E800049305F03FFB06F11C0905F11C0B10271F
:10B3F800A0463B4801210368B9401942824606D05D
:10B40800D9F80000DBF80030C01A05F0D4FB01378A
:10B41800132F09F104090BF1040BEAD106F12600F8
:10B4280005F12601002331F9024F30F9022F121BD2
:10B4380002AC44F823200133042BF4D10322002763
:10B4480002ABBF0053F82230FFB26BB103F1080121
:10B458000F2902D847F0010706E08033FF2B94BF7D
:10B4680047F0020747F0030712F1FF32E8D23846E7
:10B4780005F0F0FA00240DF10809A34607F00302CD
:10B48800022A10D0032A17D0012A4AD1BBF1000F93
:10B4980041D0D9F8000000F00F00204305F0DAFA97
:10B4A8004FF0000B3DE0BBF1000F0CD0D9F80000C5
:10B4B800C0F3031020432CE0BBF1000F1ED199F814
:10B4C800010005F0C7FA99F8000005F0C3FA28E072
:10B4D800202B002004130020A82900201C2B00206A
:10B4E800142B0020102B00204F1C0020B429002012
:10B4F80035C2724F282B0020242B0020D9F80000D9
:10B50800C0F30330204305F0A5FAD9F80000C0F3D2
:10B51800071005F09FFAD9F800402401E4B24FF073
:10B52800010B09F1040906AB99454FEA9707A5D124
:10B53800BBF1010F02D1204605F08CFADAF8003091
:10B5480013F480541FBFB6F86420B5F86410521A7B
:10B55800029218BF012499040AD50AAA02EB8401B1
:10B56800B5F86600B6F86620121A41F8202C0134A6
:10B578005A0513D502AA02EB840E06F16A0705F1F3
:10B588006A00002237F9021F30F902CFCCEB010123
:10B598004EF822100132032AF4D103341F0508D5CE
:10B5A8000AAA02EB8400A96EB26E521A40F8202C47
:10B5B800013418040BD50AAB03EB8402B5F87210FA
:10B5C800B6F872305B1A42F8203C013400E0F4B15E
:10B5D800012C03D1029805F0EEFA18E0631E002052
:10B5E80002AA400052F82320C0B20AB140F001007C
:10B5F80013F1FF33F4D205F02DFA002702AB53F80C
:10B60800270008B105F0D7FA0137A742F6DB30204A
:10B618000321FFF771FC36200321FFF76DFC314B46
:10B628003C201978FFF768FCDAF80030990506D550
:10B63800B6F95E00B5F95E30C01A05F0BCFAD8F864
:10B6480000202948D8F80430C8F80420121A9110AC
:10B65800264AC8F808304A43531C032293FBF2F2E7
:10B6680002EB42029A1A742303FB0203C8F8003063
:10B678001F4B1B681A0630D51E4C1F4D22682B68BD
:10B688009A420BD162686B689A4207D1019B1B886A
:10B69800102B11D1194B1B885B060DD1482005F0E2
:10B6A800D9F9206805F087FA606805F084FA2368FC
:10B6B8002B6063686B600EE0114A0F4B11782A7C8F
:10B6C800914208D10F4A99681068884203D152689C
:10B6D800DB689A4201D0FFF731FC05F08BF90BB01B
:10B6E800BDE8F08F4F1C0020B429002035C2724FEE
:10B6F800442900208412002094290020222B0020B5
:10B70800F21A0020F41A00202DE9F84F0C9E3A4C4A
:10B71800C2EB030B0B9BF61A6368002914BF4FF0AA
:10B72800060A4FF0040A01330546904613D12368F0
:10B7380053455ED2314A324852F82320032B98BF32
:10B74800294605F075F96368013363602D4B0022C3
:10B7580005469A7113E0002511E02B4A12789542AC
:10B7680040DA0B9BE3B109FB06F2995C01228A409F
:10B77800264909680A4213D1636801336360D4F823
:10B7880004900A9B1C4F9945E7DB2BD10A2005F052
:10B7980061F93B6801333B604FF0FF337B6021E088
:10B7A800184A917921B12C2005F054F9013501E0AE
:10B7B80001219171226809FB0BF308EB030752B9C9
:10B7C80058F8030005F024F997F904104B1C0544B8
:10B7D800D2D00F4802E03A440E48117905F028F912
:10B7E8000544C9E7206850452CBF00200120BDE86A
:10B7F800F88F0020BDE8F88F2C2B00203483010837
:10B80800419F01083C22002014010020142B002035
:10B81800509F0108F8A6010830B585B004AC002592
:10B8280024F8025D0091ADF8060021461020FFF7CC
:10B8380027FC9DF806002146FFF722FC9DF807002B
:10B848002146FFF71DFC9DF800002146FFF718FC74
:10B858009DF801002146FFF713FC9DF802002146E0
:10B86800FFF70EFC9DF803002146FFF709FC9DF841
:10B878000E00C043C0B22946FFF702FC05B030BD38
:10B8880010B5054C2068FCF7BEFB18B12068FCF722
:10B89800B7FBF6E710BD00BF701B002013B50446C8
:10B8A80001A9006806F0AEF8132006F0E7F8BDF924
:10B8B800040006F0D1F81B2006F0E0F8BDF90600F8
:10B8C80006F0CAF8232006F0D9F82368002BB4BF85
:10B8D80053204E2006F0C0F801A9606806F092F8DF
:10B8E800122006F0CBF8BDF9040006F0B5F81A20CE
:10B8F80006F0C4F8BDF9060006F0AEF8222006F0FE
:10B90800BDF86368002BB4BF5720452006F0A4F8A3
:10B9180002B010BDF0B50124B0FBF4F58D4201D39F
:10B928004C43F9E70026D4B1B0FBF4F504FB15004D
:10B93800B4FBF1F41EB9002D01DC002CF3D1092D64
:10B9480003F1010EEFB204DD002A14BF3725572595
:10B9580000E030253D441D7001367346E3E71C7056
:10B96800F0BDF0B50124B0FBF4F58D4201D34C4392
:10B97800F9E70026D4B1B0FBF4F504FB1500B4FBDD
:10B98800F1F41EB9002D01DC002CF3D1092D03F1CF
:10B99800010EEFB204DD002A14BF3725572500E059
:10B9A80030253D441D7001367346E3E71C70F0BD39
:10B9B80003685A1C0260197070472DE9F843089E05
:10B9C800002B07468846144614BF4FF030094FF045
:10B9D8002009334613F8012B0AB9254603E0002C49
:10B9E800FBDD013CF6E7002D04DD38464946C0473B
:10B9F800013DF8E724EAE4743546A01B284415F80D
:10BA0800011B11B13846C047F7E7BDE8F883024B80
:10BA18001868FCF7FBBA00BF0011002090ED017A0E
:10BA280007EE901AB5EE407AF1EE10FA01BFF8EE83
:10BA3800E77A9FED0E7A67EE877AB7EE007A04BF51
:10BA4800C7EE277AC0ED017A90ED017AD0ED007A41
:10BA580030EE877A30EE670AC0EE870AE0EE807A29
:10BA6800B0EE670AC0ED007A704700BFDB0FC9402F
:10BA780010B50278202A034600F10100F9D0092AFE
:10BA8800F7D02D2A03D10346BFEE000A04E02B2A83
:10BA980008BF0346B7EE000ADFED387A1A461346A8
:10BAA80012F8010BA0F13001CCB2092C0AD807EE2C
:10BAB800101AB8EEC77AF2EE046AA7EEA67AF0EE8C
:10BAC800477AECE72E2816D1F2EE046A1146B0EE5A
:10BAD800666A0B4611F8012B303AD0B209280AD809
:10BAE80007EE102AB8EEC77A87EE267A66EE866ADF
:10BAF80077EE877AEDE71A7802F0DF02452A35D12A
:10BB08005A782D2A02D10233012004E02B2A14BFCF
:10BB1800013302330020013B002213F8011F3039A2
:10BB2800CCB2092C03D80A2404FB0212F5E7B2F5BB
:10BB38009A7F28BF4FF49A721346B7EE007A072B04
:10BB480005D9DFED0F6A083B27EE267AF7E702F002
:10BB580007032BB1F2EE046A27EE267A013BF8E7D9
:10BB6800F0EE476A20B1C7EE877A03E0F7EE006A85
:10BB780067EEA67A20EE270A10BD00BF000000007D
:10BB880020BCBE4C30B52DED028B87B0B0EE408A9C
:10BB98000C220021054603A809F02DFCB5EEC08A49
:10BBA800DFED2A7AF1EE10FACCBF38EE278A38EEAC
:10BBB800678ADFED277A28EE278A6946FDEEC87A7C
:10BBC80017EE904A84EAE470A0EBE470FDF7D2FD2A
:10BBD800002CACBF20232D2368468DF80C3009F0CB
:10BBE8004EFC012807D130238DF80D308DF80E302A
:10BBF8008DF80F300CE0022805D130238DF80D3078
:10BC08008DF80E3004E0032804BF30238DF80D3082
:10BC1800694603A809F016FC03A809F030FC0338AC
:10BC2800C4B2224603A9284609F056FC00232B5526
:10BC38002846084909F006FC03AB2846191909F0FB
:10BC480001FC284607B0BDEC028B30BD6F12033AE9
:10BC580000007A44749F010870B5064615460846E8
:10BC6800B6FBF2F414B12046FFF7F6FF05FB1464A7
:10BC7800024B1B5D00F8013B70BD00BF769F0108B9
:10BC88002DE9F04F814689B08A4616461C460025A4
:10BC98003178002900F0DD80252902D00136484698
:10BCA80075E07278302A08BFB278A2F1300319BF64
:10BCB800B71C4FF0000BF71C4FF0010B092B4FF08E
:10BCC800000819D8A2F13003D9B2092905D80A22E7
:10BCD80002FB083817F8012BF4E7A2F16103052BE2
:10BCE80002D8A2F1570305E0A2F14103052B03D8BE
:10BCF800A2F137030A2BEADD6C2A31D13A78642A9B
:10BD080007F1010600F083800BD8252A3DD003D81F
:10BD1800002A00F09E80BBE7582A0CD0632A19D06D
:10BD2800B6E7732A22D002D86E2A37D0B0E7752A30
:10BD38005CD0782AACD1271D2068A2F15804624251
:10BD48004FF01001624155E02CD9582A32D0632AAD
:10BD58002AD13E4648462178271DD04701350FE0B5
:10BD6800642A64D00ED9732A14D13E4623680093FE
:10BD78004846514642460023FFF71FFE271D05444B
:10BD88003C4685E7252ADFD13E4648462521D0474F
:10BD980001357DE70AD86E2A06D13E462368043469
:10BDA8001D6075E7002A54D03E4671E7752A26D0F3
:10BDB800782AF9D1A2F1580304F1040C5A422068F8
:10BDC800CDF80CC04FF010015A4105ABFFF7A2FDAA
:10BDD800DDF80CC03E46644605AB00934846514624
:10BDE80042465B46FFF7E9FD054451E72068271DF9
:10BDF8000A21002205ABFFF7B4FD3C46ECE704F14D
:10BE0800040CCDF80CC020680A210022DDE7206868
:10BE1800002804F1040708DA2D238DF81430404275
:10BE28000DF115030A210022E5E705ABFAE72068C2
:10BE3800002804F1040C0ADA2D238DF8143040424E
:10BE48000DF11503CDF80CC00A210022BEE705ABA1
:10BE5800F8E7284609B0BDE8F08F0FB413B50B49D1
:10BE680004AB08680A4953F8042B09680193FFF7E3
:10BE780007FF0446074B1868FCF7BCF80028F9D000
:10BE8800204602B0BDE8104004B070478C01002085
:10BE9800880100200011002080EAE073A3EBE07322
:10BEA8008B4206DB002801DD401A704702D00844A7
:10BEB800704700207047FDEEC07A17EE903A2033A5
:10BEC800402B43D8DFED237AB4EEE70AF1EE10FAFF
:10BED80004DDDFED217A30EE670AF3E7DFED1F7A44
:10BEE800B4EEE70AF1EE10FA04D5DFED1B7A30EE76
:10BEF800270AF3E7DFED1A7AB4EEE70AF1EE10FA53
:10BF080004DD30EE670A37EEC00A0AE09FED157AC5
:10BF1800B4EEC70AF1EE10FA44BF30EE270A37EE46
:10BF2800400A60EE007ADFED106A9FED107AA7EE06
:10BF3800A67ADFED0F6AE7EE876A9FED0E7AA7EE25
:10BF4800A67A20EE276AA6EE070A70479FED0A0A2E
:10BF5800704700BFDB0F4940DB0FC940DB0F49C00A
:10BF6800DB0FC93FDB0FC9BF9A7C2E36FAAF4FB93A
:10BF78003587083CA4AA2ABE00000000DFED027A3B
:10BF880030EE270A97E700BFDB0FC93F38B52DED24
:10BF9800068B90ED008AB0EE480A0C460546FFF77E
:10BFA800EDFFB0EE40AAB0EE480AFFF784FFD5EDEA
:10BFB800018AB0EE409AB0EE680AFFF7DFFFB0EEF4
:10BFC800408AB0EE680AFFF776FFD5ED02AAF0EED8
:10BFD800408AB0EE6A0AFFF7D1FFF0EE409AB0EE61
:10BFE8006A0AFFF768FF60EE0A6A69EE297AF0EEDE
:10BFF800665AE7EEA85A29EE8A6A29EE007A69EEAF
:10C00800889A29EE489A28EE400A28EE0A8AC4ED52
:10C01800035AF0EE465AE7EE685AE6EEA87AA6EE1C
:10C02800687AC4ED009AC4ED028A84ED059A84ED1D
:10C03800088ABDEC068B84ED010AC4ED045A84ED30
:10C04800067AC4ED077A38BD10B52DED048B8AB099
:10C0580090ED009AD0ED028A90ED018A04460846D8
:10C0680001A9FFF793FFDDED047A9DED017A68EEF3
:10C07800277AE9EE077A9DED077AE8EE877A9DED53
:10C08800027AC4ED007ADDED057A68EE277AE9EEEA
:10C09800077A9DED087AE8EE877AC4ED017ADDED3E
:10C0A800067A28EE278ADDED037AA9EE278ADDEDE8
:10C0B800097AA8EEA78A84ED028A0AB0BDEC048B3F
:10C0C80010BD074B1A8822EA0000904210B518806C
:10C0D8001C4602D00120FBF723FF208810BD00BFBB
:10C0E800B01B0020064B1A881043904210B51880E8
:10C0F8001C4602D00120FBF713FF208810BD00BFAB
:10C10800B01B0020024A936823EA00009060704741
:10C118000413002008B5104B1A780023D9B29142B5
:10C1280007D20E4951F8231009680020086001332E
:10C13800F4E73220FBF797FE094B1B685A0309D531
:10C14800084B9B685B0305D440F2DC50BDE808400F
:10C15800FBF789BE08BD00BF4F1C0020781C0020DB
:10C1680044290020041300202DE9F34105F0CEFBFB
:10C17800454A6A2313704FF4FA635380BE23137140
:10C18800EF2382F8CD37002382F8CE3719461646BA
:10C19800F25C0133B3F5FA6F81EA0201F8D13A4B48
:10C1A80083F8CE17394B1A69120604D5384A5A60F3
:10C1B80002F188325A6004270020013F17F0FF0778
:10C1C8004FD0324B3422DA60002444B1002356F8B1
:10C1D80004800193FDF79EFA0428EED117E0FDF7DD
:10C1E80099FA0428E9D1294D2B6943F002032B6100
:10C1F800284B6B612B6943F040032B61FDF78AFAEA
:10C208002B69042823F002032B61DFD0D5E71F4DEB
:10C218002B6943F001032B6104F1006303F57E33BE
:10C228001FFA88F21A80FDF775FA042810D11A4B04
:10C2380023440193019B4FEA1848A3F80080FDF7B7
:10C2480069FA2B69042823F001032B6105D0B4E7B0
:10C258002B6923F001032B61AFE70434B4F5FA6FBF
:10C26800B3D10A4A1369042843F08003136102D149
:10C2780004F0FCF810B90520FBF76AFE05F030FB66
:10C2880002B0BDE8F08100BF041300200020024086
:10C298002301674500F8030802F8030810B50E4C9F
:10C2A8002068FBF723FD2068047A002202FB02F3D2
:10C2B800193B634303F6C4135343192193FBF1F36A
:10C2C800064921F812300132072AEFD10449BDE8A6
:10C2D8001040FEF749BD00BF7C120020D01000209E
:10C2E800441400202DE9F04104F0C0F810B90420EE
:10C2F800FBF72EFEB14CB24D05F008FBB1494FF4E7
:10C30800FA62204609F06CF894F8A437022B84BF2F
:10C31800002384F8A43794F8A4274FF4CC7101FBC8
:10C3280002F3E018234400F53770286093F83003CF
:10C3380003F54A73022801FB024284BF00201872E9
:10C3480092F83033A04A13700C2202FB03439F4A31
:10C3580003F2A6731360A36846F209021A401AB9D9
:10C36800964A43F400539360A368D80703D54FF463
:10C378000050FFF7C7FEA368590409D50820FFF746
:10C38800C1FE4FF40050FFF7BDFE0120FFF7BAFED3
:10C39800A3681A0706D54FF40050FFF7B3FE012033
:10C3A800FFF7B0FEA3689B0406D54FF48030FFF773
:10C3B800A9FE4020FFF7A6FE012284F80D2294F87A
:10C3C800DC217E4B2AB193F8E02112B1002283F8D8
:10C3D800E0217F4B7F4E1E604FF0000C674604EB58
:10C3E8000C03B3F8F4E14FEA5E0101F077314FEA4C
:10C3F8009E0303F03333C1EB0E00C11A4FEADE038C
:10C4080003F01133CB1A03EB23131EF0010803F0DA
:10C418000F324FF0FF0392FBF3F3C3EB032318BF74
:10C428000137A2EB030318BFFFB2012B0ADD022B71
:10C4380040F0C180B8F1000F00F0BD801EF0BC0FC5
:10C4480000F0B9800CF1080CBCF1180FC7D1013FFE
:10C45800012F00F2B080FFF721FF302200215E4853
:10C468005E4F08F0C8FF5E4BD5F800801F605D4B3B
:10C47800002108F17900C3F80080FBF777FC5A4BDC
:10C4880080F001001870594B07F126021A60584BCA
:10C4980007F1CC021A6098F80000FBF7F3FF286850
:10C4A800544B00F5C5721A60FCF734FF524B94F8F0
:10C4B800D401DFED526A07F194021A606421504BEF
:10C4C800C82211FB00225A6000229A60DA601A61C1
:10C4D8005A619A61DA6183F8202083F82120494B58
:10C4E80007F12C021A602B68474A93ED187A03F279
:10C4F80019111160454A03F289111160444A07F184
:10C5080008011160434A1760434A07F1A00111600E
:10C51800424A07F1AA011160414967EE266A0E6096
:10C52800B4F86211B6EE007A07EE901A87EE267A12
:10C53800B4F86411101DF8EE677AC2ED027A07EEBE
:10C54800901A93F85C10117193F87810517194F85F
:10C55800DF111174F8EE677AB3F81611C2ED037A99
:10C5680007EE901A2F49086053612F4A03F16401BE
:10C5780011602E4A2E4982ED007AF8EEE77A9FED97
:10C588002D7A2D4A0B60C7EE277A2C499FED2C7A1D
:10C5980067EE877AC2ED007A03F168020A602949DA
:10C5A80003F211130B60284B1F60284BBDE8F041C4
:10C5B8001A6005F095B9FDF779F84CE704130020E7
:10C5C8005812002000F80308F02800207C120020F0
:10C5D800002D00208A14002004100020441400209C
:10C5E800381000203C100020140000200C08002007
:10C5F8008806002048100020D0270020DB0F494083
:10C608000C2D0020640800209C220020740A0020C1
:10C61800E81D0020EC1D002088090020442200208D
:10C628004C0A002094080020CC080020C8080020EC
:10C63800782D002000006144840900206C2D002022
:10C648004C3D0F447809002080090020482D002027
:10C6580008B5FFF789FDFFF745FE0120BDE8084052
:10C66800FBF75EBC38B500240B4D6059254403F038
:10C67800E7FC696811B10948FFF7EFFBA96811B138
:10C688000748FFF7EAFB0748103403F0D9FCB4F574
:10C69800D87FE9D138BD00BF4C8301089B9F0108B2
:10C6A800A19F01089EA70108F0B585B0044608F0CF
:10C6B800E6FE082826D1621EE01D1F4912F8013F38
:10C6C80009681944497801F00301022908BF203B91
:10C6D80082421370F1D1254604F1080715F8016B61
:10C6E8001648314608F0BDFE20B12846314608F00C
:10C6F800B8FE10B1FDF724FE1CE0BD42EED1204685
:10C70800FDF71AF80E4803F09BFC00230D4A1A4463
:10C7180004A992F886210A440849595C02F80C1CBD
:10C728000133082BF2D1002307488DF80C3001A9FA
:10C73800FFF793FB05B0F0BD180100204A9D0108E2
:10C74800A79F010804130020E0A60108234B244CEE
:10C758001D68206880B5FEF7B5F82846FEF7B2F8E0
:10C76800206841798B0704D4036841F002015B69B2
:10C7780098471C4B4FF488521A854FF488421A8503
:10C788002068FBF740FCA0B1164E4FF48853B36104
:10C79800134B1868FBF734FC0746FCF70FFA08B18F
:10C7A80002F03CFC28463946FBF730FC4FF488532E
:10C7B80033852846FBF727FC0028E1D0094ED4F83A
:10C7C80000804FF48847B7612846FBF719FC0146FB
:10C7D8004046FBF71BFC3785D2E700BF0C29002039
:10C7E8005C220020001000482DE9F047054608F0BB
:10C7F80046FE314E0446D6F8088090B92F4803F01B
:10C808001FFC2F4B53F8241049B10123A34013EA0E
:10C81800080F02D02B48FFF720FB0134F1E72A4824
:10C8280022E028462949224608F032FE58B928480D
:10C83800284C03F005FC54F8041F0029EFD02148C8
:10C84800FFF70BFBF7E72B782D2B03BF013504F11E
:10C85800FF344FF0010A4FF0000A4FF00009184B5F
:10C8680053F8297027B91C48BDE8F04703F0E8BB26
:10C8780028463946224608F00BFEC8B9012000FABE
:10C8880009F0830501D51548EEE7BAF1000F03D08A
:10C89800FFF738FC124803E040EA0800B06011488E
:10C8A80003F0CEFB39461048BDE8F047FFF7D5BA8C
:10C8B80009F10109D3E700BF04130020AD9F010867
:10C8C800FC840108B79F01089EA70108BB9F0108C7
:10C8D800C09F0108F8840108BB9E0108CC9F01088D
:10C8E800DA9F0108E39F0108DFA6010810B5084890
:10C8F80003F0A6FB074B00241C715C63064B1C70FD
:10C90800FBF708FD03F080FD044B1C6010BD00BF61
:10C91800EB9F01085C220020BA2D00200C29002082
:10C9280070B5064600240B4BE518AA8816420AD0B3
:10C93800E1580948FFF791FA2846002103F00DFB5A
:10C94800064803F07DFB143440F66C439C42EAD160
:10C9580070BD00BF8489010817A001089EA70108BF
:10C96800F0B504788BB005460CB1002436E04B4B8B
:10C9780019680E2303FB041101F58C70B1F91D51E0
:10C98800B1F91921B1F91B31009591F820510195A0
:10C9980091F82151029590F90700039001F59071E3
:10C9A8003F4891F90210049121460134FFF755FAE6
:10C9B800082CDCD170E02D2B14D1072C1BDC284669
:10C9C80008F0B4FD0AAB661C03EB440424F8100C11
:10C9D80015F8013F303B092BFAD934462B78002B48
:10C9E800E9D104E0A3F13002092A09D8E5E7082CC7
:10C9F800BDF8182009D00BB0BDE8F040FDF7A0BC89
:10CA0800202BF8D101352646E7E7072AF3D8BDF8E9
:10CA18001A00224BA0F2EE2189B240F2DC55A9425D
:10CA28001B68E8D8BDF81C10A1F2EE24A4B2AC42F1
:10CA3800E1D8BDF81E6004B237B2A742DBDB0DB205
:10CA4800AF42D8DCA542D6DBBDF8247007F16404F8
:10CA5800A4B2C82CCFD8BDF826E00FFA8EF4112C5A
:10CA6800C9DCBDF82050B42DC5D8BDF82240B42C7F
:10CA7800C1D812B24FF00E0C0CFB0233A3F8190107
:10CA8800A3F81B11A3F81D6183F8205183F82141F5
:10CA980083F81F7183F822E10BB0F0BD5812002013
:10CAA80021A00108F0B504468FB0204608F0E7FC45
:10CAB800C5B225BBAF48B04C03F0C2FA94F8D21007
:10CAC80009B9AE4854E049B294F8D02094F8D1306E
:10CAD800009194F8D310019194F9D410029194F92B
:10CAE800D510039194F8D6100491A548294601352C
:10CAF800FFF7B3F9102D04F10704DFD1E1E7204671
:10CB0800A049052208F0C4FC0546B8B929469E4844
:10CB1800702208F070FC9D4B196828460E2303FB11
:10CB2800001301300022082883F8232183F82421E8
:10CB380083F8252183F82621F0D119E1204694496C
:10CB4800042208F0A5FC05462046002D4AD12021E4
:10CB580008F087FC002800F00B81461C304608F0DE
:10CB68008EFC2C4607468B4B53F824502DB98A4827
:10CB78000FB0BDE8F040FFF770B930462946FAB269
:10CB880008F086FC01340028EDD17B4A02F17001DF
:10CB98001646002382F8D63082F8D23082F8D13097
:10CBA80082F8D03007328A42F3D17C4901EBC401C4
:10CBB80091F80822934210DAD1F80C72C3EBC30241
:10CBC800B0183A4400F1D0011768C0F8D0709088C6
:10CBD800888092798A710133E7E729467048FFF720
:10CBE8003CF996E06F49072208F052FC05462046BA
:10CBF800002D4AD1202108F034FC064608F03FFCFD
:10CC0800C4B274BB6848FFF728F921466748013465
:10CC1800FFF723F90E2CF8D15848FFF71EF9002426
:10CC280063482146FFF719F90025584A61481168F9
:10CC38000E2202FB04120123D2F823215E49AB40E5
:10CC480013425E4B05F1010508BF1946FFF705F9C8
:10CC58000E2DEAD149480134FFF7FFF8082CDFD13F
:10CC680086E03046564908F065FC2C46002852D02C
:10CC7800022C55D008F05AFC06AB514943F8240061
:10CC8800002008F057FC0134F0E74D4908F052FC49
:10CC9800002460B1082C3ED008F048FC06AB484997
:10CCA80043F82400002008F045FC0134F1E7082C83
:10CCB80031D1069B0F2B2ED8DDF81CE0BEF1070FF3
:10CCC80029D8089F0D2F26D8099E06F16402C82A84
:10CCD80021D80A9DFF2D1ED80B9864281BD80C99C3
:10CCE800642918D8884216DA0D9C032C13D8224AD6
:10CCF800C3EBC303134483F8D0E083F8D17083F8FF
:10CD0800D26083F8D35083F8D40083F8D51083F821
:10CD1800D6402C4CC9E60FB0BDE8F040FDF710BB7B
:10CD2800069B072B20D807990D291DD80278722A4F
:10CD38000DD06E2A18D1154A12680E2000FB032365
:10CD480001228A40D3F8231121EA020209E00F4A9E
:10CD580012680E2000FB032301228A40D3F8231116
:10CD68000A43C3F8232101E0FDF7EAFA0D4C9CE6DB
:10CD78000FB0F0BD49A00108041300209EA70108C8
:10CD880074A001088B9E0108D413002058120020BB
:10CD9800B69E0108F0950108BB9E01084C83010866
:10CDA800CA9E010841A00108A59F010890A001089A
:10CDB800F8A6010895A00108E4AA01089EAB01089D
:10CDC80099A001080B9C01082DE9F7430478054652
:10CDD8008CB9324D95F89F12B5F89C2295F89E3281
:10CDE8002F48009121460134FFF737F8102C05F140
:10CDF8000405EFD14EE008F099FB0F28044636DC15
:10CE08002846202108F02DFB264EE4B2D6F83880BB
:10CE1800451CA4000027284608F088FB5FFA87F91C
:10CE2800B9F1010F83B208D0B9F1020F0BD0B3F5F5
:10CE3800B47F24D2B26B13530AE0FF2B1FD8B36B15
:10CE48002344987004E0FF2B19D8B36B2344D8709F
:10CE580028462C2108F005FB054608B1013502E0FB
:10CE6800B9F1020F0BD10137032FD4D112E00E48CC
:10CE780000210F2203B0BDE8F043FDF7DEB908EB4F
:10CE880004000021042208F0B6FA03B0BDE8F0431C
:10CE9800FDF756BA03B0BDE8F08300BF04130020C5
:10CEA8009BA001085C220020649E01082DE9F04344
:10CEB80004788FB00546002C59D17C4B00211422F0
:10CEC80009A807AED3F83C8008F095FA0722304647
:10CED800002108F090FA05A80023A700059308EBA5
:10CEE800070583801A467249B5F802E031F813C085
:10CEF8001CEA0E0F0AD00DF1380C0E3102F1010EAA
:10CF08006244595C02F81C1C5FFA8EF20133072B4D
:10CF1800E9D100210B46674AB5F802E011F802C0D2
:10CF28001CEA0E0F0AD00DF1380C063203F1010E7F
:10CF380063448A5C03F8242C5FFA8EF301310629D6
:10CF4800E9D118F807305C498DE841006A78029207
:10CF580009A81A0903F00F0304F0BAF82146574844
:10CF680009AA0134FEF779FF202CA6D19BE008F02E
:10CF7800DDFA1F28044600F3898028462021E4B200
:10CF880008F06FFA1F2C02D9FDF7DAF98BE0474B4E
:10CF9800DB6B03EB8404451C00212046042208F0C7
:10CFA8002AFA0027464B09AE304600210A2217F814
:10CFB80003905FFA87F808F01EFA002315F8012B92
:10CFC80032B10A2B04D04A4502D0F2540133F5E7B6
:10CFD8004A4561D108F1FF33032B09D8DFE803F094
:10CFE800100502420DF1230037E00DF123011FE087
:10CFF800304608F09BFA2378C0B243EA001006E0F6
:10D00800304608F093FA237800F00F001843207098
:10D0180034E00133062B0BD02A4800F2F3269E5D3C
:10D028009642F6D1034493F8ED2263881343638054
:10D0380011F8012F12B30023EEE70133072B0CD0B0
:10D04800204A02F2E6269E5D8E42F6D102EB4303A9
:10D05800B3F8D82263881343638010F8011F69B1BD
:10D068000023EDE7304608F061FA0F2804DC30466B
:10D0780008F05CFA607001E0002363700137052F47
:10D0880090D1012401F070FF6CB97DE70E480021B2
:10D098001F22FDF7D2F806E020460021042208F0FE
:10D0A800AAF90024EEE70FB0BDE8F0835C22002067
:10D0B8002486010839860108AFA00108BEA001082E
:10D0C800458601084C830108649E01082DE9F0415A
:10D0D8002DED048BB1498AB0044608F095F9B049A2
:10D0E800002820460CBF0126072608F08DF9AD4917
:10D0F8000028204608BF022608F086F9002808BF45
:10D108000426F10740F1EF80A748A84C02F098FFE9
:10D11800002002F0A1FDA64802F092FFA54802F007
:10D128008FFF6379A44AA548013B254652F823108E
:10D13800FEF793FEA248FEF790FE4FF00008274640
:10D1480095ED048AB5EE408AF1EE10FA04D19D48B7
:10D15800FEF783FE002570E09B48D5ED059A95ED16
:10D16800069AD5ED078A4146FEF777FEB5EEC08AE6
:10D17800F1EE10FA02D5202002F05AFFB0EE480A6C
:10D1880006A8FEF7FFFC01469048FEF766FEF5EE9E
:10D19800C09AF1EE10FA02D5202002F049FFB0EE55
:10D1A800690A06A8FEF7EEFC01468848FEF755FE18
:10D1B800B5EEC09AF1EE10FA02D5202002F038FF41
:10D1C800B0EE490A06A8FEF7DDFC01467F48FEF7E7
:10D1D80044FEF5EEC08AF1EE10FA02D5202002F0E6
:10D1E80027FFB0EE680A06A8FEF7CCFC08F1010894
:10D1F80001467748FEF731FEB8F10C0F05F110052E
:10D208009ED1A4E749B294F8D02094F8D130009187
:10D2180094F8D310019194F9D410029194F9D5108F
:10D22800039194F8D61004916A4829460135FEF70F
:10D2380014FE102D04F1070403D094F8D21000292D
:10D24800E0D16548654C02F0FBFED7F8088054F839
:10D25800041F19B16248FEF700FEF8E70D46614B5E
:10D2680053F8254054B10123AB4013EA080F03D00B
:10D278005D482146FEF7F1FD0135F0E75B4802F015
:10D28800DFFE21467B180AAA93F886311344584AD0
:10D298008A5C03F8102C01310829F3D1002306A970
:10D2A80054488DF82030FEF7D8FD534802F0C8FEE8
:10D2B8005248FDF785FC524802F0C2FE4F48FFF77E
:10D2C800F5FD504802F0BCFE4C48FFF77DFD4E4886
:10D2D800FEF7C3FD4020FFF723FB4C4802F0B0FEE9
:10D2E8004648FDF757FAB20739D5494802F0A8FE73
:10D2F800484802F0A5FE414802F0EEFC464802F01C
:10D308009FFE3E48FCF7A6FF444802F099FE3B48C2
:10D31800FDF792F94248FEF7A0FD3848FDF716F8E8
:10D32800404802F08DFE3548FFF71AFB00270E250E
:10D338007D4300243C4A126C2A440123D2F80A2077
:10D34800A34013421ED101340E2CF3D10137082F0C
:10D35800EDD12D48FEF781FD8020FFF7E1FA730734
:10D3680016D5324802F06CFE314802F069FE2348B7
:10D3780002F08CFC2448FEF770FD4FF48070FFF734
:10D38800CFFA05E0394622462A48FEF766FDDAE775
:10D398000AB0BDEC048BBDE8F08100BFCAA001084B
:10D3A800DAA40108D1A00108D7A0010804130020BD
:10D3B800E5A00108F7A00108F095010803A10108FC
:10D3C8000EA101081BA1010828A10108A49F0108BA
:10D3D800E0A6010840A1010830A10108F88401086D
:10D3E8005FA10108FC8401086DA101087AA1010868
:10D3F8004A9D010886A101088FA101080B9C01081C
:10D408009EA10108AAA101089EA70108B8A10108C8
:10D41800C5A10108D8A10108E6A10108F0A10108E9
:10D42800FFA101080DA201085C22002019A2010831
:10D438002AA201083CA20108026D036B70B50446DC
:10D44800D5699BB9A90611D5C36A1BB1908C80B266
:10D4580098470BE0E169928C40694E1CD2B2E661B4
:10D468004254E169E268914228BFE361616BA1B966
:10D478002A0612D5636AA26A9A42236D09D0501C03
:10D48800A669A062B25C1A852369984205D3A16295
:10D4980003E01A6822F080021A602B0742BF236D4E
:10D4A80008221A6270BD026BC168034610B5406954
:10D4B80042B11A6C8C1A013A005D08BF0A46C0B224
:10D4C8001A6410BD1A6A805C01328A4228BF0022A1
:10D4D800C0B21A6210BD436B13B190F84400704794
:10D4E800836A406A1B1A584258417047036B13B14C
:10D4F8005B68016C01E0C369016A8B423CBFC2688A
:10D508009B18581AC0B27047836A8169426B1944E4
:10D51800D160416A99429DBF0169CB1A5360CB1A09
:10D5280096BF0023536083624FF0000380F84430B5
:10D53800136888BF816243F0010313607047436A30
:10D548008269D154436A02690133934228BF002398
:10D558004362436B1BB11B68DB0705D4D4E7026D3C
:10D56800136843F08003136070474171F7F790B96F
:10D578008160F7F78DB92DE9F0410369C768054661
:10D588000E461F40002F35D0B7FA87F24FF0004300
:10D59800D340DB432B611F40A2F11B03042BF1D8BE
:10D5A800DFE803F0221F1C190300746A24B1013C50
:10D5B8000023A4B2736201E0EC6AA4B2D6F820801A
:10D5C800B8F1000FDED0D8F8003040462146984721
:10D5D800D8F80480F4E73068696B07E07068A96BD5
:10D5E80004E0B068E96B01E0F068296C036889B26F
:10D5F8009847C7E7BDE8F08101480249BBE700BF8B
:10D6080000040040F81C00204FF080400049B2E7B9
:10D61800D01C002010B5054C05482146FFF7ABFF8C
:10D6280004F1F0010348BDE81040A4E7A81C00205D
:10D63800002C014000440140014802499BE700BF1B
:10D64800002C0140A81C0020224B10B5224C5A4344
:10D65800224BB3FBF2F203880139013AA04289B2A6
:10D6680092B29BB20ED004F50064A0420AD0B0F189
:10D67800804F07D0A4F59834A04203D004F5806405
:10D68800A04202D123F070039BB2154CA04206D0F1
:10D6980004F58064A0421CBF23F440739BB203804E
:10D6A8000D4BC162984202850FD003F50063984282
:10D6B8000BD003F54063984207D003F58063984286
:10D6C80003D003F58063984201D100230386012328
:10D6D800436110BD40420F00002C014000A24A04E3
:10D6E80000100040164B800A984226D00AD84A3BC0
:10D6F800984218D00133984217D0B0F5801F1AD13C
:10D70800012070470F4B984211D004D8033B984230
:10D7180011D1042070470C4B98420AD0013398422B
:10D7280009D1072070470220704703207047052061
:10D73800704706207047FE2070470020704700BFE2
:10D748004B0010005000100051001000F8B504689C
:10D75800064620460F461546FFF7C4FF07284BD854
:10D76800B27A910847B902238B40D4F80CE0DB4326
:10D778009BB203EA0E03E3600A23204A03FB00136B
:10D7880042F82370043342F8235015463FB1B17A6A
:10D79800E268890802238B409BB21343E360282286
:10D7A80002FB00522032EFF31286502383F31288D3
:10D7B80003B203EB8303DB0003F10C011C332944A0
:10D7C8002B4451F8047F17B117600A680432994254
:10D7D800F7D100231360F3B283F31188282303FBE6
:10D7E8000050036A1BB1E36843F0010303E0E268F9
:10D7F8004FF6FE731340E360F8BD00BFA81C00207D
:10D80800004819E6A0220020004815E6F42200206E
:10D818000D4B0E484FF400525A600D4A11684FF6EE
:10D82800FE730B401360D0F8882011684FF6FE7322
:10D838000B401360826FC36F9A4201D0543063E685
:10D84800012380F89830704700000240A022002091
:10D85800440002402DE9F0471E46A54B8CB0984283
:10D86800894690469DF8507040F08B80A14BA24AA3
:10D878005A6503F1A8029A6603F5D472DA664FF482
:10D8880080721A665A669D4AC3F88420143AC3F80F
:10D898008820A2F54842203AC3F8A0200432C3F8F1
:10D8A8009C20C3F85C80C3F8A400954B9A6942F4A5
:10D8B80080429A615A6942F001025A6102238DF846
:10D8C8000830032317F0010A8DF809304FF00003E0
:10D8D8008DF80A3014BF022301233A078DF80B3064
:10D8E80019D54FF090444FF4007501958AF0010363
:10D8F8008DF80A30636A23F0F0036362636A43F0C9
:10D9080070036362204601A9FCF77AFBBAF1000FA5
:10D9180027D1A56125E0B30710D50CA94FF40073F2
:10D9280041F82C3D4FF09040436A23F0F0034362E6
:10D93800436A43F070034362FCF762FBF50710D5B6
:10D948000CA94FF4806341F82C3D4FF09040436A96
:10D9580023F470634362436A43F4E0634362FCF771
:10D968004FFB0E238DF800300022012368468DF806
:10D9780001308DF802208DF80330624C03F04AF92B
:10D9880074E0614B984240F003815A4B5A4A1A603E
:10D998004FF48072DA601A6103F52A725A6103F54E
:10D9A8006A729A61564AC3F808801865D36943F4C5
:10D9B8000033D36102238DF80830032317F0010ADE
:10D9C8008DF809304FF000038DF80A3014BF022398
:10D9D80001233C078DF80B3017D54C4C20250195B9
:10D9E8008AF001038DF80A30236A23F47003236256
:10D9F800236A43F4E0032362204601A9FCF700FBF5
:10DA0800BAF1000F23D1A56121E0B0070ED50CA90A
:10DA1800202341F82C3D3D48036A23F47003036238
:10DA2800036A43F4E0030362FCF7EAFAF1070ED550
:10DA38000CA9402341F82C3D3448036A23F0706355
:10DA48000362036A43F0E0630362FCF7D9FA262312
:10DA58008DF800300022012368468DF801308DF8DA
:10DA680002208DF8033003F0D5F8224CC4F82C902E
:10DA78000025012384F844302562E561A5626562CA
:10DA88006671C4F80880A7712046F6F701FFF2070F
:10DA980045D5236B002B3BD001A8FCF759F8E36C64
:10DAA80001934FF480530A9380230693E368ADF8FB
:10DAB800103020230993206B636902930B95059519
:10DAC800079508950395FCF76EF801A9206BFCF7FC
:10DAD8004CF8236B216D1A6842F001021A608A68BB
:10DAE80042F040028A605B689BB2236417E000BF83
:10DAF80000380140A0220020088701085800024091
:10DB080000100240F422002000440040000C0048AD
:10DB1800236D20221A621A6842F020021A60B307A5
:10DB28002FD5636B43B301A8FCF712F8A36C0193DC
:10DB38004FF480530A93802306932369ADF810307D
:10DB480000251023606B03930B95059507950895A1
:10DB58000995FCF728F8606B01A9FCF706F8636BD8
:10DB68001A6842F002021A60226D5D605D60936877
:10DB780043F08003936004E0226D136843F0800350
:10DB88001360226D136843F001031360204600E020
:10DB980000200CB0BDE8F0872DE9F74FA74CFAF745
:10DBA8003BF926686568A768861BF643451BC71BB3
:10DBB800ED43FF43F60F8046ED0FFF0F2EB93FB937
:10DBC800002D00F08682B9462CE04FF0000929E0CC
:10DBD800B14627E003EB8A0BBBF802301A050ED4D6
:10DBE80013F4805F1DBF964A9BF801101268954A8E
:10DBF800954B14BF52F82120126843F82A20BBF82D
:10DC08000230D80516D499050AD5904B1B7813F025
:10DC1800040F0CBF8E4A8F4A8B4B126843F82A2098
:10DC280009F10109207B8C495FFA89FA82450B6862
:10DC3800D0D326E0894A5046594601F025F9884B49
:10DC48001B885A0603D550465946864A16E0580797
:10DC580003D550465946844A10E0190703D5504663
:10DC68005946824A0AE09A0703D550465946804ADF
:10DC780004E0DB07D4D57F4A5046594601F004F941
:10DC8800CEE7DFF808E20093BEF906307822A3F564
:10DC98007A7353434FF47A7293FBF2F303F22B1324
:10DCA80001930022F3465FFA82FE864517D2009B55
:10DCB80003EB820EBEF802E01EF4806F0DD0DFF891
:10DCC8008891019B39F822E040F2671A9E449EFB36
:10DCD800FAFC0AFB1CEE29F822E00132E3E74DB317
:10DCE80008F5C333A0336360637B544A13BB937353
:10DCF800614B1B6813F0020F0AD0DFF894E19EF81D
:10DD080000E0BEF1000F03D04FF0010E82F80EE0E4
:10DD1800DA0506D5594BDB781BB1A37B43F0020328
:10DD2800A3734A4B1B7813F0050F02BFA37B43F084
:10DD38000403A37394F80EE0BEF1000F03D13F4B28
:10DD48005B7B002B4FD094F80DC01CF0010FACF199
:10DD58000C031DD1BCF1030F07D8DFF8E8903C4A4B
:10DD68001EF0040F08BF4A4600E0364AACF1040C26
:10DD7800BCF1070F05D8DFF81CC11EF0010F18BF52
:10DD88006246DBB2032B0ED81EF0020F3C4B06E0B6
:10DD9800DBB2032B06D82F4B2A4A1EF0020F18BFFE
:10DDA8001A4600E0274A4FF0000C5FFA8CF38342D2
:10DDB8000DD20B6803EB8C035B881B0642BF224B1A
:10DDC800D2F8009043F82C900CF1010CEDE785B1E6
:10DDD800BEF1000F08D0637B184A0133DBB2142B65
:10DDE80006D1002304E025B1637B002BF3D100E0CA
:10DDF8005373002E52D0234AB2F90250B2F90020D0
:10DE0800002DB8BF6D42002A4FF03203B8BF52420E
:10DE180095FBF3F592FBF3F2EDB2D3B2AB4238BF08
:10DE28002B46194A13B192FBF3F300E0134643441F
:10DE38002360E37B014A7BBB01232EE048270020B7
:10DE480094220020B4980108BA0E0020B72D0020B3
:10DE58007C9701086C970108982200202087010808
:10DE6800B01B0020268701082C870108328701088B
:10DE7800388701083E870108442900200C2D00201E
:10DE880084970108FC120020400D03002C2C002070
:10DE9800381B00208C9701080023D3738E4D8F4BBD
:10DEA8002D78E27BADB9002F00F00E818C4B267BDC
:10DEB8001A788C4B8C4D93F800C08C4BD3F800E04B
:10DEC8000B6802F004020021D2B203EB86060F466B
:10DED800B5E01AB9864A1A61002508E0854AFAE7CA
:10DEE8000A68AB00D6187688760604D40135EBB2FA
:10DEF8008342F5D3D7E7804EB6F90060192E25DDA9
:10DF080012F803E094F814C026690EF00F09E145F1
:10DF18000CDCDFF8C8C19CF815C0BCEB1E1FDEBFC7
:10DF2800DFF8D8E1D6F800C043F80EC012F803E0D5
:10DF380094F816C00EF00F09E14533DBDFF89CC1F9
:10DF48009CF815C0BCEB1E1F2CDC26E0193629DA1C
:10DF580012F803E094F814C026690EF00F09E145A1
:10DF68000CDCDFF878C19CF817C0BCEB1E1FA2BF01
:10DF7800DFF888E1D6F800C043F80EC012F803E0D5
:10DF880094F816C00EF00F09E1450BDBDFF84CC121
:10DF98009CF817C0BCEB1E1F04DBD6F800E0574EF8
:10DFA80043F806E0544EB6F90260192E1BDD12F84C
:10DFB80003C094F814E026690CF00F09F1450CDC55
:10DFC800DFF8189199F81590B9EB1C1FDEBFDFF840
:10DFD8002CC1D6F8009043F80C90D25C02F00F0CDC
:10DFE800F4451EDD82E7193680DA12F803C094F88A
:10DFF80016E026690CF00F09F1450CDBDFF8DC9020
:10E0080099F81590B9EB1C1FDEBFDFF8F0C0D6F801
:10E01800009043F80C90D25C02F00F0CF445FFF628
:10E0280065AF94F817E0BEEB121FA2BF334A3668FB
:10E038009E505BE75888000504D404330435B34286
:10E04800F8D122E04AB101EB0C0A06209AFBF0F95C
:10E0580000FB19A001280DDC01E057B9012793F84E
:10E0680001900EEB89003EF829A090F80290C07844
:10E0780003E01746002081468246013125F802ACAC
:10E0880085F800906870C9B2D7E7164A1378013B43
:10E0980013F0FF0308BF06231370114B1B785B07AF
:10E0A80041BFBBF90630A3F57A7303EBC3034FF402
:10E0B8007A7243BF93FBF2F30133DBB20123104AB8
:10E0C80092FBF3F34344A36003B0BDE8F04FF6F7C7
:10E0D80041BD03B0BDE8F08F6B0F0020482700203A
:10E0E800B72D0020A8000020BC0E0020942200209C
:10E0F80088970108B4980108FC120020BA0E002085
:10E10800400D0300064B1B7803F0040303F0FF00E7
:10E118001BB1044B1888C0F3C01000F00100704711
:10E12800B72D0020B01B00202DE9F04F2DED028BFC
:10E1380089B000260693C34B0591B3F90270B3F971
:10E1480000300392002FB8BF7F42002BB8BF5B425C
:10E158009F42B8BF1F46B7F5FA7F8046A8BF4FF465
:10E16800FA770190B3460296B2463446B64D2B88EC
:10E1780099075AD0B34BB54A33F8143032F9142002
:10E18800022013FB0022039B5B429A424FEA4401A0
:10E1980003DB039B9342A8BF1346AD4A31F90290B3
:10E1A800069A32F91420C9EB030303EB0209FFF7BF
:10E1B800A9FF88B107EE909AA64BB8EEE70AB2EE2F
:10E1C800048A185D80EE080A02F06EFD20EE080A47
:10E1D800FDEEC07A17EE909A98F80830642203FB97
:10E1E80009F393FBF2F398F81C206FF0040A0AFB7A
:10E1F80002FA534504DB02EB820A9A45A8BF9A4605
:10E20800954A52F8241009EB010342F210718B422F
:10E21800A8BF0B4691498B42B8BF0B4642F8243041
:10E2280098F8122053431B1302932D8805F003031B
:10E23800012B38D0834B8A4933F914B0019B51F82C
:10E2480024E093F801C0874B33F9140080EAE073A7
:10E25800A3EBE073B3F5206F4FEA840616DC0BEBF3
:10E268008B031A0192FBFCF3042290FBF2F0181ABC
:10E278008644BEF57A5FA8BF4FF47A5E7A4B9E4516
:10E28800ACBF41F824E041F8243002E0002341F813
:10E2980024308B597D2693FBF6F6019BDB7A73437A
:10E2A800402693FBF6F6AA0711D50298C7F5FA722D
:10E2B80007FB0BF907FB06F54FF4FA7102FB0A9905
:10E2C80002FB005599FBF1F395FBF1F505E0EB072F
:10E2D8004DBF029D35465B46534662000492614A33
:10E2E800624932F814E0624AA25C0FFA8EF04FF0ED
:10E2F800040C90FBFCF909FB02F26FF04F0992FB4A
:10E30800F9F931F9142021F814E0821A081D0C31AA
:10E3180050F824E092FBFCF2994451F8243041F87B
:10E3280024E0734498F8501040F8242013444FEA2E
:10E33800840C00EE103A79B14E4B4F48D3ED000AE9
:10E34800CDF81CC0B8EEC00A00EBC400FDF766FBB0
:10E35800DDF81CC0BDEEC00A484A0498125D484961
:10E3680010EE103A5343202293FBF2F309EB050217
:10E37800D21A42524348444A4CF80050434D4CF894
:10E3880002905B424CF80530019B013301930CB9B4
:10E398000124EBE62B4B98F80D70B3F90440059B6C
:10E3A8009B790F335B0063435B112E4C002B4FF0BE
:10E3B8000406B4F9044094FBF6F4294EA3EB0404D4
:10E3C800B8BF5B42322BD6F808E00BDC304B07FBBA
:10E3D80004E7BB42A8BF3B462E4FBB42ACBFB3606D
:10E3E800B76001E00023B36098F803305C432A4B20
:10E3F8001B78032B4FEAA4140CD9B8F84E30B3F5A8
:10E40800FA7F07D25F42BC4203DB9C42A8BF1C468E
:10E4180000E03C46B368946043F34F33B3F5807F24
:10E42800A8BF4FF480736FF0FF06B342B8BF3346FE
:10E43800E618836000238E80AB6009B0BDEC028BC8
:10E44800BDE8F08FFC120020B01B0020AE2D00208C
:10E458003C290020287E010860270020F0D8FFFF13
:10E46800C41B00203C12002080C1FFFF6827002049
:10E47800381C0020F41B0020DC1B00204C1C002052
:10E48800F81B00200C1C0020001C0020181C002079
:10E49800FEFFFF0F020000F04F1C00202DE9F04F97
:10E4A8002DED028B85B081460293AD4B01911C88FE
:10E4B800009204F00204A4B294B1AA4BB3F902404A
:10E4C800B3F90030002CB8BF6442002BB8BF5B42E0
:10E4D8009C42B8BF1C46B4F5007FA8BF4FF4007437
:10E4E800CA4600259F4BA04833F815209F4B50F88B
:10E4F800256033F9153083EAE377A7EBE37711B2A8
:10E50800B7F5206F4FEA450B4FEA41014FEA8508FE
:10E5180011DC042793FBF7F3CB1A1E44B6F57A5F98
:10E52800A8BF4FF47A56924B9E42ACBF40F8256084
:10E5380040F8253002E0002340F8253050F80870F4
:10E548009AF80B309AF80160FF115F43844B1B88DF
:10E558004E439B074FEAA7174FEAA61656D0854B9E
:10E5680033F90B30022112FB0132009B5B429A42C5
:10E5780003DB009B9342A8BF13467F4A3BF9022066
:10E588009A1A029B33F91530D31808EE103AFFF7A0
:10E59800B9FD68B1B8EEC80A784BB2EE048A80EECD
:10E5A800080A585D02F080FB20EE080ABDEEC08A1A
:10E5B800734918EE102A58F8013042F210701344CB
:10E5C8008342A8BF03466F4899F808208342B8BF22
:10E5D800034648F8013018EE101A4A4399F81C10FF
:10E5E80001EB8101D2114842824203DB8A42A8BF73
:10E5F8000A46104699F8122053431B13FF1A361A7D
:10E608006743664303EB672700EB662657485E4976
:10E618003BF800E0495D0FFA8EF34FF0040C93FBD2
:10E62800FCF24A435949A6EBA2163BF901202BF804
:10E6380001E001EB0C0E0C319A1A58F8013092FBEC
:10E64800FCF258F80EC048F801C0634499F850101D
:10E6580048F80E20134400EE103A024669B10390C0
:10E668004B4B4C48D3ED000AB8EEC00A00EBC5008E
:10E67800FDF7D4F9039ABDEEC00A47494748495DFA
:10E6880010EE103A4B435B11F119C91A2BF8001020
:10E69800434948F80160434E48F80670424F5B42D0
:10E6A80048F807300AF1010A0DB901251AE72D4B80
:10E6B800B2F90420B3F90440019B9B790F335B0046
:10E6C80063435B11002B4FF00405274C92FBF5F5D3
:10E6D800A3EB0505B8BF5B42322BD4F808E099F8E4
:10E6E8000D200BDC314B02FB05E29342A8BF134619
:10E6F8002F4A9342ACBFA360A26001E00023A3604D
:10E7080099F8032002FB05F32A4A1278032A4FEAF4
:10E71800A3130CD9B9F84E20B2F5FA7F07D25542A7
:10E72800AB4203DB9342A8BF134600E02B46A26826
:10E738008B6042F34F32B2F5807FA8BF4FF48072EE
:10E748006FF0FF04A242B8BF22469C1800238480C1
:10E75800B260BB6005B0BDEC028BBDE8F08F00BFB6
:10E76800B01B0020FC120020C41B00203C1200201B
:10E7780080C1FFFFAE2D00203C290020287E010823
:10E7880060270020F0D8FFFF381C00207C270020DD
:10E79800F41B0020DC1B00204C1C0020F81B002070
:10E7A800001C00200C1C0020181C0020FEFFFF0F7E
:10E7B800020000F04F1C00202DE9F04F2DED028BD8
:10E7C80087B000260493A14B0292B3F90270B3F903
:10E7D80000300096002FB8BF7F42002BB8BF5B42C5
:10E7E8009F42B8BF1F46B7F5FA7F8346A8BF4FF4CC
:10E7F800FA778246B146B0463446954D2B8899073C
:10E808005AD0022C58D0914B924A33F8143032F92E
:10E818001420022013FB0022029B5B429A424FEA1B
:10E82800440103DB029B9342A8BF13468A4A8A5ECF
:10E838009B1A049A32F91420134408EE103AFFF791
:10E8480061FC68B1B8EEC80A844BB2EE048A80EE67
:10E85800080A185D02F028FA20EE080ABDEEC08A00
:10E8680018EE102A9BF808305343642293FBF2F306
:10E878009BF81C206FF0040808FB02F8434504DBF2
:10E8880002EB82089845A8BF9846754A18EE101AF8
:10E8980052F8243019440B4642F210718B42A8BF3B
:10E8A8000B4670498B42B8BF0B4642F824309BF8A0
:10E8B800122053431B1300932B8803F00302012AF1
:10E8C80001D1022C3FD16848604A30F914006749E9
:10E8D80032F914909AF8016051F824E080EAE07562
:10E8E800A5EBE075B5F5206F4FEA84021EDC022C1B
:10E8F80016D009EB8901090191FBF6F6042190FB7A
:10E90800F1F0361AB644BEF57A5F58495848A8BFA0
:10E918004FF47A5E8645ACBF42F801E0505007E0FC
:10E9280089EAE975A5EBE975642DE2DD00208850D8
:10E938004E497D26525892FBF6F69AF80B20724300
:10E94800402692FBF6F69A0713D5022C11D00098B0
:10E95800C7F5FA7207FB06F507FB09F302FB083354
:10E968004FF4FA7102FB005293FBF1F392FBF1F5BD
:10E9780008E0DB0704D5022C02D0009D434601E0E5
:10E9880035464B4662000392374A32F814E0394A5A
:10E99800A25C0FFA8EF04FF0040C90FBFCF14A4396
:10E9A8006FF04F0192FBF1F23349134431F914200F
:10E9B80021F814E0821A01F10800143150F824E01B
:10E9C800019351F8243041F824E092FBFCF273449F
:10E9D8009BF8501040F8242013444FEA840C00EEB2
:10E9E800103A79B1254B2648D3ED000ACDF814C06A
:10E9F800B8EEC00A00EBC400FDF710F8DDF814C04B
:10EA0800BDEEC00A1F4A2049125D039810EE103A65
:10EA18005343202293FBF2F3019A2A44D21A42521A
:10EA28001A4A01994CF80210194A01344CF802505C
:10EA3800184A5B42032C4CF802300AF1010A7FF4B1
:10EA4800DCAE07B0BDEC028BBDE8F08FFC120020F5
:10EA5800B01B0020AE2D00203C290020287E010894
:10EA680060270020F0D8FFFF3C120020C41B0020C4
:10EA780080C1FFFF381C002090270020F41B0020D5
:10EA8800DC1B00204C1C0020F81B0020001C002070
:10EA98000C1C0020181C00202DE9F04F2DED088BD0
:10EAA80085B009EE902A0193C74B02931A8812F099
:10EAB800020F8246B7EE009A4CD0169BC348DC89F9
:10EAC800B0F900301B1B03F2F31540F2E632954211
:10EAD80003D8002BB8BF5B4201E04FF4FA73B0F9DA
:10EAE8000220121B02F2F31440F2E630844203D8EB
:10EAF800002AB8BF524201E04FF4FA729AF84C006B
:10EB080058B39342B8BF1346C3F5FA7307EE903A69
:10EB18009FEDAF7AF8EEE77A6423C7EE877A93FB26
:10EB2800F0F307EE103A77EEC97AB8EEC77AF0EE4E
:10EB3800498AE7EE878AF7EE006AF5EEC08AF1EEB9
:10EB480010FA0AD4F4EE668AF1EE10FAC8BFF0EEB5
:10EB5800668A04E0F0EE498A01E0DFED9E8A9E4D68
:10EB6800CF1CD0460024022C17F801BFDFF8BC9256
:10EB78004FEA4406B2EE04AA0ED1B9F904209FED7B
:10EB8800977A0BF10A0B02FB0BF307EE903AF8EEBB
:10EB9800E77AC7EE877A66E0F8EE697A9FED8C6AC5
:10EBA80039F91430C7EE867A06EE903A8C4B33F971
:10EBB800143007EE103A19EE903AF8EEE66AB8EE1D
:10EBC800C77A5B42A6EEA77A07EE903AF8EEE77AA4
:10EBD800B4EEE77AF1EE10FA08D4F8EEE97AB4EE7A
:10EBE800E77AF1EE10FAD8BFF0EE477A7D4B9B5FDB
:10EBF80008EE103A019BB8EEC88A33F9143077EE64
:10EC0800C87A08EE103AB8EEC88A37EE888A88EED5
:10EC18000A8AFFF777FA38B1734B185DB0EE480AE5
:10EC280002F042F8B0EE408A029B1A88D10704D558
:10EC3800DAED117A68EE277A15E039F906309FED9A
:10EC4800677A0BF1140B03FB0BF307EE903AF8EE1F
:10EC5800E77A9307C7EE877A42BF9AED127A28EED1
:10EC6800078AE8EE287A614B614A9B5FD8ED08AACB
:10EC78009FED608A07EE103A5F4BB8EEC77AD3ED86
:10EC8800186AA35CE7EE667AD8ED0B6A27EEAA7AD3
:10EC98000AEE903A594BF8EEEAAAD3ED000A67EE6D
:10ECA8002AAA27EEA07ACAEE88AA27EE267AD5EDF8
:10ECB800006AE7EE0A6A9FED527AF4EEC76AF1EE4F
:10ECC80010FAB0EE66AAB0EE48BA09D49FED4D7AB4
:10ECD800F4EE476AF1EE10FAC8BFB0EE47AA01E0B9
:10ECE800B0EE47AA89EE208A474B4FEA840B5B4473
:10ECF80093ED000A85ED00AAC3ED007A37EEC00A4D
:10ED08009AF8501020EE080A31B14048039200EBFF
:10ED1800C400FCF783FE039A135DF0EE087A80EED8
:10ED2800270A08EE103AD8ED0E7AB8EEC88A60EED7
:10ED3800277A27EE880ADFED367A80EE0B8AB4EE62
:10ED4800E78AF1EE10FA09D4DFED327AB4EE678A79
:10ED5800F1EE10FAC8BFB0EE678A01E0B0EE678A3C
:10ED68003AEE8A0A013430EE080A06F053FD2A4BBF
:10ED7800B0F57A7FA8BF4FF47A709842B8BF1846AA
:10ED8800FDEEEAAA254B1AEE902A9853BDEECAAAC0
:10ED9800234BBDEEC88A4BF80320224B1AEE102AEB
:10EDA8004BF80320204B18EE102A032C4BF80320B5
:10EDB80008F1040805F104057FF4D5AE05B0BDECF3
:10EDC800088BBDE8F08F00BFB01B00202C2C002062
:10EDD8000000FA4300000000241C00200000484204
:10EDE800AE2D00203C290020287E01083C1200207E
:10EDF800C01B00200000C84260270020F41B002030
:10EE080000007AC300007A43C4270020DC1B0020DE
:10EE1800000096C30000964318FCFFFFF81B002073
:10EE2800001C00200C1C0020181C0020FC120020D4
:10EE3800044B00221A605A60034B00221A605A6081
:10EE4800704700BF60270020301C002010B50B4C15
:10EE58000123E3704FF48060022384F82030FDF72B
:10EE680041F9074A074B126F1B685178642212FB5D
:10EE78000133636123880133238010BD0C2D0020EA
:10EE8800602700206829002010B54B88DC0641BFA8
:10EE98002F4B14791B6853F8244044BF2D4B43F87B
:10EEA80020404B889B0641BF294B54791B6853F877
:10EEB800244044BF274B43F820404B881C070ED5FD
:10EEC800254B0C781B78B3EB141FA1BF204BD478CB
:10EED8001B6853F82440A4BF1E4B43F820404B88BE
:10EEE8009B070ED51D4B0C781B78B3EB141FDFBFA7
:10EEF800174B54781B6853F82440DCBF154B43F874
:10EF080020404B88DC070FD5154C0B78247803F08C
:10EF18000F03A342DFBF0E4B14781B6853F824403D
:10EF2800DCBF0C4B43F820404B885B070FD50B78B0
:10EF38000C49097803F00F038B42A1BF044B927868
:10EF48001B6853F82220A4BF024B43F8202010BDB1
:10EF580094220020BA0E00205F2700205D270020A1
:10EF68005C2700205E270020254A264826490023E2
:10EF7800F0B5156803700B701C461A462E19768872
:10EF88004EB92F5D3FB9037000230A704B700778A4
:10EF98001C461A460CE0360548BF013204F1040449
:10EFA80003F1010348BFD2B2802CDBB2E6D1EAE715
:10EFB800E0B2B8420CD215F8240006099E4200F0CF
:10EFC8000F00A8BF731C9042A8BF421C0134EFE792
:10EFD8008A704B70C2F3470102F001020A444C1ECA
:10EFE8000A490B480A70C3F3470203F001031344AC
:10EFF80004700849501E084A08701370F0BD00BF1D
:10F008009822002054270020D42700205E270020C3
:10F018005C2700205F2700205D2700202DE9F04FA6
:10F02800C24BDA682DED028B1A61C14A1168D960AA
:10F03800C0490B6843F020030B60BF4B19780129C6
:10F0480090460CBF002201221A70BC4B1A78910717
:10F0580089B040F13D83BA490978042940F23883E0
:10F06800B849097801F0040101F0FF0011B922F054
:10F0780001021A701B78DB0702D408B1FAF7ACF961
:10F08800B149CA78531C052293FBF2F202EB8202C3
:10F098009A1AAE4BCA701B78039392000023AC4CAB
:10F0A800DFF8CCC2DFF8D8925CF8231091FBF9F5B1
:10F0B80004F1080004F1100640F82350A54844F86C
:10F0C800231000FB051142F2107091FBF0F080B2A2
:10F0D80026F813004FF0140E04F1140604F13C0A4C
:10F0E8000EFB036E5AF823605EF802704EF80210A9
:10F0F800F61B314444344AF82310052691FBF6F1F7
:10F1080009FB051144F82310039C012C4FEA830BDB
:10F11800E24605D10238B0F5797F98BF4BF80C105C
:10F128000BB90123BBE7884CD8F80030226D9FED5E
:10F138008A7A8A4E8A4D9B1A07EE903AF8EE677AD9
:10F14800D8F800302365C7EE877A7C4B1B78B7EE7A
:10F15800008AF4EEC87AF1EE10FA58BFF0EE487A59
:10F1680013F00103C4ED157A12D005AA00927D4B65
:10F1780006AA01920CCB9AE80300FAF72BF864214F
:10F18800059A069BB2FBF1F293FBF1F3328000E0A3
:10F1980033802B8094F858306B48002B3BD0D0ED4F
:10F1A800157AC26DDAF80030C8EE276A9B1A026E2B
:10F1B800022507EE103AB8EEC77ADAF8043027EEDF
:10F1C800267A9B1AFDEEC77AB0F9662017EE901AD8
:10F1D80007EE903A644BB8EEE77AD3ED007A67EE23
:10F1E800277A67EEA67AFDEEE77A17EE903A02FAEA
:10F1F80083F3B0F9642093FBF5F302FA81F29BB232
:10F2080092FBF5F292B2A0F86A30A0F86820A0F854
:10F218006630A0F86420012384F85830534BDAF89C
:10F2280004101B88DAF80000474D514E216603F0A0
:10F238003003E065002B00F04B8205F17403009366
:10F2480005F178030193EA6E2B6FF9F7C3FF726833
:10F258002B6F9B1A07EE903A434B326893ED007A76
:10F26800EB6EF8EEE77A9B1AEB67384B67EE877A16
:10F278001B78FDEEE77A012BC5ED207A03D0022B2F
:10F2880000F0DF8024E2D5ED287A3A4BD5ED215AFB
:10F2980095ED255A95ED156A95ED264AD5ED274A3F
:10F2A80035491D68B1EE677ABDEEC77AFDEEE77A9B
:10F2B80017EE10EA17EE90CA0020304A91ED007A56
:10F2C80052F8207007EE907AF8EEE77AA2F114036C
:10F2D80067EEA57A33F81060FDEEE77A283217EE6C
:10F2E800903A9B1B9BB222F810301BB207EE903A63
:10F2F800F8EEE77A3B4467EE857A4400FDEEE77A5C
:10F30800CDED037A07EE903AF8EEE77ABDF80C8077
:10F3180067EE847AA7EE867AFDEEC77A17EE902A12
:10F32800724531DB6245A8BF62462EE0E007002047
:10F3380068290020E81A002082120020EC1A002018
:10F34800F21A0020B72D0020D427002044100020F6
:10F35800D8270020806967FF00007A44661B0020D8
:10F36800681B002084120020AC000020B01B002085
:10F37800F41A00204810002078100020502800209F
:10F3880080969800DB0FC940724607EE902AF8EE87
:10F39800E77A5FED046AC1ED007AFDEEE77A31366F
:10F3A80017EE903A43449AB2AB78D1ED027A07EE61
:10F3B800103AB8EE477A4B684F6027EE267AFB1A68
:10F3C80088EE077AB6B2622E06EE903AF8EEE66A52
:10F3D80037EE067AC6EE866A86EE077A76EEE76A32
:10F3E800E7EE267AC1ED047AC1ED027A0FD964EE10
:10F3F800A77ABA4EFDEEE77A17EE903AB3F5FA6FB0
:10F40800A8BF4FF4FA63B342B8BF334600E0002305
:10F4180013441BB240F6B8329342A8BF1346B04A11
:10F428009342B8BF1346AF4AA352AF4A142303FB13
:10F43800002351F8142B1A60002840F0498101205C
:10F448003BE7AA4BD5F874801F68D4F878903E89BA
:10F45800DFEDA78A4FEA58039E4228BF1E46B5F83B
:10F46800A8301AB29642C3BFD5ED157A9FEDA17A9E
:10F4780067EE877AB6B2C1BFFDEEE77A17EE906AFB
:10F48800F618B6B2C8BFA5F8A860D4F8AC50C5EB5A
:10F4980009052846F9F7E2FE0028D8BF404241F2A4
:10F4A80093129042CCBF0020012088B307EE905AF7
:10F4B800B8EEE70A20EE280AFCF7FDFC07EE908A72
:10F4C800F8EE677A40F6B83320EE270AFDEEC07AE8
:10F4D800CDED037ABDF80C20A4F8B02012B29A4200
:10F4E800A8BF1A467E4B9A42ACBF09EB02034B44B5
:10F4F80048F6A042934203DDA3F50C43A03B04E089
:10F50800002BBCBF03F50C43A033C4F8B43001E0B2
:10F51800C4F8B490D4F8B450C5F50C53283307EEAA
:10F52800903AF8EEE77A67EEA88AB0EE680AFCF738
:10F5380025FD8DED070AB0EE680AFCF7BCFCD4ED9A
:10F54800317AD4ED2E4AD4ED155A94ED2F4A94ED24
:10F55800305A65498DED060AB1EE677ABDEEC77A75
:10F56800FDEEE77A0DF1180E17EE10AA17EE90BA15
:10F578000020614AFEEC016A32F91030DFF88C9104
:10F5880007EE903A07EE106AF8EEE77AB8EEC77A17
:10F598003C32D6EE877A4FEA400CFDEEE77ACDEDA5
:10F5A800037ABDF90C30B3F57A7FA8BF4FF47A73AC
:10F5B8004B45B8BF4B461FFA83F922F810900FFA53
:10F5C80089F207EE902AF8EEE77A27EEA47ABDEEE4
:10F5D800C77A8DED037A27EE847AD1ED007ABDF8EB
:10F5E8000C90E7EE257AFDEEE77A17EE902A524561
:10F5F80003DB5A45A8BF5A4600E0524607EE902A58
:10F60800F8EEE77A9FED3D6AC1ED007ABA7891EDA0
:10F61800027A06EE902AF8EE666A4A684B6066EE51
:10F62800866A9A1AC8EE266A143106EE102AB8EECF
:10F63800C66A76EEA56A86EE256AC5EEA66A36EE35
:10F64800476AA6EE867A01ED017A01ED037A25EE86
:10F65800077ABDEEC77A17EE103ABDEEE77A4B444B
:10F6680017EE102A13441BB240F6B8329342A8BFD3
:10F6780013461B4A9342B8BF13461A4A2CF8023065
:10F688001F4A142303FB0023C3ED007A08B90120A5
:10F698006FE73B7923B1642395FBF3F5194B1D8084
:10F6A8003B8898450DD9D4F8AC30A06FC01AF9F74B
:10F6B800D5FD80EAE072A2EBE07242F210739A4242
:10F6C80006DD114B01221A700E4BB4F8C8201A80BF
:10F6D80009B0BDEC028BBDE8F08F00BF30F8FFFF2A
:10F6E80048F4FFFFCC100020A01000204810002094
:10F6F800D30237390000C8423C280020DB0FC9403C
:10F7080078100020401000204410002018FCFFFF53
:10F7180082B01B4B1B4A8DF807101968106860B33C
:10F728001268052A29D1184A106810BB9DF80810DC
:10F738009DF8073043EA012314490B80144B1968DC
:10F74800144B89B20B445B001968012119601368D6
:10F758000B441360104A136823F4E04323F040037A
:10F768009BB283F0300343F4004343F080031360FB
:10F7780003E01A68521A312AD5D902B0704700BF7F
:10F7880068290020942D0020A028002080610040D6
:10F79800505C00400A300020045C0040014B58686F
:10F7A800C0B27047A02800200120704770477047FA
:10F7B80020B9034B1B6808221A827047014870471A
:10F7C8001C200020B000002020B9034B1B68082231
:10F7D8001A827047014870471C200020B0000020A2
:10F7E80021B901288CBF02200020704702207047F1
:10F7F80010B5094B1A68D378042B0BD8074C518ADB
:10F80800DB00234418B99B895B1A138210BD9B68DF
:10F81800581810BD002010BD1C200020B00000208A
:10F82800054B1968054B4A8A18B99B8D9B1A0B82A0
:10F838007047986A104470471C200020B0000020D0
:10F84800054B1968054B4A8A18B99B8E9B1A0B827F
:10F858007047186B104470471C200020B00000202F
:10F86800074B1B681B7803F07F03212B06D100F0A0
:10F87800DF00022814BF02200020704702207047D2
:10F888001C200020212810B508D1114B1B681B78BB
:10F8980003F07F03212B10D0022010BD2028FBD1BC
:10F8A8000B4B0C4A1B6810701B7803F07F03212B4D
:10F8B800094B18BF00230BB9EEE7084B044A12683E
:10F8C80000249361548220469847204610BD00BF0B
:10F8D8001C200020BB2D0020B9F70008D1F7000834
:10F8E8007047034B1A78202A04BF00221A70704709
:10F8F800BB2D0020014B04221A607047942D002074
:10F90800034B9B7A13B1034B05221A60704700BF63
:10F9180000220020942D0020F7B51C4B5A681D4684
:10F928000AB95C6800E00124187A0021CAB2A24230
:10F9380001F1010107D202AE2F1816443A44527A57
:10F9480006F8042CF2E75A68121B5A601A7A5D68A6
:10F9580022441A729DB903204021FAF72DF80C4A67
:10F96800136823F4804323F070039BB283F440535D
:10F9780043F4004343F080031360044B1D72002CD2
:10F98800CBD09DF8040003B0F0BD00BFA028002034
:10F998000C5C00402DE9F843664B674E1B68DFF8A6
:10F9A800B881664A00254FF0C0099D7283F8099016
:10F9B800DD723560D8F8003023F4EC4323F070038F
:10F9C80043F400739BB2C8F80030D8F8003023F431
:10F9D800E04323F040039BB248F2800483F0100315
:10F9E8002343C8F80030336812FA83F35B004027DA
:10F9F8001A681F6033689BB203F1005303F5405344
:10FA08005B0028461A6880221A60D8F8003023F470
:10FA1800F8731B051B0D2343C8F80030484B93F8B7
:10FA28002C10F9F7C9FFD8F80030464A464923F4A4
:10FA3800804323F070039BB283F440532343C8F8F8
:10FA48000030136823F4EC4323F070039BB2136077
:10FA5800336811FA83F35B0003201968C3F8009038
:10FA680013683A4923F4E04323F040039BB283F040
:10FA7800200323431360136823F4804323F07003A7
:10FA880023439BB21360536823F4EC4323F07003C1
:10FA980043F4C0639BB25360336811FA83F35B008D
:10FAA80019684FF480711960536823F4804323F078
:10FAB800700323439BB25360536823F4E04323F05D
:10FAC80040039BB283F0200323435360D8F80C30E3
:10FAD8001F4A23F4EC4323F070039BB2C8F80C30A0
:10FAE800336812FA83F35B0039461A684FF4887258
:10FAF8001A60F9F761FFD8F80C3023F4804323F03B
:10FB080070039BB283F440532343C8F80C30D8F8F1
:10FB18000C3023F4E04323F040031C43A4B2C8F89C
:10FB28000C402846F9F7BCFE0A4B01221A60BDE8D2
:10FB3800F88300BF1C200020505C004004300020E7
:10FB480020000020045C0040083000201030002015
:10FB58001C300020942D0020005C0040134A144BF8
:10FB680050681B68181810B5146808D01149082285
:10FB7800F7F7A1FC204610490422F7F79CFC0F4B2D
:10FB88001A68002393720E4A012111600D4913600F
:10FB98004FF4E0500B6010600B480B604FF4364197
:10FBA800A0F84A101160094A136010BDB0F7FF1F92
:10FBB800ACF7FF1FEA000020FA0000201C200020FC
:10FBC800405C0040445C0040A0280020942D0020A8
:10FBD800104B93F84C2013B51C46C2B90E4B1B684A
:10FBE800ABB11A681AB10D49486902434A619A884B
:10FBF800ADF8042002228DF807209868002201A998
:10FC08008DF80620F5F784F8012384F84C3002B00B
:10FC180010BD00BFA02800200803002000100240EB
:10FC28000A4B10B519684FF6FB720A401A60084A69
:10FC3800927A1C46074B0AB1052200E001221A609D
:10FC480000F08AFE4FF43643236010BD405C00404C
:10FC580000220020942D002007B5064B0093064B88
:10FC680001930649064A074B0748FCF7F6F803B024
:10FC78005DF804FB18990108ED9801087EA60108B3
:10FC880088A601080C9901085DA6010808B5037843
:10FC980033B90C4B0C481978BDE80840FCF7DDB8BF
:10FCA80005F044FC02280CD8064B1870074B0C22B0
:10FCB80002FB0030064B06301860FCF7EFFA0548E7
:10FCC800E5E708BDF02800208FA60108A41A002047
:10FCD8007C1200200B9C010808B503783BB90B4B3C
:10FCE8000B4893F8A417BDE80840FCF7B6B805F030
:10FCF8001DFC022808D8054B83F8A407FCF734FA42
:10FD0800FCF7F0FA0348E8E708BD00BF0413002039
:10FD180093A601080B9C010838B5037803BB214B57
:10FD28001B6801330F2B07D81F490C2202FB031253
:10FD38001C4695682DBB00E01C4601340F2C01DDE4
:10FD4800002400E005D818490C2202FB041295682B
:10FD5800BDB99C42F1D11548BDE83840FCF77DB8E3
:10FD680005F0E4FB0F28044605D80F4A0C2303FBD3
:10FD780000239D682DB921460D48BDE83840FCF7A1
:10FD88006CB8084B1C60F8F78DF821462A460948DC
:10FD9800FCF763F80C235C43034B185DBDE838405F
:10FDA800F8F798B804010020E4870108A0A6010824
:10FDB800B6A60108CEA6010873B5037813B9FAF7F9
:10FDC800BFFA3DE01F4901AA05F011FC00240146D5
:10FDD8002646254699B134B1012C08D1084605F0CC
:10FDE800A5FB064603E0084605F0A0FB05461549B5
:10FDF800002001AA05F0FBFB01340146EAE70B2DC0
:10FE080002D911480C220BE0022C10D1A6F57A7306
:10FE1800B3F57A7F07D90D484FF47A714FF4FA6237
:10FE2800FAF70BFA0CE00A4B03EB45035E80084B2C
:10FE3800084803EB45032946B3F90220FCF70DF8FF
:10FE480002B070BD99A00108649E0108FCA30108D6
:10FE5800F0280020E5A6010838B50D4C2368834238
:10FE6800054606D1FAF739FD204600214C2205F057
:10FE7800C2FAE36CAB4209D12846FAF72EFD0548D1
:10FE880000214C22BDE8384005F0B5BA38BD00BFA6
:10FE98002420002070200020034B1A68D379591CB5
:10FEA8001344D171187A7047901B002010B5FFF7E2
:10FEB800F3FF84B2FFF7F0FF04EB002080B210BD1F
:10FEC80010B5FFF7F3FF0446FFF7F0FF04EB00401F
:10FED80010BD064B10B5044621461868F8F796F889
:10FEE800034B1B6898796040987110BD941B0020E3
:10FEF800901B002038B5044624200D46FFF7E9FF83
:10FF08004D20FFF7E6FF002C084C14BF21203E20AF
:10FF1800FFF7DFFF2368002228469A71FFF7D9FF11
:10FF2800236893F84900BDE83840D2E7901B0020C9
:10FF380001460020DEE710B50446C0B2FFF7C9FF4E
:10FF4800200ABDE81040C4E710B5044680B2FFF7A8
:10FF5800F2FF200CBDE81040EDE737B582888368D2
:10FF6800044610060D4641BF2B4991F8A4174FF4DB
:10FF7800CC7000FB0133D10544BF2849097802F051
:10FF88003F0244BF01EB410103EB8103042A12D075
:10FF980006D8012A0DD0022A32D193F9001030E098
:10FFA800102A0AD0202A0AD0082A29D1B3F9001029
:10FFB80027E0197825E0198823E0196821E093EDF6
:10FFC800000A6846FBF7DEFD01461548FBF745FFCA
:10FFD80005B3D4ED037A6846B8EEE70AFBF7D2FD1D
:10FFE80001461048FBF739FF94ED040A6846B8EE5D
:08FFF800C00AFBF7C7FD01463A
:020000040801F1
:100000000A48FBF72EFF09E000210948FBF729FF0A
:1000100025B10848E1682269FBF723FF03B030BD32
:1000200004130020F0280020A49F01089D9F0108D0
:10003000F8A60108F4A60108024B0146D869F7F7B3
:10004000E9BF00BFF028002010B5441E14F8011FBE
:1000500021B1034BD869F7F7DDFFF7E710BD00BF0B
:10006000F0280020F7B52B492B4B08782B4D1C6846
:100070002B4B05EB80001A882A4BD0F8C0101B7858
:10008000294800914FF47A71B4FBF1F1FBF7E9FED6
:1000900026484821FBF7E5FE254B1F680026F3B2F2
:1000A00005EB8302D2F8D010E9B101249C403C4218
:1000B00017D0220715D01F4AD25C0B2000FB032368
:1000C000164A1D4802EB8303D3F8F020FBF7C9FE64
:1000D000022C06D1194B93F8281011B11848FBF7E0
:1000E000C0FE0136DBE71748FFF7AEFF164B174897
:1000F0001A68174B9A420CBF164B174B1A88174BAE
:10010000198892B24FF4FA6303B0BDE8F040FBF7F0
:10011000A8BE00BF381B002068290020E487010822
:10012000D81A002008010020FBA601083EA70108FC
:10013000E81A0020100100204EA70108F028002036
:1001400056A701089EA70108141200205AA701080B
:1001500000540040181200201A1200201012002033
:100160002DE9F0410024804625460F4EA75941460F
:10017000384605F0C7F958B139460C48FBF771FE0F
:1001800030190021FFF7EDFE0948FFF75DFF01354B
:10019000143440F66C439C42E7D11DB90548BDE8D4
:1001A000F04151E7BDE8F081848901081BA00108F6
:1001B0009EA70108BB9E01082DE9F04F2DED028B93
:1001C00083B0054605F05FF9064620B1012818D135
:1001D0002B782A2B15D15C48FFF736FF00245B4DA6
:1001E0005B486159FBF73DFE28193146FFF7B9FE20
:1001F0005848FFF729FF143440F66C439C42EED177
:100200009CE028463D2105F030F9002800F08F8061
:100210000346994613F8012D202AFAD0441C2046A3
:1002200005F088F980462046FBF726FCC5EB090956
:10023000B0EE408A0026DFF834A1142202FB06F457
:100240000AF5D07B54F80B70384605F01CF90346CC
:100250001A4628463946019305F01EF9019B0028ED
:100260005BD15FFA89F29A4257D10AEB0402D2EDD0
:100270006B7AF8EEE77A0BEB0405B4EEE78AF1EE61
:1002800010FA48DBD2ED6C7AF8EEE77AB4EEE78A42
:10029000F1EE10FA3FD8B2F8A431D2F8A82113F049
:1002A000200F08BF08EE108A1C0641BF2A4991F8AA
:1002B000A4174FF4CC7404FB0122D90544BF27498D
:1002C000097803F03F0344BF01EB410102EB8102D7
:1002D000042B18EE100A0BD004D8013B012B0ED8CA
:1002E00010700CE0102B05D0202B06D0082B06D167
:1002F000108004E082ED008A01E082ED008A394638
:100300001748FBF7AEFD2846002103B0BDEC028B79
:10031000BDE8F04F25E6134803E001369F2E8AD151
:10032000114803B0BDEC028BBDE8F04F8CE62846C7
:1003300003B0BDEC028BBDE8F04F11E703B0BDEC9C
:10034000028BBDE8F08F00BF8CA7010884890108EB
:100350001BA001089EA7010804130020F02800201C
:10036000A1A70108ACA70108BB9E0108E48701080A
:1003700070B50546284605F086F8064658B9194B6B
:1003800019485A79194B03EB8203BDE87040D3F842
:10039000081EFBF766BD28461549324605F07CF875
:1003A00060B91448144CFFF74FFE54F8041F19B1FC
:1003B0001248FBF756FDF8E7114805E00024114B01
:1003C00053F8241019B91048BDE870403CE628469F
:1003D000324605F061F801340028F0D1014B0B4D95
:1003E0005C71C7E704130020CCA70108E48701086B
:1003F000BB9F0108D8A70108EC950108B79F010829
:100400009EA70108F0950108BB9E01080B9C0108FE
:1004100008B50748FFF718FE064BD869FAF756FAF1
:10042000F7F758FFFBF77AFE034B044ADA6008BD82
:10043000EBA70108F028002000ED00E00400FA0519
:1004400008B50548FFF700FE00F036F8FBF790FE10
:10045000BDE80840DCE700BFF7A7010808B504487D
:10046000FFF7F2FDFBF784FEBDE80840D0E700BFD0
:100470000DA801080E4B1A786A2A16D15A88B2F5CF
:10048000FA6F12D11A79BE2A0FD193F8CD27EF2A2D
:100490004FF000000BD113F8012B5040054A934256
:1004A000F9D1B0FA80F040097047002070477047DA
:1004B00000F80308D0FF03082DE9F04F2DED028B63
:1004C000EB4D00214FF4FA6285B0284604F097FF07
:1004D000E84B05F537721A60E74A00231370E74AC4
:1004E00005F2A67111606A222A7003226A714FF424
:1004F0008072AA604FF41672A5F86221FA22A5F85C
:100500006421BC22A5F860214FF4FA722021A5F8DD
:100510006A21012285F85E2185F8661185F87A2125
:100520006E2185F88221052285F8781185F81B2235
:100530000A2140F2DC5285F87911A5F894212B218B
:1005400040F24C4285F87B11A5F89621212140F21A
:100550006C7285F87C11A5F89821232140F2753240
:1005600085F87D11A5F89A214FF4C87140F6430231
:10057000A5F89C21A5F87E112A462C46032BCCBF5A
:100580000121002103F1010382F89E1114BF1E21F5
:100590007521122B82F89F1102F10202EED14FF465
:1005A000FA63A4F8C431A4F8C831A4F8CC31A4F893
:1005B000D03140F27E41052340F27E5684F8DE3190
:1005C000A4F84011C82340F23A71A4F8486140F2FF
:1005D000EA5601274FF47A794FF0320BA4F8E23152
:1005E000A4F842114FF4C87340F2DC51A4F84A61F8
:1005F000DFF880A2A4F8E63140F2B4561E2019229A
:10060000A4F84611A4F84C61A4F8C291A4F8C691CC
:10061000A4F8CA91A4F8CE9184F8E07184F8E1714D
:1006200084F8E471A4F84491A4F84EB184F89101DF
:10063000039084F8DF2101920291A4F8503184F8EC
:10064000DD7184F8EA71A4F852B184F8ED71F9F71C
:1006500031F8DAF800300398677300262673D872F1
:1006600018735520019AD8700F205871DA71222022
:10067000212298715A740E2053224FF0170E1874CD
:10068000DA7635200A224FF0280883F815E083F83F
:1006900016E098764FF02D0E5A209A7401924FF082
:1006A000780C642283F80DE018721A7783F80AC078
:1006B0001E7083F8018083F80280DE7583F804B031
:1006C0009E731E76DE735E7683F8098083F814E0ED
:1006D0004FF4FA7EA3F84EE0DFF8C0E1C3F838E04B
:1006E000C3F83CE0DFF8B8E1C3F828E0DFF8B4E194
:1006F000C3F834E0DFF8B0C1DFF8B0E19FED608A05
:10070000C3F82CC0C3F830C0C3F848E0F7EE087A4D
:10071000DFF89CC102999F774FF04B0E83F8508011
:10072000C3ED087AC3ED097A83ED108AC3F844C09B
:1007300083F84CE084F8A607A4F8B0174120042100
:1007400084F8A70784F8A8B784F8A96784F8AD6788
:1007500084F8AE6784F8AA6784F8AB6784F8AC675E
:1007600083F85C101521A3F85860A3F85A60A3F829
:100770005660C3F860C083F8648083F8658083F8AE
:1007800068104049D966404919674049596783F85C
:1007900078703F48F8F7D4FFDAF80030019A83F810
:1007A00011614FF44871A3F8161183F8126183F8B0
:1007B000138183F8147183F8186184F8D421C82256
:1007C00084F8D5216422A4F8D69184F8D861A4F8DD
:1007D000DA2119460E2202FB06326FF0170082F86A
:1007E0001901032082F81A016FF02F0082F81B0113
:1007F000072082F81C016FF0230082F81D010520FC
:1008000082F81E0101365A2081F8200181F8210169
:100810006422FF20082E81F81F2181F8220101F1B6
:100820000E01D7D1002183F88911C821A3F88A11BC
:10083000142183F88C11A3F890211E214FF4967295
:1008400083F88D11A3F892210121282283F88E11BB
:10085000A3F894210F4B18EE102A45F8102F9D4253
:10086000F9D10D480021402204F0C9FD002321E008
:100870000413002058120020F02800207C120020D1
:10088000000000009A99193FF6287C3F3D0A773F07
:10089000BFB20108C4130020A01500208FC2F53C90
:1008A000000060406666663FCDCCCC3E0000404014
:1008B0000000A040274D284C59591A1904330868E4
:1008C000C2F89C02382BF5D104F507700021802274
:1008D00004F095FD05F13801702204F5077004F06D
:1008E00083FDFEF745FBDAF8006000230125314661
:1008F00004F274404FF4CC7284F8CC3784F8CA57B1
:1009000084F8CB5704F070FD04F20C6031464FF4CC
:10091000CC7204F069FD114B1B681A68C4F8B22749
:100920005A68C4F8B6279A68C4F8BA271A68C4F88F
:10093000BE275A68C4F8C2279A68C4F8C62702239B
:1009400084F8C85484F8603605B0BDEC028BBDE86D
:10095000F08F00BFB8960108041300207C1200201D
:100960001549D1F8883043F47003C1F88830134B2F
:100970001A6842F001021A605868114A02405A602F
:100980001A6822F0847222F480321A601A6822F403
:1009900080221A605A6822F4FE025A60DA6A22F053
:1009A0000F02DA62186B074A02401A6300229A604B
:1009B0004FF000638B60704700ED00E000100240D4
:1009C0000CC07FF8CCFC00FF38B5094B93F8CC572E
:1009D00065B9084C2068F9F784FF074B25601B7840
:1009E000022B03D1BDE83840F8F723BE38BD00BF65
:1009F00004130020902900208C290020044B93F838
:100A0000CC371BB9034B1868F7F7F8BA00207047CA
:100A1000041300209029002038B5054604462046DE
:100A200014F8011B21B1034B1868F7F7F3FAF6E746
:100A3000401B38BD902900200FB407B504AB064910
:100A400053F8042B01930020FBF71EF903B05DF867
:100A500004EB04B0704700BFC70B0108024B01460E
:100A60001868F7F7D7BA00BF90290020F8B5011F22
:100A700006460023083051F8042F02F120043F2CD1
:100A80003AD802F108040F2C06D80232032A04D9FE
:100A9000002B08BF012300E002238142EBD1012B90
:100AA00030680ED0022B1AD0736803F003039B004A
:100AB00000F0030043EA0010B36803F00303184397
:100AC00017E000F00F0040F04000FFF7C7FFB068EC
:100AD000736800F00F0040EA0310C0B209E000F0B4
:100AE0003F0040F08000FFF7B9FF3079FFF7B6FF15
:100AF000307ABDE8F840B1E706F10C0734463A46D3
:100B0000002552F8043D03F18001FF294FEA8505D5
:100B100010D903F50041B1F5803F02D245F001053F
:100B200008E003F50003B3F1807F34BF45F0020510
:100B300045F00305B242E4D165F03F00C0B2FFF7D3
:100B40008DFF05F00303022B207807D0032B0CD078
:100B5000012B13D1FFF782FF60780FE0FFF77EFFD4
:100B60006078FFF77BFFA07808E0FFF777FF6078F9
:100B7000FFF774FFA078FFF771FFE0780434FFF708
:100B80006DFFBC424FEAA505DBD1F8BD10B50446A8
:100B9000C0B2FFF763FFC4F30720BDE810405DE774
:100BA00010B504467F2C06D964F07F00C0B2FFF771
:100BB00055FFE409F6E7E0B2BDE810404EE7430018
:100BC00083EAE070ECE7084648E700BF40F2E9330B
:100BD0000F4A1289920704D4013B9BB2002BF7D134
:100BE0000BE00C4A40F2E933107009490989C90742
:100BF0000AD4013B9BB2002BF7D1074A138801337B
:100C00009BB21380FF2070471078C0B2704700BFBE
:100C1000003001400C300140342900200C4B0D49BC
:100C2000DA684378D243C2F30222C2F1040293404D
:100C300002781B010A44DBB282F8003303780122F8
:100C4000580903F01F0302FA03F341F820307047FC
:100C500000ED00E000E100E073B50546002100680A
:100C60000122FCF7F5FC2A6813889BB243F00103CC
:100C70001380EB7A8DF804300124002601A88DF84A
:100C800005408DF806608DF80740FFF7C7FFEB7A47
:100C90001B2B0BD1192301A88DF804308DF80540CA
:100CA0008DF806608DF80740FFF7B8FF02B070BD01
:100CB000F0B5BE4CA3782DED028B013B012B85B026
:100CC00000F26F81E578854240F06B812379022B39
:100CD00000F06781B64B5B5D6371A3796D00F2EE46
:100CE000048A1BB16319B3F9083009E06319D4ED24
:100CF000037AB3F90830F1EE677AC4ED037A5B4208
:100D000008EE103A2369A94EB8EEC88A1A0388EE95
:100D1000288A35D5D6ED037AFDEEE77A28EE280A43
:100D200017EE903AD6ED057A8DF80A30FDEEE77AA7
:100D300017EE903A8DF80B3004F0B6FDFCEEC07A59
:100D400096ED060A17EE903A20EE280AADF8083024
:100D500004F0AAFDFCEEC07A96ED070A17EE903A71
:100D600020EE280AADF80C3004F09EFDFCEEC07AAF
:100D70000C2017EE903A02A9ADF80E30FAF7C0F940
:100D8000D4ED077A894BF5EE407AF1EE10FA60D196
:100D9000D3ED067AB4EEE78AF1EE10FA04DDDA68F4
:100DA00083ED068A5A61E8E0F5EEC07AF1EE10FABA
:100DB00040F3E38093F8202042B1022A00F2DD8064
:100DC0005A6B83ED078AFA329A63D6E0D3ED037A41
:100DD00038EE678AF7EE007AB4EEE78AF1EE10FAA1
:100DE000ACBF01210021D3ED0A7A69B19FED717A80
:100DF00027EE877ADFED707AB4EEE77AF1EE10FA3B
:100E000058BFF0EE477A03E09FED6C7A67EE877A81
:100E1000C3ED0A7A2369654A1B0311D58DF80810C2
:100E20005379116B0B440B205A788DF80920DA7A2C
:100E30008DF80A205B7D8DF80B3002A9FAF760F976
:100E40000123226B84F82030637913440022DA7284
:100E500091E0B4EEE78AF1EE10FA48BF83ED078A1D
:100E6000A16B636B94ED067AD4ED076A591AC943F6
:100E7000C90F77EE667A59B9B7EE006AF4EEC67A12
:100E8000F1EE10FA79DDB4EEE68AF1EE10FA74DDD7
:100E9000D4ED056A454BB4EEE67AF1EE10FACCBF1C
:100EA0000126002666B1D3ED097A9FED427A67EEFE
:100EB000877A9FED427AC3ED097AD3ED0B7A0AE087
:100EC000B0EE007AF4EEC77AF1EE10FA08DDD3ED59
:100ED0000B7A9FED387A67EE877AC3ED0B7A07E0DD
:100EE000D3ED097A9FED357A67EE877AC3ED097AFB
:100EF000D4ED097A206B627967EEA87A1044FCEE93
:100F0000E77ACDED017A9DF804304370D4ED0B7A89
:100F10002769FCEEE77A3F03CDED017A9DF80420C6
:100F200042750ED546EA41018DF808108DF809305A
:100F3000C37A8DF80A300B2002A98DF80B20FAF73E
:100F4000DFF894F82020194B022A11D1D3ED0A7A48
:100F50009FED1B7A196B67EE877A002283F82020B9
:100F6000FCEEE77A5A7917EE903A0A44D37202E01F
:100F7000022283F82020F8F79FFAA2790B4B0AB1DE
:100F8000104A00E0104ADA602544D4ED037AB5F93E
:100F9000083000EE103AB8EEC00A80EE280A37EEAC
:100FA000C00A05B0BDEC028BF0BD00BF34290020A3
:100FB00090970108EC51783F6F12833A0AD7833F2C
:100FC00000007A440000A0410000A0C12B4BF0B506
:100FD0002B4D1E6805F110002F78F3192C46597817
:100FE00001F00401013501F0FF0219B18542F3D18E
:100FF0000020F0BD224D631B022B0ADD1AB102EB6B
:1010000082025200D2B215F8013B303B1A44D2B2F0
:10101000F1E70021AC420AD919B101EB8101490085
:10102000C9B215F8013B303B1944C9B2F2E72E2F83
:1010300016D10134042000232578771903EB8303AC
:101040007F785B007F079BB244BF303D5B1900F1A6
:10105000FF3044BF01349BB210F0FF00ECD100E040
:10106000002308484143642000FB03130620B3FB20
:10107000F0F3054800FB0230F0BD00BF180100206E
:101080007029002040420F008096980030B5002360
:101090001A4610498C1894F83C40BCB12E2C06D14D
:1010A000013298B18C180444002584F83C50114456
:1010B0000A2491F83C106343A1F13004092C9CBF31
:1010C000303B5B180E2A03D80132E2E7184630BDE8
:1010D000002030BD342900200EB40FB5074901901F
:1010E00006AB01A8064A0393FAF7CEFD019B002246
:1010F0001A7004B05DF804EB03B07047B9B900088A
:10110000AFA001082DE9F04FAE490B7813F0010FA5
:1011100087B003F0040200F07981002A40F0838157
:10112000A948066816F0806640F07D81980700F1B6
:101130006D8143F004030B70A44BA54F1A88A54B97
:101140001A803B681B0340F11D81A34B80201E7059
:10115000F8F76EFB08B1FEF783FEA04C2578012D51
:1011600040F010819E4B93F8CA1721B193F8CB271A
:101170000AB1914203D3012283F8CA2711E09646AF
:101180000846BEF1000F06D090FBFEFC0EFB1C0CC7
:101190007046E646F5E791FBF0F183F8CA1792FB3B
:1011A000F0F283F8CB2793F8CC271AB18C4A0021B0
:1011B00082F8CC17626893F8CC9702EBC20241F632
:1011C00069018A4284BF40F2E241B2FBF1F28549F3
:1011D0008CBFD2B204220A70B9F1000F1FD1802057
:1011E000F9F7BEFD8046D0B18021F9F793FD98F85C
:1011F00006207D4B207253F8223098F90000DFF86A
:10120000DC81B3F5613F0CBF0222002202218DE890
:10121000060080214A46F9F77FFBE06008B9002309
:10122000AFE0494608F11000142204F0E8F808F194
:101230003003C8F8243008F1A403C8F8283008F5B2
:101240008C73C8F82C30694B39681B88A8F88C312E
:10125000634B93F8902193F8CA8793F882A1002AF0
:10126000634A10685A7993F8CB37A2F1190EC1F38B
:10127000C03C18BF4FF0010CDEF1000747EB0E0732
:10128000012A14BF3A4601225A4F049298455A4BFC
:10129000D7F800E01B78039301F40069C0F3800BDA
:1012A000C1F34001C0F3C0002CBF4FF000084FF065
:1012B000010805976A1ED2B2531E132B3DD8DFE8F2
:1012C00003F00C0C0C0C0C0C0C0C0AACAE292B3FD4
:1012D00037121212393F049BA2E0039B9342B4BF22
:1012E0000023012328E09EF80030022B0BD10EEBE7
:1012F000820353ED027AF5EE407AF1EE10FA14BF54
:101300000123002318E00EEB02035B79003318BFC2
:10131000012311E00B4683E0B9F1000F04D00AF17C
:10132000FF377B427B4100E04B4603F0010377E04F
:10133000634675E0434673E013B1012393401E43B7
:10134000142D02D80135EDB2B4E7059BC4F89061C5
:10135000186819217930F6F70DFD0023C4F898318B
:10136000A4F89C31A4F89E31C4F8A831234BD4F8DA
:10137000A4211B68C4F8AC3184F89401C4F8A021FE
:10138000022323701D4B164A1B6892F8DE214FF48E
:101390007A7101FB02331A4A13600D4B1B681A065F
:1013A00009D5184B1B789B0705D5174B1B78042BC9
:1013B00001D9062000E0052007B0BDE8F04FF6F7A0
:1013C0008DBD00BFB72D00201C120020F41200209C
:1013D0004429002042100020C5200020842900203C
:1013E00004130020140100202C7E01083821002065
:1013F000E81A0020581200204F1C00206829002005
:10140000F40F0020EC1A0020F21A00205AB9012033
:1014100007B0BDE8F04FF6F787BD034600E05B4636
:10142000002B8AD18EE707B0BDE8F08F10B5154AC2
:101430001378590725D523F004031370124B1B684A
:101440001B0319D5114C2378A3F10802012A0BD8EC
:10145000FF200021F9F754FE0D4B1B68C4F8AC3196
:10146000FFF7CCFA0A2306E0012B05D90A2B03D09B
:10147000FFF7AAFA012323700420BDE81040F6F715
:101480002DBD10BDB72D0020442900208429002047
:101490006829002003788B4286BF024B33F8110085
:1014A00000207047382B002070B5002213462349D6
:1014B00014180C44247E83EA0423082413F4004FF8
:1014C0004FEA430318BF83F4815304F1FF3418BF7C
:1014D00083F0010314F0FF049BB2EFD10132192A0B
:1014E000E5D100F1190200F11A050A440D44167EF7
:1014F0002A7E02EB062292B29A421ED10F4B93F83B
:101500003950E2B2AA4215D2431C03EB4203DBB2CC
:10151000CA1801330B44127E1B7E03EB02239BB2DD
:101520004FF4AF6253431B1303F5487321F8143093
:101530000134E6E7012381F83A3070BD382B0020F2
:1015400003788B420BD9074B1A78074B8900194453
:10155000C86B02B1400800F5777080B27047002078
:10156000704700BFC4200020382B002007299DBFF2
:10157000034B03EB8101B1F86C000020704700BF02
:10158000382B0020034B03EB4101B1F88C00C0085D
:10159000704700BF382B00200A4BDFED0B7A03EBBE
:1015A000810191ED2B7AB8EE477AF6EE046AE7EE08
:1015B000267A82B0FCEEE77ACDED017ABDF8040020
:1015C00002B07047382B002000005C44024B03EB54
:1015D0004101B1F8F4007047382B0020024B03EBB7
:1015E0004101B1F818017047382B0020024B03EB82
:1015F0004101B1F818017047382B002000207047D6
:1016000070B5334C0546F6F70BFCD4F83031C4F80E
:101610003001C31AB3F5FA5FC4F8343182BF002336
:1016200084F8383184F8393194F838312BB9A12D48
:1016300002BF274A012182F8391194F83911244A4E
:1016400029B1D118EDB201330D7682F8383194F812
:10165000385194F83A31AB4239D11D4B93F83B31B4
:10166000052B02D0062B03D02CE00020FFF71CFF37
:10167000637E1E2B26D100200246C1B26B1E99420A
:1016800019DA21440B7E0821DBB283EA0206F60751
:1016900044BF83F01803C3F3460301F1FF3154BF85
:1016A0005B0843F0800311F0FF01C2F34702ECD165
:1016B00001301A46E1E723441B7E9A4202D10320FF
:1016C000FFF7F2FE002384F8393184F8383170BD19
:1016D000382B002010B50446F6F7A2FB0F4BD3F8C9
:1016E0003C21C3F83C01821A41F288318A42C3F896
:1016F000402184BF002283F8442193F84421074904
:1017000013440F2AE4B218BF013283F8454112BFD7
:1017100081F84421012381F8553110BD382B002078
:1017200010B50446F6F77CFB0F4BD3F85821C3F8ED
:101730005801821A41F288318A42C3F85C2184BF81
:10174000002283F8602193F8602107491344142A8A
:1017500018BF013283F8614112BF81F86021012373
:1017600081F8763110BD00BF382B002038B5044613
:10177000F6F756FB274A2749D2F87831C2F87801A4
:10178000C31AB3F57A6F84BF002382F87C3192F8D4
:101790007C3133B9A82C3BD181F87D31A1F87E3161
:1017A00006E0022B02D181F8804101E0242B02D80F
:1017B000D11881F8814192F88011164D0133023120
:1017C000DBB249008B4282F87C3118DAB5F87E3101
:1017D000E0B283EA0020082310F4004F4FEA4000F3
:1017E00018BF80F4815003F1FF3318BF80F001006F
:1017F00013F0FF0380B2EFD1A2F87E0138BD0131B2
:101800008B4201BF002385F87C31012385F87D31AF
:1018100038BD00BF382B002010B50446F6F700FB9A
:10182000104AD2F8A83140F6AC51C31A8B42C4BF5B
:10183000002382F8AC3192F8AC31D11881F8AD4177
:1018400023B90F2C0DD10749C1F8A8010133DBB230
:10185000192B044982F8AC310CBF0123002381F815
:10186000C63110BD382B0020094B1A68137844F696
:10187000FB7103EB431300FB03135078C0EB003004
:10188000B3FBF0F39078B3FBF0F080B2704700BF89
:10189000D41A0020124B10B5D3F8C82102EB400136
:1018A0000C7E14B1022C11D00BE0022805D90328BC
:1018B00007D10C4B1B68DB0401D5D08910BD908A81
:1018C00010BD03EB4003B3F8F40010BD487E00EBFD
:1018D000800000EB800000F2EE2080B210BD00BF5F
:1018E000382B00204429002008B5F6F799FA074B59
:1018F000022283F8D021064AC3F8CC011268C3F84B
:10190000DC21012283F8F52108BD00BF382B00201F
:101910006829002008B5F6F783FA084B022283F8FD
:10192000D021D3F8DC2100F5B71000F5587002F291
:10193000DC52C3F8CC01C3F8DC2108BD382B0020F1
:10194000044B1B6842F201021A420CBF0120002026
:10195000704700BF44290020114B93F8F821012A59
:1019600010B51C460ED008D3022A0FD10D4A938A17
:101970009BB283F48853938208E00A4B4FF4885259
:101980001A8503E0074B4FF488529A61F6F748FA3C
:1019900000F5F42000F59070C4F8FC0110BD00BF04
:1019A000382B002000100048022803D0431E584264
:1019B00058417047064B1B681B7823B1054B1868CC
:1019C000C0F3C0407047044B1878C0F380007047E4
:1019D000880600201C120020B72D002010B50A4CEC
:1019E0005E280146206805D15D21F6F713FB2068CB
:1019F0003E2105E05D2903D1F6F70CFB20683D216F
:101A0000BDE81040F6F706BB382D002030B50028A1
:101A1000104C114AB8BF40423C2590FBF2F304FB46
:101A2000030068430D4D90FBF2F22D682D7B25B924
:101A300003EB830303EB830301E0C3EB031302EB2C
:101A400083030B8004FB02024FF47A7392FBF3F2E0
:101A50004A8030BD806967FF80969800DC1A0020BC
:101A600010B50446C0B2FFF7B9FFC4F30720BDE8C4
:101A70001040B3E7024B5E211868F6F7CBBA00BFFF
:101A8000382D002038B5064C05465E212068F6F753
:101A9000C1FA20682946BDE83840F6F7BBBA00BF56
:101AA000382D0020674B73B51878674DFFF77CFF22
:101AB0002B788342044620D0C8B1644B1B68E3B145
:101AC00093F9000002230093614B1B685B7800339D
:101AD00018BF0123019304214FF416530022F8F795
:101AE0001BFF5C4B186040B101232B7005E0594E81
:101AF0003068F8F7F6FE34602C70574B574D187865
:101B0000FFF752FF2B788342044618D088B1544B1C
:101B10001B68A3B10022012493F9000000944FF444
:101B2000964301920821F8F7F7FE4E4B186028B94A
:101B300005E04C4E3068F8F7D4FE34602C704A4B08
:101B40004A4D1878FFF730FF2B78834204462E4623
:101B500042D0002837D0464B1A68002A3CD0D379AF
:101B600092F90000434C002B08BF0223022200928E
:101B7000002254F8233001921021F8F7CDFE3E4B9D
:101B80000546186040B33D4C94F84A30022B0BD008
:101B900094F89620022A01D14C3405E023B1002AA2
:101BA00004F14C0418BF0024354B1C6044B120469E
:101BB00000214C2203F023FC0223256084F84A30E4
:101BC0000123337008E02C4E3068FEF749F9306885
:101BD000F8F787FE34602C702A4B2B4D1878FFF7EE
:101BE000E3FE2B788342044629D000B3274B1B68C1
:101BF0002BB3274A93F9000012685278002A0CBFD1
